:100000000C941C1A0D94A1210D9476210D944B2172
:100010000D9420210D94F5200D94CA200D949F205D
:100020000D9474200C944D1A0C944D1A0C944D1A86
:100030000C944D1A0C944D1A0C944D1A0D94FB3BD4
:100040000C944D1A0C944D1A0C944D1A0C944D1A94
:100050000C944D1A0C944D1A0C944D1A0D94DF1EED
:100060000C944D1A0D9407250D94DD240C944D1A13
:100070000C944D1A0C944D1A0C944D1A0C944D1A64
:100080000C944D1A0C944D1A0C944D1A0C944D1A54
:100090000D94772A0D94ED290D942F2A0D94933DFC
:1000A0000C944D1A0C944D1A0C944D1A0C944D1A34
:1000B0000C944D1A0C944D1A0C944D1A0C944D1A24
:1000C0000C944D1A0C944D1A0C944D1A0D94B324A3
:1000D0000D9489240C944D1A0D945F240D943524AD
:1000E0000C944D1A07634236B79BD8A71A39685645
:1000F00018AEBAAB558C1D3CB7CC5763BD6DEDFD4A
:10010000753EF6177231BF000000803F0800000006
:10011000BE922449123EABAAAA2ABECDCCCC4C3EFC
:1001200000000080BEABAAAAAA3E00000000BF00EB
:100130000000803F0000000000084178D3BB4387E7
:10014000D1133D190E3CC3BD4282AD2B3E68EC82FB
:1001500076BED98FE1A93E4C80EFFFBE01C4FF7F80
:100160003F00000000000C94156A0C9422DF0C94F0
:1001700060EE0D942F1D0C943CFA0C9471AB0C9412
:10018000CC740C94F1AB0D94992F0C940AAB0C9495
:1001900016780C94E3F40C943BA70C9465320C9401
:1001A000A5C20C946E3A0C9406DE0C947FB70C94A6
:1001B00017A10C940A1C0C947DDD0D9494370C94BB
:1001C0001B1B0C94C3750C94E2520D9470050C9497
:1001D000421B0C9440E90C94565F0C9471AA0C9449
:1001E00061320C9493B70C94FEC70C9425760C9452
:1001F00075310D949D1C0C941B680C943A4E0C9414
:1002000076520C94B41B0C948AA70D94F21B0C9498
:1002100034820C946A9B0C94F6DB0C944E530D9430
:10022000891C0C9489C80C9412FA0C945D320C94BD
:1002300025710C9406AB0D942E1D0C949E270D94E5
:10024000A61B0C9491BA0C94E7FE0C94D1310C943B
:100250003F1B0C944AE90C9498F30D94731C0C9476
:10026000B19B0C9451DC0C9432EE0C94A7B70C9417
:100270000E1C0C94E32C0C9417B40C943D330C948A
:100280003EB70C940D680C94366C0C9492370C9419
:1002900016760D941C1C0C94BF670C94A0B50C949E
:1002A0000FB50C944F1A0C94AAAD0D949B300D947D
:1002B000D53A0C94BCFE0C947E640C942A4E0C949B
:1002C00027440C942AAF0C94F61A0C94A4930C9423
:1002D00047B70C94DBB60D94AC2D0C949A200C947B
:1002E000B02D0C9475780D947D1A0C940BFA0D9426
:1002F000511D0C9462A60C94BCB70D94D41D0C94A3
:10030000B21B0C94D2750C945AA70C942A770C94B7
:1003100088A70C948D820C941D320C9404530C9479
:10032000A1A60C944CFF0C945EAB0C9480230C940F
:100330002EFF0C945AB70C94B6440C94EBA60C9474
:1003400063320C94144E0C94C4AB0C941FAB0C94FD
:100350002C6A0C9489470C941AAB0C94B1B70C948A
:100360004DCB0C9451A30C94ED6A0D94D01E0C94BB
:100370006E1B0C943FDC0C9476330C947C1B0D9418
:10038000E1330C94BDF50C94711B0C94ACDF0C9410
:10039000C3A60C946FA60C94B81B0C9407760C940F
:1003A00006B50C9417E70C94581C0C9477AB0C947E
:1003B0004EE90D94911A0D94B41D0C947E460C9444
:1003C00033C90C94AE1B0C9446A60C945F470C9456
:1003D0004D9B0C940D760D9471300C94821D0C94F1
:1003E0009CC90C9456FF0C9494260D942E1C0C94CE
:1003F00019FA0C945CDC0C94D1A10C94C4F30C9409
:1004000091370D94B81C0C94ADA20C94F2440C944A
:10041000116A0D94A2220C9493370C9435FA0C9423
:1004200012AB0C9419EE0C94ACB30C940FF40C9426
:10043000F4360C948AAB0C94FDA20C9450DD0C9411
:100440002E250D943A340C943AE90C94998A0C9424
:10045000A2AD0D9482050C9433E90C94A8F30C948E
:1004600025460D9422330C948C210C9432470C9425
:10047000D3F30C9449A70C94A6530C94549B0C945E
:100480009FDD0C942EA70C9427370C9414A70C9482
:100490004EDC0C9404450C941EAB0C94041B0C9481
:1004A00054770C9499A20C9406770D94A41C0C9488
:1004B000AA3D0D94E3420C94BE530C949DAB0C9456
:1004C00029530C94F5990C9438FF0C94D3FE0C949A
:1004D000B2B30C940BFF0C94FBF30C9442DC0C9421
:1004E00022AB0C9457B10C94E6370C94D3740C9453
:1004F0005CE90D94812F0C9442770C948D5C0D94E3
:10050000351C0C94196A0C9495530C9492250C94F8
:10051000EDB70C94D1200D948C230C9468200D948D
:10052000581D0C94DB290C94BBA50C94E2C20C94CE
:10053000E9A30D94C31B0C946BDE0C942FE90C946F
:10054000304B0C94F7FE0C9404680C9468C30C9424
:1005500013A30C94EFAB0C94A9770D94DA1C0C94B4
:10056000F1F30D94F8420C9491A20C94DDC30C9419
:1005700038B10C9452E90C944F760C94892C0C945D
:1005800093310D94281A0D94251A0C94879F0C947E
:100590002E700D943E1D0D94E41B0D94993A0D940C
:1005A00021370C9428370C945A240C9451B70C948E
:1005B0000C320C9491A60C9420EE0C9409B50C947A
:1005C000815C0C9466B20C9425370C941DDC0C9461
:1005D000EFFE0C94AAC90C9475AB0C9455A70C941F
:1005E0006EA50C940ADC0C94A6A50C94DA5B0C9412
:1005F00057AA0C9490780C9434DC0C94F0A20C94D0
:10060000E5430C9471A60C945BDB0C94DA750C94A6
:1006100095460C9488DF0C9436AA0C94AAC30C94CB
:1006200056440C949CDE0C94F2530C943F6B0C9447
:1006300025E90C94AD460C943A2D0C944B330D9453
:100640006E1A0C94C55B0C94A3A50C94F9710D94CF
:10065000B71C0C94BEB70C944D320C94B6F30C94AA
:1006600011750C9458E90D94B6320C9465AE0C9447
:100670002D310C9414B50C94A0740C94C4FE0C94FD
:1006800065E90C94871B0C9436490C9442FF0C943A
:1006900066A30C94521A0C9416AB0C943AC80C94A2
:1006A000B9B00C94D2F40C947C5C0C9466E90C9474
:1006B000EC2C0C94CEC80C94B7220D9471050C94BC
:1006C00084DF0C94DA3D0C9405F40C94F1680C94DE
:1006D00020DE0C94BA750C94B43A0C94101C0C9453
:1006E00089A50C947F320C9441EE0C94F64D0D9438
:1006F000AC330D94493B0C948BBA0C946E420C9421
:1007000084AA0C941EB40C94E71A0C94B3310C9484
:1007100015FF0C94E9580D94971B0C9498DB0C94DE
:1007200085DE0C94DDF30D946C340C94B01B0D94A9
:100730002D1D0C94E8260C946AE90C94AC1B0D94C6
:100740007F050C948CDF0D9493330C9482BA0C9437
:10075000472D0C94ECF40C94B61B0C94C1260C940D
:10076000D86B0D94AF1C0D94CE1C0C94E4A10C948A
:10077000B3AB0C94A9B30C9426780C94E7F30C94C7
:1007800009A10C9454AB0C9430A60D94851D0D94C6
:10079000D81C0C9426370C9424FF0C9433330C94FF
:1007A000D6A60C9401FF0C945A760C9446750C94C2
:1007B000B7AB0C94DBDD0C9469760D9404340C9487
:1007C00020FA0C9470760D94EC1D0C94C9FE0C94D8
:1007D00034AB0C945E4D0C94C8A20C942EFA0C947D
:1007E00073CB0C9443750C94C5A50C9444760C946F
:1007F00050C90C941E1B0D9452300C94121C0C9476
:100800000CB50C9484F50C94F6200C940C1C0C94F0
:100810004C4E0D948D1C0C940EAB0C9472F50D94F3
:10082000DC2F0C94C2C90C9471530C94E1750C9498
:10083000DDFE0C942C6B0C9460E90C9447300D9405
:10084000381B0C9477EE0C94DAA20C9477C90C94B4
:10085000282F0D94641C0C9437E90C9437DE0C940B
:1008600011C90C94C9AD0C94BFA70C9468A70C9443
:1008700000760D94271A0C94EE6B0C940AA70C9436
:10088000CF3D0C946B380C944BCB0C9442680C9479
:100890002BE90C942D660C94DFA70D94BA320C94BE
:1008A0006CB70D94EB1A0C9403F50C9444E90C947A
:1008B000591A0D94261A0C94AC780C9406B10D9428
:1008C0009F1A4E414E494E495459494E46CDCCCCC3
:1008D0003D0AD7233C17B7D13877CC2B329595E614
:1008E000241FB14F0A000020410000C84200401CF4
:1008F0004620BCBE4CCA1B0E5AAEC59D74636469CB
:100900006E6F70737578585B00432C2052483D0021
:10091000484443313038303A205374617475733D24
:1009200000484443313038303A204E6F7420696EAD
:10093000697469616C697A6564004D7367496E76A4
:10094000616C69640052656164526567496E7661E5
:100950006C6964004D6561734D6F6465496E7661C5
:100960006C6964004D6178526573697374616E637C
:1009700065004865617465724661756C7400486510
:1009800061746572537570706C79004343533831EC
:10099000313A204572726F7220004343533831312F
:1009A0003A204661696C656420746F206765742025
:1009B0004552524F525F49442072656769737465AE
:1009C000722E005D20626173656C696E655B005D0F
:1009D0002074564F435B0020434F325B00636373C8
:1009E0003831313A2064617461206E6F7420617611
:1009F00061696C61626C6500636373383131206ECC
:100A00006F7420696E697469616C697A656400202D
:100A10003C3C0041433A200041433A20536572690F
:100A2000616C2075736564206279204143202D201C
:100A300064697361626C696E672073657269616C69
:100A4000206C6F6767696E6720616E6420636D64F8
:100A50000041433A204F7574206F66206D656D6FBD
:100A600072790041433A20496E69743A200041434B
:100A70003A2044652D496E69743A2000455252006F
:100A800041433A20426164204352430041433A20AB
:100A90004F4B00203E3E200041433A200041433A64
:100AA00020506F6C6C696E670041433A20556E6D43
:100AB000757465000000000000000000004F4E004B
:100AC0000000000000004F464600000000000052F9
:100AD0004553540000000000544F47474C45000068
:100AE0000048414C540000000000584F4E000000E8
:100AF000000000584F46460000000000494E435297
:100B00004541534500444543524541534500454EF8
:100B100041424C4500000044495341424C450000CD
:100B2000554E465245455A4500465245455A4500A0
:100B300000004155544F000000000046414E5F4FF9
:100B40004E4C59004849474800000000004D4544BC
:100B500049554D0000004C4F570000000000004870
:100B60004541540000000000434F4F4C000000007E
:100B70000044525900000000000053544F50000040
:100B80000000005247420000000000004853560099
:100B90000000000000726177007175656974007370
:100BA00077696E67006C6F636B00556E6B6E6F7765
:100BB0006E207375666669782000556E6B6E6F7770
:100BC0006E20636D642000436F756E7465723A2009
:100BD00000444D582D4F757420496E69743A2000B9
:100BE000444D582D4F75742073746F703A20004136
:100BF000737369676E65643A00444D58206374727C
:100C00006C3A2000693136000169333200027531D7
:100C10003600037533320004693868000569386CA2
:100C20000006753868000775386C000878313000A8
:100C300009313030000A44656661756C7420736553
:100C40007269616C206D6F6465204E383120757358
:100C5000656400384531002600384E310006003802
:100C60004532002E00384E32000E00384F3100362B
:100C700000384F32003E00374531002400374532FE
:100C8000002C00374F31003400374F32003C003722
:100C90004E31000400374E32000C00206164646560
:100CA00064206279206E756D20004D4255533A20C4
:100CB00000416464696E67207265677320776974A8
:100CC0006820616374696F6E733A00416464696E91
:100CD0006720726566657272656420726567733A33
:100CE00000416464696E672070726566657463684C
:100CF00020726567733A004D4255533A204D6F6438
:100D00006275732074656D706C617465206E6F74AC
:100D100020666F756E643A20004D4255533A204963
:100D20006E76616C69642074656D706C6174652E9B
:100D3000002C002C002C002C004D4255533A20630F
:100D40006F6E666967206661696C65643A004D4242
:100D500055533A20636F6E666967206572726F72D1
:100D6000004D4255533A20636F6E666967206C6F81
:100D70006164656420004D4255533A204F757420DC
:100D80006F66206D656D6F7279004D4255533A2044
:100D9000506F6C6C696E67206572726F7220004DC7
:100DA0004255533A204E6F7420737570706F727491
:100DB00065642072656720747970650A004D42553C
:100DC00053443A2049676E6F726564202D20657127
:100DD00075616C207769746820736574746564202C
:100DE00076616C004D425553443A204D61707065F8
:100DF000643A004D425553443A204E65737465641D
:100E00004D61707065643A004C6173744B6E6F771E
:100E10006E2076616C75653A200053656172636877
:100E2000696E67207265673A2000206F7574206FC5
:100E3000662072616E6765206275666665722C2039
:100E40006665746368696E670064656620726567CD
:100E50002320004D425553443A2053656172636824
:100E6000696E672072656723003A002066726F6DB5
:100E7000207479706520004D425553443A20206714
:100E80006F7420002076616C3A0020004D4255536B
:100E9000207265733A20002076616C206E6F74209A
:100EA0006368616E6765642E20436F6E74696E754A
:100EB00065004D4255533A003A20657175616C20CA
:100EC000746172676572742E003D004D4255533A4D
:100ED000002076616C206368616E6765642E004D4A
:100EE0004255533A00204E6F773A00204C6173749C
:100EF0003A002023002070726566657463682000E4
:100F0000205265672F636F696C206D757374206262
:100F10006520696E740020696E7465726E616C2064
:100F200073656E64206572726F72202D206E6F2063
:100F30007265672F636F696C0020696E7465726EED
:100F4000616C2073656E64206572726F72202D2053
:100F50006E6F2074656D706C6174650020696E74CD
:100F600065726E616C2073656E64206572726F725B
:100F7000202D206E6F2073746F7265004D425553A3
:100F8000443A20656E64506F6C6C20004D4255539E
:100F9000443A20506F6C6C2000206E6F7420666F96
:100FA000756E64004D4255533A2020706172616D38
:100FB00020002073656E64696E672063616E6365EF
:100FC0006C6C6564004D4255533A2020706172612B
:100FD0006D20004D4255533A2020002073656E6409
:100FE000206572726F722E20004D4255533A2020B8
:100FF000004164642040563A20002056616C3A203B
:10100000004D425553443A207375666669783A003C
:10101000206F722073756666697820004D425553C3
:101020003A204E6F2074656D706C61746520666F38
:101030007220004D6F746F723A2074696D656F7520
:101040007400556E6B6E6F776E20636D64004D6F2C
:10105000746F723A20466F726365642065786563C9
:101060007574696F6E0056454E543A20636F6E6614
:101070006967206661696C65640056454E543A2084
:10108000696E69740056454E543A205049442050C8
:101090003D0056454E543A2044652D496E69740012
:1010A000207365742052455645525345206D6F6438
:1010B000650056454E543A205049443A200020736A
:1010C000657420444952454354206D6F6465005651
:1010D000454E543A205049443A2000206F75743AE6
:1010E00000207365743A0020696E3A0056454E54EC
:1010F0003A2000204F75743A00205265713A00562C
:10110000454E543A2000206D33002066726F6D20EA
:1011100000204D6178207265713A002066616E256D
:101120003A002061637469766520563A0056454E50
:10113000543A20546F74616C20563A004143206148
:1011400069722074656D703A200056454E543A001D
:101150005049443A20616C726561647920696E6916
:101160007469616C697A6564005049443A20496E3B
:1011700076616C696420706172616D206172726168
:10118000792E002C002C002C002C005049443A20D1
:10119000636F6E666967206661696C65643A0050CA
:1011A00049443A20636F6E666967206572726F7298
:1011B000005049443A20636F6E666967206C6F6126
:1011C00064656420005049443A204F7574206F666E
:1011D000206D656D6F7279005049443A2044652D49
:1011E000496E69742000203C414C4D3E0020443A39
:1011F0000020493A0020503A0020696E3A002073DE
:1012000065743A005049443A20005049443A204914
:101210006E76616C696420706172616D20617272BA
:1012200061792E00536574206F757420746F2000EF
:101230002050494420616C61726D2E20002050497D
:101240004420616C61726D3A20636C6F7365640059
:101250005049443A20556E6B6E6F776E20737566F9
:1012600066697820005049443A20556E6B6E6F775E
:101270006E20636D64200020536574706F696E7416
:101280003A005049443A200020496E707574207627
:10129000616C75653A005049443A200020696E69D6
:1012A0007400200050574D2D4F757420230020737B
:1012B000746F7000200050574D2D4F75742023001F
:1012C0003D0050696E3A0020696E69740070696E65
:1012D000230072656C61794374723A200020737444
:1012E0006F700052656C61792D4F75742023007208
:1012F000656C61794374723A200020697320004F55
:101300007574200072656C61794374723A200055DF
:101310006E6B6E6F776E20737566666978200072EB
:10132000656C61794374723A2000556E6B6E6F770D
:101330006E20636D64200072656C61794374723A4B
:101340002000616374696F6E0072656C617943742B
:10135000723A200053686F770020636D643D002D62
:10136000005B305D3A2000202D202D202D20EFBB8A
:10137000BF003E003E31202D200000000000006331
:101380006D640000736574000076616C0000646534
:101390006C00004853560000524742000066616EE0
:1013A00000006D6F6465006374726C0068756500A1
:1013B00000736174000074656D70007261770000E5
:1013C00020002E00696E00735F6F7574006D796880
:1013D0006F6D65004354524C2F657865633A204F1A
:1013E00075744F664D656D6F72793A2000202D3E01
:1013F00020004D5154543A2000202D3E2000456DD0
:1014000069743A203C00202D3E20004974656D43EC
:101410006D643A2000202D3E20004974656D3A200D
:1014200000206661696C65643A004D6F6462757393
:10143000206F7020004D423A206F6B003D004D42FE
:101440003A205643230020636D643D003D004D4229
:101450003A2056435F6865617423004D423A204E3E
:101460006F7420737570706F727465642072656735
:1014700020747970650A002056616C3A307800203B
:10148000543A00205265673A3078004D423A204184
:101490006464723A00444D58000000000000444D5E
:1014A00058524742570000444D58524742000000EE
:1014B00050574D0000000000004D42555344494D27
:1014C0000000544845524D4F00000052454C4159D0
:1014D0000000000047524F55500000000056435492
:1014E000454D500000004D42555356430000004109
:1014F00043484149455200005350494C454400007F
:10150000004D4F544F52000000005049440000006D
:101510000000004D42555300000000005541525458
:10152000425244470052454C415950574D00444D9A
:101530005852474257570056454E5453000000003A
:10154000454C455641544F5200434F554E54455219
:10155000000048554D0000000000004D4552435525
:101560005259000020002D3E00436F6E7665727464
:10157000696E6720002D3E0057726F6E67204173C1
:101580007369676E6D656E742000524742783A2029
:101590000020764C6576656C3A0020436F6E765677
:1015A0003A0020436F6E76533A0020486F743A0039
:1015B000436F6C643A0020436F6E766572746564A5
:1015C00020563A00436F6E76657274656420533A14
:1015D000002D3E0057726F6E672041737369676E0E
:1015E0006D656E7420002D3E0057726F6E6720414E
:1015F000737369676E6D656E7420004D41503A20BB
:1016000076616C206D617070656420746F202000BD
:101610004D41503A2076616C75652061626F766548
:1016200020726967687420626F756E64200020699B
:10163000732062656C6F77206C65667420626F75CD
:101640006E6420004D41503A2076616C7565200033
:101650004D41503A20636D64206D61707065642067
:10166000746F20000000000000000000004F4E00DA
:101670000000000000004F4646000000000000523D
:101680004553540000000000544F47474C450000AC
:101690000048414C540000000000584F4E0000002C
:1016A000000000584F46460000000000494E4352DB
:1016B0004541534500444543524541534500454E3D
:1016C00041424C4500000044495341424C45000012
:1016D000554E465245455A4500465245455A4500E5
:1016E00000004155544F000000000046414E5F4F3E
:1016F0004E4C59004849474800000000004D454401
:1017000049554D0000004C4F5700000000000048B4
:101710004541540000000000434F4F4C00000000C2
:101720000044525900000000000053544F50000084
:1017300000000052474200000000000048535600DD
:10174000000000000020537566663A002041543ABC
:101750000052453A2064656C657465640053746F8B
:101760007070696E6720496E7075747300206973BC
:10177000200044656C6574696E6720636F6E662E29
:101780002052414D207761733A0053746F70706539
:1017900064006E6F7468696E6720746F2073746F75
:1017A000700053746F7070696E67206368616E6E4D
:1017B000656C73202E2E2E0043616E206E6F742098
:1017C000636C65616E202D206C6F636B6564004DEA
:1017D0005154543A20436F6D706C6574652E2052DD
:1017E000656D6F766520746F706963200024636F88
:1017F0006D6D616E64004D5154543A20436C6561C7
:101800006E55702072657461696E656420746F70C6
:1018100069632000220022004F75744F664D656D8C
:101820006F727921005D20003A5B004D5154543AAB
:10183000005D00456D7074793A205B000A003A0043
:101840004D41433A00554450205379736C6F6720E3
:10185000696E697469616C697A65642E0A005379EE
:10186000736C6F6720706172616D733A002E6C6FDC
:1018700063616C0053657276696365207265636F9E
:1018800072643A20006D444E5320726573706F6E1F
:1018900064657220737461727465642E004572729F
:1018A0006F722073657474696E67207570204D4483
:1018B0004E5320726573706F6E6465722100476FBE
:1018C0007420495020616464726573733A0027691B
:1018D00070205B69705B2C646E735B2C67775B2C8C
:1018E0007375626E65745D5D5D5D27202D20736587
:1018F00074207374617469632049500A00466169F9
:101900006C656420746F20636F6E666967757265BD
:101910002045746865726E6574207573696E672002
:10192000444843502E20596F752063616E207365C3
:1019300074206970206D616E75616C6C7921002076
:101940004D41534B3A002047573A0020444E533AFA
:10195000004C6F616465642066726F6D20666C6117
:1019600073682049503A000A7573657320444843F0
:10197000500A005374617274696E67206C616E0066
:101980004D5154543A2074727969796E67206E65AE
:101990006E78742062726F6B6572004D5154543AC8
:1019A00020546F6F206D616E7920636F6E6E65637A
:1019B00074696F6E206572726F72732E2052657338
:1019C00074617274204C414E0020747279206167FA
:1019D00061696E20696E2035207365636F6E647374
:1019E000004D5154543A206661696C65642C207234
:1019F000633D004D5154543A204177616974696EDA
:101A00006720666F722072657461696E6564207408
:101A10006F7069637300636F6E6E656374656420D5
:101A200061732000202E2E2E0020757365723A00FF
:101A30003A000A4D5154543A20417474656D7074E3
:101A4000696E6720636F6E6E656374696F6E207474
:101A50006F2000646973636F6E6E65637465640004
:101A60005573696E67204D515454207061737377BC
:101A70006F72642066726F6D20636F6E66696700B7
:101A80002E6C6F63616C006D444E53206E616D650A
:101A900020757064617465643A20004465766963FA
:101AA00065204E616D653A004D5154543A204174A1
:101AB000206C6561737420646576696365206E616E
:101AC0006D6520616E642062726F6B657220495093
:101AD000206D75737420626520636F6E666967752B
:101AE00072656400246E6F646573004F4E2C4F4620
:101AF000462C48414C542C524553542C584F4E2C94
:101B0000584F46462C544F47474C450024666F7249
:101B10006D617400656E756D002464617461747923
:101B200070650068737600636F6C6F7200302D32E1
:101B3000353500696E746567657200666C6F617437
:101B400000332E302E310024686F6D69650075708A
:101B500074696D652C6672656568656170003837FB
:101B600035346133355F323032352D30342D3330FA
:101B7000004C696768744875622000246E616D6569
:101B800000526562696E6420737563636573732EBA
:101B900020495020616464726573733A0045727223
:101BA0006F723A20726562696E64206661696C00CA
:101BB00052656E6577656420737563636573732E14
:101BC00020495020616464726573733A00457272F3
:101BD0006F723A2072656E65776564206661696C24
:101BE000000A4E6F206C696E6B00436F6E74696EF5
:101BF000756520776974682070726576696F757392
:101C00006C79206C6F6164656420636F6E666967D0
:101C10000033307320454550524F4D206973206E7C
:101C20006F742072656C6F616465642E205265620A
:101C30006F6F74004D5154543A2041636365707462
:101C4000696E6720636F6D6D616E64732E2E2E0A50
:101C5000004E6F204D51545420636F6E6669677556
:101C6000726564004C6F6164696E6720636F6E66B5
:101C700069672066726F6D20706F7274616C20648A
:101C8000697361626C65642E207573652067657485
:101C9000204F4E20746F20656E61626C6500436F4B
:101CA0006E6669672069732076616C696400436FB2
:101CB0006E74696E756520776974682070726576D8
:101CC000696F75736C79206C6F6164656420636FF4
:101CD0006E666967005365747570204F5441004DFE
:101CE0005154543A2073657420666972737420628B
:101CF000726F6B65720043757272656E74204C4131
:101D00004E20636F6E6669672869702C646E732C51
:101D100067772C7375626E6574293A000A5573658E
:101D200020746865736520636F6D6D616E64733ACE
:101D3000202768656C7027202D20746869732074D3
:101D40006578740A276D61632064653A61643A625C
:101D5000653A65663A66653A3030272073657420C7
:101D6000616E642073746F7265204D41432D616410
:101D7000647265737320696E20454550524F4D0A59
:101D8000276970205B69705B2C646E735B2C6777CE
:101D90005B2C7375626E65745D5D5D5D27202D2023
:101DA000736574207374617469632049500A2773E2
:101DB00061766527202D20736176652063757272C8
:101DC000656E7420636F6E66696720696E204E567B
:101DD00052414D3B204F4E7C4F4646202D20656E94
:101DE00061626C652F64697361626C6520617574F2
:101DF0006F736176650A2767657427205B636F6E72
:101E000066696720616464725D27202D20676574B0
:101E100020636F6E6669672066726F6D20707265F1
:101E20002D636F6E666967757265642055524C202C
:101E3000616E642073746F726520616464722C201B
:101E40004F4E7C4F4646202D20656E61626C652F9B
:101E500064697361626C6520646F776E6C6F616436
:101E6000206F6E20737461727475700A276C6F61D5
:101E70006427202D206C6F616420636F6E66696734
:101E80002066726F6D204E5652414D0A277077645E
:101E900027202D20646566696E6520616E6420735D
:101EA000746F7265204D5154542070617373776F55
:101EB00072640A276F746170776427202D2064652F
:101EC00066696E6520616E642073746F7265204868
:101ED000545450204150492070617373776F72647D
:101EE0000A276C6F67205B73657269616C5F6C6F4A
:101EF000676C6576656C5D205B7564705F6C6F67A1
:101F00006C6576656C5D27202D20646566696E655D
:101F1000206C6F67206C6576656C2028302E2E371C
:101F2000290A276B696C6C27202D20746573742037
:101F30007761746368646F670A27636C65617227F1
:101F4000202D20636C65617220454550524F4D0A2B
:101F50002773656172636827202D20736561726342
:101F60006820312D77697265206465760A2772656D
:101F7000626F6F7427202D207265626F6F7420630B
:101F80006F6E74726F6C6C657200536F6674207242
:101F900065626F6F74696E672E2E2E00206E6577F6
:101FA0000020697320003157543A003157543A20C9
:101FB000536561726368696E67206465760052419B
:101FC0004D3D000A5379736C6F6720000A312D77FD
:101FD00069726520000A6D71747420000A6D6F6467
:101FE000627573207632000A6D6F646275732076B5
:101FF0003120282B29000A696E7075747320000A3D
:102000006974656D7320000A436F6E666967757247
:1020100065643A00204D6F64653A0052453A20638A
:102020006F6E66696775726564206F6E2070696E89
:102030007320002F00496E3A2000496E697469616F
:102040006C697A696E6720496E70757473003157D8
:10205000543A207365747570207265736F6C757473
:10206000696F6E20003157543A204453323438326D
:102070002D313030206E6F742070726573656E7410
:10208000003157543A204453323438322D313030F5
:102090002049324320726573746F72656400315752
:1020A000543A2042757320726573657420657272AC
:1020B0006F72003157543A20427573205265736530
:1020C0007420646F6E65003157543A2044533234A3
:1020D00038322D3130302070726573656E742C206B
:1020E0007265736574004572726F7220312D7720AE
:1020F000696E6974003157543A204453323438328F
:102100005F3130305F4932435F544F5F31575F4238
:10211000524944474520696E697400444D584F75D3
:10212000742E20467265653A00444D58696E20420F
:10213000756666657220616C6C6F632065727200F3
:10214000496E697420696E2063683A003B003D0067
:1021500050696E3A003B003D4C4F57005468657221
:102160006D6F3A004F6E6520776972652052656128
:1021700064790A00467265653A00444D58206F75CF
:102180007420737461727465642E204368616E6E8E
:10219000656C733A2000444D5820696E2073746159
:1021A000727465642E204368616E6E656C733A00CC
:1021B00042726F6B65727320636F6E6669677572CA
:1021C00065643A004170706C79696E6720636F6E68
:1021D000666967004C6F6164656420455441473A05
:1021E000004E6F2073746F72656420636F6E666952
:1021F00067004C6F616465642066726F6D204545B1
:1022000050524F4D006C6F6164206661696C65646B
:10221000004A534F4E206465746563746564004CD6
:102220006F6164696E6720436F6E666967206672CE
:102230006F6D20454550524F4D00436F6E66696784
:10224000206175746F736176653A000A5379736C17
:102250006F67206465627567206C6576656C3A000F
:1022600053657269616C206465627567206C657680
:10227000656C3A0053617665640A005365742064A6
:10228000796E616D69632049500A004F54412050B6
:10229000617373776F726420757064617465640A2A
:1022A000004E6F20495020616472657373002053A3
:1022B00061766564004C6F6164696E6720485454B0
:1022C0005020636F6E666967206F6E207374617251
:1022D0007475703A000000000000000000004F4ECE
:1022E000000000000000004F464600000000000013
:1022F000524553540000000000544F47474C4500DE
:10230000000048414C540000000000584F4E0000AF
:1023100000000000584F46460000000000494E43B0
:1023200052454153450044454352454153450045BC
:102330004E41424C4500000044495341424C450047
:1023400000554E465245455A4500465245455A4568
:102350000000004155544F000000000046414E5F10
:102360004F4E4C59004849474800000000004D4579
:102370004449554D0000004C4F570000000000003C
:10238000484541540000000000434F4F4C000000FE
:10239000000044525900000000000053544F500008
:1023A0000000000052474200000000000048535661
:1023B000000000000000636F756C64206E6F742075
:1023C00070617273653A2000557064617465640AC7
:1023D00000454550524F4D20636C65617265640A3B
:1023E000004D5154542050617373776F726420759F
:1023F0007064617465640A002B002D0045546167A8
:102400003A200047657420455441473A200048541B
:1024100054502F312E310025733A2025730D0A00B8
:1024200020485454502F312E310D0A486F73743A9E
:102430002025730D0A4163636570743A202A2F2AA0
:102440000D0A436F6E6E656374696F6E3A20636C3C
:102450006F73650D0A0025730020000D0A004745C3
:1024600054006661696C656420746F20636F6E6EE2
:102470006563740A004552524F523A205365727692
:1024800065722072657475726E65642000436F6EAC
:10249000666967206E6F74206368616E6765640AA1
:1024A00000446F6E652E0A00436F6E666967207088
:1024B000617273696E67206661696C65640A0047C2
:1024C00065742061626F7274656400676F74204385
:1024D0006F6E6669670A0068747470207265746351
:1024E0006F64652000667265652000436F6E6669E3
:1024F00067205552493A20687474703A2F2F002093
:1025000044656661756C7420636F6E6669672073DD
:10251000657276657220757365643A20006C617A25
:1025200079686F6D652E7275000A282D29435259FE
:102530005054000A282D2950554C5345206F6E20C9
:1025400050494E3132000A282D2943414E000A28B5
:102550002D294D455243555259000A282B294D55D6
:102560004C544956454E54000A282B2950574D5F6C
:1025700052454C4159000A282B294D444E53000A1C
:10258000282D2955415254425249444745000A28B2
:102590002B295359534C4F47000A282B29504944A3
:1025A000000A282D294D43503233303137000A2894
:1025B0002D294152544E4554000A282D294F54418B
:1025C000000A282B29535049204C4544000A282B47
:1025D000294D4F544F5220435452000A282B294171
:1025E00043204841494552206F6E2053657269610E
:1025F0006C33000A282B29434353383131202620DD
:1026000048444331303830000A282B29524553546E
:102610004152545F4C414E5F4F4E5F4D5154545F99
:102620004552524F5253000A282D294841524452D4
:10263000455345542C207573696E6720736F66741B
:10264000000A282B29434F554E544552000A282B87
:1026500029444854000A282B294453323438322D57
:10266000313030000A282B294F57495245000A289B
:102670002D2949504D4F44425553000A282B294DCE
:102680004F444255532030783036206174205365D2
:102690007269616C322073706565643A3936303026
:1026A000000A282B294144414652554954204C45A3
:1026B00044000A282B29444D58000A282B29576921
:1026C0007A6E657435313030000A282B29467265E0
:1026D0006552616D207072696E74696E67000A28B8
:1026E0002B295741544348444F47006C617A79681D
:1026F0006F6D652E7275000A436F6E666967207391
:1027000065727665723A003230313130334C0020D8
:10271000432B2B2076657273696F6E3A003837351C
:10272000346133355F323032352D30342D33300063
:102730000A4C617A79686F6D652E7275204C6967F5
:10274000687448756220636F6E74726F6C6C65722A
:102750002000204F464600204F4E00204259504155
:10276000535300536176656420746F204545505281
:102770004F4D00536176696E6720636F6E666967BF
:1027800020746F20454550524F4D2E2E0043435329
:102790003831313A20416C726561647920696E6923
:1027A0007469616C697A6564004343533831313A26
:1027B00020496E6974206572726F72200043435322
:1027C0003831313A20496E69740048444331303819
:1027D000303A20416C726561647920696E69746970
:1027E000616C697A65640044657669636520536548
:1027F0007269616C204E756D6265723D00204465A2
:10280000766963652049443D3078004D616E756698
:10281000616374757265722049443D3078004844A4
:1028200043313038303A20496E69742E2000696493
:102830006C65006F66660068656174696E67006646
:10284000616E00647279696E6700636F6F6C696EA8
:102850006700616374696F6E00556E6B6E6F776EA3
:10286000207375666669782000556E6B6E6F776EA3
:1028700020636D642000636C724374723A200045DB
:102880004F46002500C2B04320483D002044485434
:10289000323220747970652E20543D00494E3A0042
:1028A000204E6F20656D6974206461746121002081
:1028B000436F756E74657220747970652E20766131
:1028C0006C3D00494E3A0020436F756E746572206E
:1028D000747970652E20494E434F5252454354201F
:1028E000496E74657272757074206E756D62657272
:1028F000212121004952513A004163746976617483
:102900006520696E20004163746976617465206991
:102910006E20002D3E00200023002D3E00200050A0
:10292000656E6465643A2023003D00494E3A003DDF
:10293000004C454741435920494E3A0020666F728A
:1029400020286D73293A004354524C3A205363684F
:102950006564756C6520636D642000206D730020D4
:10296000666F7220004354524C3A2041726D656488
:1029700020002044697361726D6564004354524CB9
:102980003A20002074696D653A004354524C3A2055
:102990005265733A002054533A0020543A00544888
:1029A00045524D3A00436C65616E696E6720616CFB
:1029B00061726D20003D0050696E3A004354524CE4
:1029C0003A20436F6D6D616E6420626C6F636B655E
:1029D0006420627920647269766572004354524CB7
:1029E0003A204F4E3A416C726561647920416374BC
:1029F0006976650A004354524C3A2048414C543A97
:102A0000416C726561647920496E616374697665B1
:102A10000A004354524C3A20584F4E3A20446973AE
:102A200061626C65640A004354524C3A20584F4E20
:102A30003A416C7265616479204163746976650A14
:102A4000004354524C3A20584F464620736B6970ED
:102A50007065642E205072657620636D643A004381
:102A600054524C3A205475726E6564206F6666202D
:102A700066726F6D3A004354524C3A20526573743B
:102A80006F7265642066726F6D3A004354524C3A1F
:102A90002049676E6F7265642C206368616E6E6595
:102AA0006C20636D643D0020457865633A004354B3
:102AB000524C3A204163746976653A004354524C53
:102AC0003A2048414C543A416C726561647920491E
:102AD0006E6163746976650A004354524C3A20581B
:102AE0004F4E3A2044697361626C65640A00435436
:102AF000524C3A20584F4E3A416C726561647920CD
:102B00004163746976650A004354524C3A20584F29
:102B1000464620736B69707065642E20507265762E
:102B200020636D643A004354524C3A205475726EDF
:102B30006564206F66662066726F6D3A004354527A
:102B40004C3A20526573746F7265642066726F6DC3
:102B50003A0044697361726D696E67206E6F74200C
:102B6000617574686F72697A6564004354524C3AB7
:102B700020636F6D6D616E64206A75737420666F7B
:102B80007220004354524C3A204E6F7420656E6F91
:102B9000756768206D656D6F727920666F7220674A
:102BA000726F7570206F7065726174696F6E004925
:102BB0006E76616C69642061726700496E76616C43
:102BC00069642061726700496E76616C6964206196
:102BD0007267004354524C3A20556E6B6E6F776E9D
:102BE0002073756666697800536B697070696E67EB
:102BF000207363686564756C65642067726F7570B7
:102C00002065786563004354524C3A206368616ED6
:102C10006E656C2066726F7A656E004354524C3A52
:102C2000206368616E6E656C2066726F7A656E00F7
:102C3000536B697070656420686F6D69652073748B
:102C4000756666002000205375623D00204974655A
:102C50006D3D004354524C3A2052414D3D00435487
:102C6000524C3A204F75744F664D656D6F72793ACC
:102C70002000282D292000282B2920002076616C97
:102C80007565206973200020756E6B6E6F776E0A14
:102C9000005D3D005B0020696E76616C6964002018
:102CA000004143544956453A00206F6B003A0020DA
:102CB0006661696C6564003A005265747279696E88
:102CC0006720564354454D5020434D440A005265F9
:102CD000747279696E6720564320434D440A00524E
:102CE00065747279696E67206D6F646275732043D5
:102CF0004D440A005265747279696E6720434D44F1
:102D00000A00206572726F723D004D423A20706F6A
:102D10006C6C696E6720002056616C3A20004D4251
:102D20003A20004D423A204E6F7420737570706FD8
:102D3000727465642072656720747970650A004D4D
:102D4000423A20706F6C6C696E672064696D6D65C6
:102D50007220004D423A20496C6C6567616C2061BD
:102D60007267756D656E74730A00206572726F729A
:102D70003D004D423A20706F6C6C696E672050497F
:102D800020002D004D423A2050492056616C203AD7
:102D9000004D423A20706F6C6C696E67205049207C
:102DA000004D423A20706F6C6C696E6720464D2072
:102DB0006661756C742000206572726F723D004D03
:102DC000423A20706F6C6C696E6720002D004D4296
:102DD0003A20464D2056616C203A004D423A207010
:102DE0006F6C6C696E6720464D20004354524C2F27
:102DF000706F6C6C3A204F75744F664D656D6F72D5
:102E0000793A2000207365632072656D61696E698F
:102E10006E670053746174757320646566666572CD
:102E200065640A002D3E005075623A20002D3E0078
:102E30005075623A20002D3E005075623A20000025
:102E400000000000636D640000736574000076612B
:102E50006C000064656C0000485356000052474205
:102E6000000066616E00006D6F6465006374726CD3
:102E7000006875650000736174000074656D700012
:102E800072617700002D3E005075623A20002D3EA1
:102E9000005075623A200053454E445354415455F6
:102EA000533A20556E6B6E6F776E20636D64200A07
:102EB000000000000000000000004F4E0000000075
:102EC0000000004F464600000000000052455354E9
:102ED0000000000000544F47474C450000004841A7
:102EE0004C540000000000584F4E0000000000004D
:102EF000584F46460000000000494E43524541539A
:102F00004500444543524541534500454E41424CDE
:102F10004500000044495341424C450000554E468F
:102F20005245455A4500465245455A450000004124
:102F300055544F000000000046414E5F4F4E4C5923
:102F4000004849474800000000004D454449554DA0
:102F50000000004C4F57000000000000484541545D
:102F60000000000000434F4F4C000000000044529E
:102F70005900000000000053544F500000000000B2
:102F80005247420000000000004853560000000075
:102F9000000000002200250028002B002E00310038
:102FA000340002010000050108010B0100002000AF
:102FB0002300260029002C002F0032000001000011
:102FC00003010601090100000A0B02090C0D0E089D
:102FD00007030401000000000000000000000000E2
:102FE00000000000000000000000000000000000E1
:102FF000000012111000000000000000000000009E
:103000000000000000000000000000004D42555389
:103010003A204164642040533A20000000210024FB
:103020000027002A002D00300033000101000004B9
:103030000107010A01010210202008081020401099
:10304000204080020102010804020101020408106C
:10305000204080804020100804020180040201808A
:1030600040201008040201080402010102040810B3
:103070002040800102040810204080050505050756
:103080000508080808020202020A0A0808040404E3
:10309000040101010101010101030303030303030F
:1030A00003040707070C0C0C0C0C0C0C0C0202029E
:1030B0000206060606060606060B0B0B0B0B0B0B91
:1030C0000B556E737065636966696564206572721D
:1030D0006F722E0047454E455249435F4552524F4D
:1030E0005200494E5445524E414C5F4552524F5248
:1030F000004932435F4552524F520049445F4552A6
:10310000524F5200535543434553530043435338A2
:1031100031313A200057726F6E67207061796C61AF
:1031200064004D5154543A204354524C2F747874D7
:103130003A204F75744F664D656D6F72793A200075
:10314000202D3E2041543A004368616E207479700E
:10315000653A004E6F2073746F7265642076616CFF
:10316000756573202D2064656661756C743A200066
:10317000536176656420455441473A005365742095
:10318000455441473A20003157543A204275732044
:103190007265736574206572726F72003157543AAC
:1031A0002042757320526573657420646F6E6500EC
:1031B0003157543A20445332343832207072657398
:1031C000656E742C20726573657400493243205219
:1031D0006573657400005EBCE2613FDD83C29C7E66
:1031E00020A3FD1F419DC3217FFCA2401E5F01E380
:1031F000BD3E6082DC237D9FC1421CFEA0E1BF5D1D
:103200000380DE3C62BEE0025CDF81633D7C22C065
:103210009E1D43A1FF4618FAA427799BC584DA387E
:1032200066E5BB5907DB856739BAE406581947A537
:10323000FB7826C49A653BD987045AB8E6A7F91BE0
:1032400045C6987A24F8A6441A99C7257B3A64861D
:10325000D85B05E7B98CD2306EEDB3510F4E10F24A
:10326000AC2F7193CD114FADF3702ECC92D38D6FE7
:1032700031B2EC0E50AFF1134DCE90722C6D33D1B4
:103280008F0C52B0EE326C8ED0530DEFB1F0AE4CCD
:103290001291CF2D73CA947628ABF517490856B40E
:1032A000EA6937D58B5709EBB536688AD495CB29AF
:1032B00077F4AA4816E9B7550B88D6346A2B759768
:1032C000C94A14F6A8742AC896154BA9F7B6E80A95
:1032D00054D7896B35436F6E6E65637465642E00D9
:1032E000436F6E6E2E2061626F72746564003E3EA5
:1032F0002000496E76616C696420636F6D6D616E4C
:1033000064003E3E3E004E6F204D414320636F6E91
:10331000666967757265643A2073657420666972C0
:103320006D776172652773204D41430A0045455012
:10333000524F4D207369676E6174757265206F6BB3
:1033400000496E697469616C697A696E67204545E8
:1033500050524F4D2E002072656164206572726F6D
:103360007220666F7220003E2000203C00315754CE
:103370003A003157543A206E6F7420696E697400B8
:103380003157543A20425553592074696D656F7511
:1033900074003157543A204453323438325F455226
:1033A000524F525F434F4E464947003157543A20DF
:1033B000312D776972652073686F7274656400726D
:1033C0006561647900247374617465007570746953
:1033D0006D6500667265656865617000247374616F
:1033E00074730020457870697265640A00202D743A
:1033F0006172676574207A6F6E652D0020416C6183
:10340000726D20457870697265640A0020636D648E
:103410003A00204375723A00205365743A002054F4
:10342000696D65723A00204C6F636B733A005241CC
:103430004D3D0000B102590211241FBECFEFD1E271
:10344000DEBFCDBF00E00CBF1AE0A0E0B2E0E0E4D8
:10345000F1EC02E00BBF02C007900D92A638B10755
:10346000D9F722E1A6E8BAE001C01D92AF3BB2074E
:10347000E1F71AE1CBE1DAE100E006C021970109AA
:10348000802FFE010F946458CA31D10780E00807ED
:10349000A9F70F9452470D948E600C94000090E0B1
:1034A00080E00895DC01ED91FC910284F385E02D2C
:1034B0001994DF92EF92FF920F931F93CF93DF93B4
:1034C000EC010C891D890115110559F01D8A1C8A12
:1034D000C801DF91CF911F910F91FF90EF90DF9086
:1034E0000895EC85FD858E859F85DF01A80FB91FA6
:1034F0002C91243209F055C011962C912B3709F0EC
:1035000050C00296E80FF91FF12CE12CDF01D19099
:10351000DD2009F446C08DE7D816E9F08FEFE81AF0
:10352000F80AF4CF198A188A2C853D8521153105B2
:1035300079F08E859F85280F391FF901208122237C
:1035400021F001969F878E873EC01D861C86C0CFC6
:103550000FEF1FEFBDCFE114F10419F11C928E851E
:103560009F8502966C857D85680F791FE881F981BA
:103570000684F785E02DCE011995998B888B1B8ADF
:103580001A8AEC85FD858E859F85E80FF91FEE0D63
:10359000FF1DD2828E859F850396E80EF91EFF8659
:1035A000EE86288939892115310509F4BDCF8A892C
:1035B0009B89280F391FF9012081222309F4B2CFFA
:1035C00001969B8B8A8B022F220F110B81CFDC017E
:1035D0001C96ED91FC911D971E968D919C91E80F84
:1035E000F91F8081082E000C990B0895DC011596B7
:1035F0008D919C91009739F0DC01ED91FC91068052
:10360000F781E02D19940895FC01838594859C0130
:1036100044E0359527954A95E1F756E095958795CD
:103620005A95E1F72817390719F081E090E00895DD
:1036300082E090E0089583E090E00895DC01129626
:10364000ED91FC9113973097B9F016968D919C915E
:103650008430910541F08530910541F0039749F49C
:1036600082E090E0089581E090E0089581E190E0AB
:103670000895828590E0089590E080E0089585E0C7
:1036800090E008958EE090E00895CF93DF93FC01E1
:10369000C681D78180858F70853079F08630E1F4DE
:1036A0002097D1F0E881F981309719F080818F7BE4
:1036B00079F40A80DB81C02DF3CF209769F0CE0129
:1036C0000E94451B811105C00A80DB81C02DF5CF0A
:1036D00081E0DF91CF91089580E0FBCF84E190E01D
:1036E0000895DC01ED91FC910484F585E02D60E006
:1036F000199581E090E00895DC011496ED91FC911C
:1037000080E0309711F085A1817090E00895CF930B
:10371000DF93EC0160EE7BE089E390E10F94E4231A
:10372000EA81FB810280F381E02D6081718189E370
:1037300090E10F94CE2389E390E10F947822E88101
:10374000F9810484F585E02D60E0CE01199581E0D2
:1037500090E0DF91CF9108950D94114F0D94114F8A
:103760000D94114F0D94114F0D94114F0D94114F55
:10377000EF92FF920F931F93CF93DF938C0162E937
:1037800070E189E390E10F94E42389E390E10F94E1
:103790007822D8011496ED91FC91309749F1C681B9
:1037A000D781209729F1E881F9813097E9F080816C
:1037B0008823D1F065E775E0CE010E943AED7C01E7
:1037C000009791F0FC0181859285A385B4850097CF
:1037D000A105B10549F00F94114FD70119961D921B
:1037E0001D921D921C921C970A80DB81C02DD9CF9F
:1037F000D801ED91FC910484F585E02D60E0C801CD
:10380000199581E090E0DF91CF911F910F91FF908A
:10381000EF9008950D94114F0D94114F0D94114F89
:103820000D94114FEF92FF920F931F93CF93DF935D
:10383000EC018B018091900A9091910A0097A9F078
:10384000FC0120852F70263081F40E943AEDFC01A6
:1038500090859F70943049F481859285DF91CF9156
:103860001F910F91FF90EF900895EE88FF88C70198
:1038700001970D97D0F469E775E0C8010F94D15C0A
:10388000892B99F48FE2888F85E08E9DB0018F9D02
:10389000700D112466587C4E46E050E0CE014996EA
:1038A0000F94E550CE014896D9CF90E080E0D6CF76
:1038B0004F925F926F927F92BF92CF92DF92EF9280
:1038C000FF920F931F93CF93DF9300D000D0CDB71B
:1038D000DEB77C01B62E80918D0A882309F4BDC025
:1038E000D70114969C9180914402891708F4B5C0C1
:1038F0008091EC0A9091ED0ABAE06B13EFC0845608
:10390000954FFC011082D70118960D911C9101155D
:10391000110509F49EC0F801618572856115710574
:1039200091F445805680678070848091790D9091E4
:103930007A0DA0917B0DB0917C0D481659066A0650
:103940007B0609F486C0D8011B964D915C911C97AB
:103950004115510509F47DC0F701248153968C91DE
:10396000539790E0322F377002C0959587953A951E
:10397000E2F780FF6EC0C22ED12CC601887F937003
:10398000892B39F451968D919C91887F9370C82A28
:10399000D92AD8018D919C91DC01ED91FC916115A2
:1039A000710509F485C00688F789E02D19950197FE
:1039B00009F04FC06CE3F801808191810F943623A8
:1039C0004AE050E0B601D8018D919C910F94952268
:1039D000F80122818081918164E773E1222311F053
:1039E00062E773E10F94E423D8011D966D917C91F9
:1039F0001E978D919C910F94CE2360E2F8018081F7
:103A000091810F943623D8011F966D917C91509728
:103A10008D919C910F94CE23F80122818081918118
:103A200067E673E1222311F061E673E10F94E4236A
:103A30006CE97AE0D8018D919C910F94CE23F80126
:103A400080819181DC01ED91FC91008CF18DE02D64
:103A500019951092ED0A1092EC0AD70115968D91E6
:103A60009C911697009771F014963C912091450215
:103A7000231740F0DC01ED91FC910190F081E02DE5
:103A80006B2D199581E090E026960FB6F894DEBF75
:103A90000FBECDBFDF91CF911F910F91FF90EF909F
:103AA000DF90CF90BF907F906F905F904F90089580
:103AB0000488F589E02D20E535E03A832983D80193
:103AC00015964D905D906D907C9018974B825C821E
:103AD0006D827E82BE016F5F7F4F68CF8F3491050C
:103AE0000CF0BBCFBDE06B1709F4B7CF9C012F5F83
:103AF0003F4F3093ED0A2093EC0A8456954FFC011A
:103B00006083ABCF2F923F924F925F926F927F92E2
:103B10008F929F92AF92BF92CF92DF92EF92FF92DD
:103B20000F931F93CF93DF93CDB7DEB7AA970FB64E
:103B3000F894DEBF0FBECDBF5C010E8F1F8F28A390
:103B400039A34AA35BA36CA37DA31C8A1B8ADC0157
:103B500018968D919C9101979E8B8D8BE114F104A9
:103B6000D1F0CE0145969F938F9302979F938F93A9
:103B70008DE795E09F938F93FF92EF920F94865D70
:103B80000FB6F894DEBF0FBECDBF019721F48B892D
:103B90009C899E8B8D8B6B897C894AE050E089E300
:103BA00090E10F9485236FE573E189E390E10F9431
:103BB000E4236D897E894AE050E089E390E10F9427
:103BC000852369E573E189E390E10F94E423FE8D99
:103BD000FAA74AE050E06F2F89E390E10F949B220F
:103BE00089E390E10F94782219861A861B861C8639
:103BF0001D861E861F86188A8A85807F84608A8734
:103C0000D50118968D919C912D893E8928173907E9
:103C10001CF001979E8B8D8B8B899C8997FF02C02E
:103C20001C8A1B8A8B889C885401312C212C8D89FD
:103C30009E898A159B050CF46AC1BAA5B13091F131
:103C4000B23009F453C1EE24EA94FE2C0E8D1F8D80
:103C500028A139A14AA15BA16CA17DA1CE01099641
:103C60000E9415A529833A834B835C836D837E83F1
:103C70008F83988780919A0A90919B0AFC012281F8
:103C80003381A216B30608F088C06F852E8530E018
:103C900050E040E0542F432F322F2227462B6D85D2
:103CA000262B33C1E0909A0AF0909B0AF70182819B
:103CB0009381A816B90608F070C0968553850185D2
:103CC00012854084A92FB0E06484712C658570E072
:103CD0009401220D331D951372C0A901440F551F85
:103CE000240F351F200F311FA20FB31F9C91F3012A
:103CF000E20FF31F1081260F371FD9010C914420CA
:103D000009F452C0512C712C612C692F70E0762F70
:103D10006627072E000C880B990BA30192010F94C4
:103D2000ED57C901772766276EA37FA388A799A7B8
:103D3000612F70E0762F6627072E000C880B990BF9
:103D4000A30192010F94ED57542F432F322F2227B6
:103D50008EA19FA1A8A5B9A5822B932BA42BB52B2F
:103D60008EA39FA3A8A7B9A7602F70E0762F662720
:103D7000072E000C880B990BA30192010F94ED57AD
:103D80006EA17FA188A599A5262B372B482B592BEF
:103D9000232B242B252B09F4A0C0FFEFAF1ABF0A59
:103DA0002FEF221A320A43CF212F30E050E040E0BB
:103DB000542F432F322F2227492B202BE9CFC90123
:103DC000880F991F880F991F800F911FA80FB91F87
:103DD0003C91DC01A50FB11D0C91F301E80FF91F17
:103DE000D080860F971FDC011C91442009F463C02A
:103DF000512C712C612C632F70E0762F6627072ED3
:103E0000000C880B990BA30192010F94ED57922F90
:103E10008827772766276EA37FA388A799A7602F97
:103E200070E0762F6627072E000C880B990BA301F4
:103E300092010F94ED57A901332722278EA19FA14C
:103E4000A8A5B9A5822B932BA42BB52B8EA39FA33A
:103E5000A8A7B9A7612F70E0762F6627072E000C60
:103E6000880B990BA30192010F94ED576EA17FA1CE
:103E700088A599A5622B732B842B952B6EA37FA30A
:103E800088A799A76D2D70E0762F6627072E000C66
:103E9000880B990BA30192010F94ED57542F432FD8
:103EA000322F22278EA19FA1A8A5B9A5282B392B97
:103EB0004A2B5B2B6DCF802F90E0B0E0A0E0DC01BF
:103EC00099278827B32BAC01412B8A019D011D291D
:103ED000012B022B032B09F060CF2FEF3FEF4FEFA9
:103EE00050E0B501C7010F94D72857CF80919A0AA7
:103EF00090919B0ADC0112962D913C91A216B3067B
:103F000008F04BCF20E030E0A901B501ECCFCC2088
:103F100009F488C000919A0A10919B0AD801199659
:103F20008D919C91892B09F473C00E9478FFF80150
:103F3000C784D088E188F2886C157D058E059F05C1
:103F400020F46787708B818B928BF801C784D088AF
:103F5000E188F2886C197D098E099F096C327140E5
:103F60008105910510F3F894D80114968D919C91D8
:103F700015979A8B898B1996ED91FC917F01BFEF74
:103F8000EB1AFB0A80818D8FF80190810388F489F8
:103F9000E02DD80155968C91992309F45EC090814B
:103FA000982B9C8F9081809589238B8F8B8D888F08
:103FB00088E08F8B5C8D6B8D4D8D3F89288D898935
:103FC0009A89D701508347FD252F3A952083262FC4
:103FD00039F0441F00C000006083000000C0F2CF31
:103FE00038E04D9160830000019761F7D801549645
:103FF000FC93EE9353974D8F3F8B288F9A8B898B31
:1040000078940E9478FFF8016787708B818B928B80
:1040100064E573E189E390E10F94E42389E390E19F
:104020000F94782281E090E0AA960FB6F894DEBF54
:104030000FBECDBFDF91CF911F910F91FF90EF90F9
:10404000DF90CF90BF90AF909F908F907F906F90B8
:104050005F904F903F902F9008959081982B9C8F68
:104060009081809589238B8F8B8D8A8F88E0898FB3
:104070005C8D6B8D4D8D398D2A8D89899A89D701FB
:10408000508347FD252F00C000C0208300C000C022
:1040900000C000C000C060830000262F3A9541F0A8
:1040A000441F000000C000C000C000C000C0E8CF36
:1040B00038E04D9100C0608300C0019709F7D80136
:1040C0005496FC93EE9353974D8F398F2A8F96CF4A
:1040D000CF93DF93EC016FEE72E189E390E10F94EF
:1040E000E42363EE72E189E390E10F94E4236C81B1
:1040F0007D814AE050E089E390E10F9485236DEDE6
:1041000072E189E390E10F94E42389E390E10F9455
:10411000782260E08C810E9448FEE881F981048465
:10412000F585E02D60E0CE01199581E090E0DF910A
:10413000CF9108950F931F93CF93DF938C0163E882
:1041400075E089E390E10F947C22C0919A0AD091A6
:104150009B0A4C815D8170E060E089859A850F94AF
:10416000FE55209771F089859A850F94114F8E81A5
:104170009F8197FD03C060E00E9448FECE010F942E
:10418000114FD801ED91FC910484F585E02D60E09C
:10419000C801199581E090E0DF91CF911F910F91B7
:1041A0000895CF93DF93EC0163E975E089E390E133
:1041B0000F947C2240E050E0BA018A819B810E94EA
:1041C000C1AFE881F9810484F585E02D60E0CE017E
:1041D00019956D858C810E941AFE6D858D810E94D6
:1041E0001AFE81E090E0DF91CF910895CF92EF9297
:1041F000FF920F931F93CF93DF9300D000D01F92B5
:104200001F92CDB7DEB77C0109831A832B833C83D1
:104210004D835E836F83788767EC7BE089E390E171
:104220000F94E423CE0101960E94B5788981811113
:1042300029C00B81013071F128F010E00230E9F55E
:10424000CC20E9F060E0CE0101960E948074F70175
:1042500002811381892B69F0C8010E9402B0672B8B
:10426000682B692B61F480E00F94C542AB01BC015F
:1042700003C040E050E0BA01C8010E94C1AF81E034
:1042800090E02EC08031D0F58E30D8F58130C9F164
:104290008230D9F16AEB7BE089E390E10F94E4236B
:1042A0004AE050E0698189E390E10F949B2289E321
:1042B00090E10F94782201E010E06AEA7BE089E364
:1042C00090E10F94E4234AE050E0B80189E390E1E3
:1042D0000F94852389E390E10F94782290E080E0A9
:1042E00028960FB6F894DEBF0FBECDBFDF91CF91F9
:1042F0001F910F91FF90EF90CF90089583518330DD
:1043000048F6F70102811381A7CF40E050E0BA01DF
:10431000F70182819381B1CFFC01828193810E9458
:10432000E0B721E030E0823011F430E020E0C90154
:1043300008950F931F93CF93DF938C01D0E0C0E0DB
:1043400001151105B1F0BE016C5F734FC8010F94E8
:10435000AE50892B51F4FE01E85FF34F849190E059
:10436000DF91CF911F910F9108952596C233D1050A
:1043700039F781E090E0F4CFCF92DF92EF92FF9295
:104380000F931F93CF93DF93EC018C819D81892B39
:1043900009F49DC08A819B81892B09F498C07A0118
:1043A0006B01E881F9810284F385E02DCE01199536
:1043B0000397D9F4EC81FD8180A591A5A2A5B3A5B1
:1043C000892B8A2B8B2B89F00F947F02EC81FD8146
:1043D00000A511A522A533A5601B710B820B930BC1
:1043E000663971058105910528F38F81988521E053
:1043F000E21AF108DC01ED91FC910280F381E02DDD
:10440000A701B60119958F819885DC01ED91FC918A
:104410000190F081E02DD601129660E09D012C19EB
:104420003D092E153F0518F42D91620FF7CF199510
:104430000C811D8180E00F94C542F80160A771A72F
:1044400082A793A763E17AE089E390E10F94E423E4
:104450004AE050E06E8189E390E10F949B226FE087
:104460007AE089E390E10F94E4238601C8018C1976
:104470009D098E159F05B8F4D8016C9140E150E07C
:104480006A3050F462EA75E089E390E10F94CE233C
:1044900040E150E0F801608189E390E10F949B22B4
:1044A0000F5F1F4FE3CF89E390E10F947822E881FB
:1044B000F9810484F585E02D63E0CE01DF91CF9191
:1044C0001F910F91FF90EF90DF90CF901994DF91A3
:1044D000CF911F910F91FF90EF90DF90CF900895B3
:1044E0001F93CF93DF93EC01162F6E81112311F0F0
:1044F00081E068278C810E941AFE8F819885A985AA
:10450000BA85883E9340A105B10568F164E073E186
:1045100089E390E10F94E4236FEF72E189E390E186
:104520000F94E4236C817D814AE050E089E390E1BF
:104530000F9485236AEF72E189E390E10F94E423FD
:10454000612F70E04AE050E089E390E10F94852309
:1045500089E390E10F947822612FCE01DF91CF9112
:104560001F910C943AE6DF91CF911F910895AF927D
:10457000BF92CF92EF92FF920F931F93CF93DF934F
:1045800000D000D01F921F92CDB7DEB75C01098327
:104590001A832B833C834D835E836F83788769E422
:1045A00073E189E390E10F94E423CE0101960E9428
:1045B000B578E114F10439F062E473E1C7010F94B6
:1045C000AE50009759F1F5010281138101151105D3
:1045D00019F18981811162C08B81813009F466C033
:1045E00078F1823059F1082F10E06FE173E189E32F
:1045F00090E10F94E4236FE073E189E390E10F947D
:10460000E4234AE050E0B80189E390E10F94852368
:1046100089E390E10F94782290E080E028960FB62D
:10462000F894DEBF0FBECDBFDF91CF911F910F91E8
:10463000FF90EF90CF90BF90AF900895CC20C1F045
:1046400060E0CE0101960E948074892B09F44DC070
:10465000C8010E9402B0672B682B692BE1F480E04F
:104660000F94C542AB01BC01C8010E94C1AF13C089
:10467000C8010E94E0B78E3019F050F4813059F42F
:1046800060E0CE0101960E948074892B21F0E0CF7A
:1046900083518330A8F381E090E0C0CF803100F5F2
:1046A0008E30B0F68130A1F28230F9F067E373E129
:1046B00089E390E10F94E4236AE273E189E390E1F6
:1046C0000F94E4234AE050E0698189E390E10F947C
:1046D0009B2289E390E10F94782201E010E085CFDE
:1046E0008351833008F4B4CFE1CF40E050E0BA0109
:1046F000C8010E94C1AF60E0C5010E947022CBCF0B
:104700004F925F926F927F928F929F92AF92BF92E1
:10471000CF92DF92FF920F931F93CF93DF9300D03E
:1047200000D01F921F92CDB7DEB76130710509F43A
:104730007FC0FC01628173816115710509F478C045
:104740008C0119821A821B821C821D821E821F828A
:1047500018868A81807F8A8340E050E2CE010196EC
:104760000E94BD7360E0CE0101960E9480746C01CE
:10477000F801828193810E9402B02B013C01F80173
:104780002781308541855285D6010F9439582FEF06
:1047900030E040E050E00F94ED5749015A010F948A
:1047A0007F02FF24F39481149104A104B10461F009
:1047B0006419750986099709FF24F394681579052A
:1047C0008A059B0508F4F12C41145104610471041D
:1047D00079F1F80187809084A184B2840F947F02DC
:1047E000F80181149104A104B10451F06419750910
:1047F00086099709681579058A059B0508F446C05E
:10480000A280B38080E00F94C542AB01BC01C5011A
:104810000E94C1AFCD2861F0F80184810F94AE42AF
:10482000F8019681891304C061E0C8010E947022DA
:1048300090E080E028960FB6F894DEBF0FBECDBFA3
:10484000DF91CF911F910F91FF90DF90CF90BF909C
:10485000AF909F908F907F906F905F904F90089552
:10486000FF20D9F060E0C8010E947022F801828127
:1048700093810E94F2B9892BD9F640E050E0BA0149
:10488000F801828193810E94C1AFD2CF84810F94BD
:10489000AE42F80196818913E3CFCD2849F2F801A1
:1048A00084810F94AE42F80196818913C1CFF11033
:1048B000BFCFBACFAF92BF92CF92DF92EF92FF926B
:1048C0000F931F93CF93DF93CDB7DEB768970FB6E3
:1048D000F894DEBF0FBECDBFFC01098B1A8B2B8B6A
:1048E0003C8B4D8B5E8B6F8B788F82819381009791
:1048F00009F4A1C024813581232B09F49CC0CC206C
:1049000009F499C06F0170E060E00E948EB0192F29
:10491000D601ED91FC91008CF18DE02DC601199529
:104920005C018230910509F47AC0039709F445C00F
:1049300095E0F1E0AF16B10409F091E019861A860E
:104940001B861C861D861E861F86188A8A85807F88
:10495000892B8A87EE24EA94FE2C09891A892B89EF
:104960003C894D895E896F89788DCE0109960E94B8
:1049700015A5F1E0AF16B10409F453C082E0A81602
:10498000B10409F049C06F8570E0D60114968C918E
:104990000E9484FE61E070E0C6010E9425E66E85FB
:1049A00070E00E9484FE62E070E0C6010E9425E68D
:1049B0006D8570E00E9484FE2FC0612F661F662700
:1049C000661FCE0141960E9480745C01BC01D60135
:1049D00014968C910E9484FE62EC72E189E390E16E
:1049E0000F94E423F601648175814AE050E089E385
:1049F00090E10F94852360EC72E189E390E10F94DC
:104A0000E4234AE050E0B50189E390E10F94852367
:104A100089E390E10F94782281E090E00EC094E069
:104A20008DCF63E070E0C6010E9425E6688970E0E2
:104A30000E9484FEA8CF90E080E068960FB6F894BC
:104A4000DEBF0FBECDBFDF91CF911F910F91FF90C1
:104A5000EF90DF90CF90BF90AF900895CF93DF930A
:104A6000EC0166EB72E189E390E10F94E4236C8141
:104A70007D814AE050E089E390E10F94852364EB67
:104A800072E189E390E10F94E423EA81FB810280E3
:104A9000F381E02D6081718189E390E10F94CE2351
:104AA0006EEA72E189E390E10F94E42389E390E1F7
:104AB0000F947822E881F981008CF18DE02DCE01F0
:104AC00019958130910529F0029759F060E08C81A9
:104AD0001AC063E070E0CE010E9425E660E00E940B
:104AE00048FE60E08C810E9448FE61E070E0CE01EB
:104AF0000E9425E660E00E9448FE62E070E0CE0180
:104B00000E9425E660E00E9448FEE881F981048465
:104B1000F585E02D60E0CE01199581E090E0DF9110
:104B2000CF910895CF92DF92FF920F931F93CF936F
:104B3000DF9300D000D01F921F92CDB7DEB76C017B
:104B4000F02E1A83022F10E0FF2029F00115110525
:104B500011F401E010E040E050E061E070E0F601A7
:104B6000828193810E9496B10130110591F102304A
:104B7000110541F0012B99F56EE470E189E390E1B4
:104B80000F94E4238A818F70A1F1F60102811381D1
:104B9000C8010E9402B0672B682B692B89F401E0E1
:104BA00010E0C80128960FB6F894DEBF0FBECDBF47
:104BB000DF91CF911F910F91FF90DF90CF900895DB
:104BC00080E00F94C542AB01BC01C8010E94C1AF97
:104BD000E6CFF1E0FF1681F082E0F81669F062E4BA
:104BE00070E189E390E10F94E42389E390E10F946D
:104BF000782210E000E0D5CFF601C280D380C60154
:104C00000E9402B0672B682B692B49F280E00F9459
:104C1000C542AB01BC01C6010E94C1AFC2CFCF9259
:104C2000DF92EF92FF920F931F93CF93DC011296C6
:104C3000ED91FC9160E0848195810E94ECED8C0106
:104C4000009729F0FC0180858F708530D1F06AE0F3
:104C500072E182E99FE00F94E42382E99FE00F94E0
:104C60007822C12CD12C90E8E92E9FEBF92EC701B8
:104C7000B601CF911F910F91FF90EF90DF90CF90F1
:104C80000895C8010E947DEE813040F18630A8F180
:104C9000893020F565E0C8010E94ECEDFC019085AB
:104CA0009F709330F9F4C184D284E384F484C1E02A
:104CB00060E0C8010E94ECEDFC0190859F7093308C
:104CC00009F5618572858385948520E030E0A9012E
:104CD0000F94A35687FF1FC0C111C9CFC12CD12C7F
:104CE0007601C5CF923049F46185728583859485BC
:104CF0000F94AA566B017C01DACFC0E0C12CD12CF5
:104D00007601D6CF923039F461857285838594859A
:104D10000F94AA56DACFC111AACFC12CD12C8FE79C
:104D2000E82E83E4F82EA3CFCF93DF93EC0168ED58
:104D300071E189E390E10F94E423EA81FB81028031
:104D4000F381E02D6081718189E390E10F947C22F1
:104D5000EC81FD81309721F0808191810F94114F7A
:104D60008C819D810F94114F70E060E08A819B815E
:104D70000E947EAF1D821C8281E090E0DF91CF9186
:104D80000895CF93DF93EC0164EA75E089E390E145
:104D90000F94CE23EA81FB810280F381E02D6081B4
:104DA000718189E390E10F947C228C819D81009731
:104DB00011F00F94114F70E060E08A819B810E9496
:104DC0007EAF1D821C8281E090E0DF91CF9108953B
:104DD000CF93DF93FC0122813381232B59F1EC0126
:104DE0006EE67AE089E390E10F94E4234AE050E034
:104DF0006E8189E390E10F949B2289E390E10F9407
:104E000078228C819D810F94114F70E060E08A813F
:104E10009B810E947EAF1D821C82E881F9810484FF
:104E2000F585E02D60E0CE01199581E090E0DF91FD
:104E3000CF91089590E080E0FACFCF92DF92EF9289
:104E4000FF920F931F93CF93DF93009761F4D0E00D
:104E5000C0E0CE01DF91CF911F910F91FF90EF90B5
:104E6000DF90CF900895DC011896EC91EF70E6305A
:104E700071F769017A018B01EC010E943AED892BEF
:104E800031F70E944DF3AC01B801CE010E94DCFA6B
:104E9000B801CE010E943AEDEC01892BC1F2888560
:104EA000982F9F70923039F0933071F09111D1CFDB
:104EB000807F82608887C701B6010F947559698722
:104EC0007A878B879C87C5CFC986DA86EB86FC8676
:104ED000C0CFCF92DF92EF92FF920F931F93CF93A9
:104EE000DF93009701F1DC011896EC91EF70E6304A
:104EF000D1F469017A018B01EC010E943AED892B12
:104F000091F4A7019601B801CE010E9404FBB801FB
:104F1000CE01DF91CF911F910F91FF90EF90DF9025
:104F2000CF900C943AED90E080E0DF91CF911F910B
:104F30000F91FF90EF90DF90CF9008954F925F9286
:104F40006F927F928F929F92AF92CF92DF92EF9269
:104F5000FF920F931F93CF93DF93CDB7DEB7A09748
:104F60000FB6F894DEBF0FBECDBF4C0161307105A6
:104F7000C9F5DC0112968D919C910E9402B0672BBD
:104F8000682B692B79F180E00F94C5426B017C019D
:104F9000F40102811381C8010E9402B0C61AD70A27
:104FA000E80AF90AF0E6CF16FAEEDF06E104F104AA
:104FB000C8F040E050E0BA01C8010E94C1AFD4017E
:104FC00012960D911C911397ED91FC910288F38933
:104FD000E02DC401199562E0892B09F061E0C80158
:104FE0000E94C1B7D4011496ED91FC91309709F459
:104FF000CAC1668077806114710409F4C4C1D30109
:10500000ED91FC91309709F4E0C08081882309F488
:10501000DCC065E775E0C3010E943AED2C01009702
:1050200009F4D3C0FC0181859285A385B4850097DE
:10503000A105B10509F4C9C08C01FC0122AD2223F0
:1050400009F4C3C00F949325882309F4BEC065EC0E
:1050500075E0C3010E943AED6C01009709F4B5C0F8
:10506000DC0118968C918F70833009F0AEC06CEE25
:1050700070E189E390E10F94E423D4011296ED915D
:10508000FC910280F381E02D6081718189E390E1E0
:105090000F94CE2362E179E089E390E10F94CE236F
:1050A000F3016081718189E390E10F94CE2367EE73
:1050B00070E189E390E10F94E423D8015C96ED91CF
:1050C000FC91408151816281738189E390E10E946A
:1050D00080F261EE70E189E390E10F94E423D8015E
:1050E0009096ED91FC91408151816281738189E3B9
:1050F00090E10E9480F26BED70E189E390E10F9402
:10510000E423D8015E96ED91FC914081518162814A
:10511000738189E390E10E9480F268EC75E089E395
:1051200090E10F94CE23F801408151816281738117
:1051300089E390E10E9480F26CEC75E089E390E1F4
:105140000F94CE23D80114964D915D916D917C9171
:10515000179789E390E10E9480F260ED75E089E3A2
:1051600090E10F94CE23F8014085518562857385C7
:1051700089E390E10E9480F2D80158968D919C912C
:1051800069EB75E0892B11F063EB75E089E390E141
:105190000F94CE23F80182AD6FEB75E0811102C050
:1051A00062EC75E089E390E10F94CE2389E390E10E
:1051B0000F947822D40112968D919C910E94E0B7B1
:1051C000833141F0843109F476C0D30112966D9099
:1051D0007C9011CF70E060E0F201818592850F94A0
:1051E000F5266FEC70E189E390E10F94E423D4019C
:1051F0001296ED91FC910280F381E02D6081718126
:1052000089E390E10F94CE2362E179E089E390E1B4
:105210000F94CE23F3016081718189E390E10F94B3
:10522000CE236EEB70E189E390E10F94E42389E3F0
:1052300090E10F947822D401ED91FC91408851883F
:10524000F301E080F18019861A861B861C861D8674
:105250001E861F86188A8A85807F8A87D6011996BE
:105260006D917D918D919C911C970F947559CE01F4
:1052700009960E944C74298B3A8B4B8B5C8B6D8BFF
:105280007E8B8F8B988F67E0CE0141960E94507382
:10529000298F3A8F4B8F5C8F6D8F7E8F8F8F98A366
:1052A000A12CCC24C39489019A01AB01BC01C40197
:1052B000F20119958ACF61E070E0D20119968D91C3
:1052C0009C910F94F52662EB70E189E390E10F94D5
:1052D000E423D4011296ED91FC910280F381E02D3C
:1052E0006081718189E390E10F94CE2362E179E0DE
:1052F00089E390E10F94CE23F3016081718189E30A
:1053000090E10F94CE2360EA70E189E390E10F947D
:10531000E42389E390E10F947822D401ED91FC918C
:1053200040885188F301E080F18019861A861B8637
:105330001C861D861E861F86188A8A85807F8A871E
:10534000D60119966D917D918D919C911C970F942A
:105350007559CE0109960E944C74298B3A8B4B8B60
:105360005C8B6D8B7E8B8F8B988F67E0CE01419627
:105370000E94507329833A834B835C836D837E83C1
:105380008F8398878DCF81E090E0A0960FB6F89438
:10539000DEBF0FBECDBFDF91CF911F910F91FF9068
:1053A000EF90DF90CF90AF909F908F907F906F9015
:1053B0005F904F9008952F923F924F925F926F921D
:1053C0007F928F929F92AF92BF92EF92FF920F9334
:1053D0001F93CF93DF93CDB7DEB72C970FB6F8941A
:1053E000DEBF0FBECDBF6130710509F460C18C0115
:1053F000FC01E280F38040E050E061E070E0C70132
:105400000E94BFB1672B682B692B09F450C140E0A3
:1054100050E062E070E0C7010E94BFB1672B682BCB
:10542000692B89F480912702882309F440C140E068
:1054300050E062E070E0C7010E9496B180912702BF
:10544000815080932702F801E280F380C7010E9417
:1054500002B04B015C0119821A821B821C821D82E0
:105460001E821F8218868A81807F8A8340E050E2F4
:10547000B701CE0101960E94BD7360E0CE01019696
:105480000E9480747C01F801828193810E94E0B7C0
:10549000823011F0853011F4F12CE12CF801868175
:1054A0009AEC980F903108F0B1C121853285A9019D
:1054B00070E060E049875A876B877C874384548417
:1054C000712C612C0E945BFF9C01990F440B550BC2
:1054D0002419350946095709AFEFB0E00F942E584B
:1054E00029853A854B855C85241935094609570974
:1054F0000F940F58390137FDB3C15FEF6516710482
:1055000011F00CF0B0C181149104A104B10409F0B0
:1055100085C1E618F70856EFE5165FEFF5060CF0C3
:10552000F3C0F801658585810E941AFEF801A2800A
:10553000B380C5010E9402B0672B682B692B41F430
:1055400080E00F94C542AB01BC01C5010E94C1AF10
:10555000F801B48065858EEF8B0D8C3028F084EDDA
:105560008B0D833008F070C0AA27BB27AE19BF0986
:10557000662309F45CC09D01A1E0BFEF0F9473584E
:1055800029E130E040E050E00F940F58BA01A90142
:1055900041505F4F6F4F7F4F942F852F692F782F8A
:1055A0006F3F710519F014F06FEF70E0663471050C
:1055B00014F466E470E08B2D78C063E370E189E356
:1055C00090E10F94E42389E390E10F94782264ED55
:1055D00075E089E390E10F947C22F8016585848170
:1055E0000E941AFEF801658585810E941AFE40E03E
:1055F00050E0BA01F801828193810E94C1AF40E07E
:1056000050E061E070E0F801828193810E946DB109
:1056100040E050E062E070E0F801828193810E94F6
:105620006DB1809127028F5F8093270240C02FEFDA
:1056300030E00F947B5829E130E040E050E00F94D7
:105640000F58922F832FAACF858191E069279EEF73
:10565000980F9C3020F08C52833008F0D3C08B2DF3
:105660000E941AFEAA27BB27AE19BF09F80185853B
:105670008823B1F12FEF30E00F947B5829E130E01F
:1056800040E050E00F940F58922F832F692F782F0E
:105690006F3F710519F014F06FEF70E0663471051B
:1056A00014F466E470E0F80185810E9484FE90E0C5
:1056B00080E02C960FB6F894DEBF0FBECDBFDF9111
:1056C000CF911F910F91FF90EF90BF90AF909F905F
:1056D0008F907F906F905F904F903F902F900895A4
:1056E0009D01A1E0BFEF0F94735829E130E040E045
:1056F00050E00F940F58BA01A90141505F4F6F4F0E
:105700007F4F942F852FC2CFFBE0EF16F1040CF4EE
:105710005ECFF801658584810E941AFEF801A2809F
:10572000B380C5010E9402B0672B682B692B41F43E
:1057300080E00F94C542AB01BC01C5010E94C1AF1E
:10574000F801B58065858EEF8B0D8C3020F084EDEF
:105750008B0D8330B0F4662351F09701A1E0BFEFC9
:105760000F94735823E330E040E050E00DCF2FEF6B
:1057700030E0D7010F947B5823E330E040E050E065
:105780005ECF848191E069279EEF980F9C3018F0DE
:105790008C528330B8F58B2D0E941AFEF801858556
:1057A0008823E1F02FEF30E0D7010F947B5829E1F7
:1057B00030E040E050E00F940F58922F832F692F74
:1057C000782F77FF02C070E060E06F3F710519F03D
:1057D00014F06FEF70E0F801848167CF9701A1E0CA
:1057E000BFEF0F94735829E130E040E050E00F9490
:1057F0000F58BA01A90141505F4F6F4F7F4F942F4F
:10580000852FDDCF8B2D0E941AFE51CF66246A941E
:10581000762C81149104A104B104F1F0F8012780E1
:105820003084032C000C440855080F947F02211487
:1058300031044104510409F4C0CE681979098A0978
:105840009B09621573058405950508F0B6CEFFEF38
:105850006F167F0609F05DCE4FE7E41AF1085BCEC4
:10586000712C612C50CE66246A94712C4CCE8F9290
:105870009F92AF92BF92CF92DF92EF92FF920F93DF
:105880001F93CF93DF93CDB7DEB760970FB6F89431
:10589000DEBF0FBECDBFE986FA860B871C872D873A
:1058A0003E874F87588B6115710511F0011103C0B8
:1058B00090E080E0CCC07B015C01DB018D909C908E
:1058C00019821A821B821C821D821E821F821886E8
:1058D0008A81807F8A8362EE75E0C7010E943AED7B
:1058E0006C0167EE75E0C7010E943AED7C01C114BE
:1058F000D10451F1F60180858F70843029F58185BE
:1059000092850E949921182F8930B1F134F48130A9
:10591000E4F4C12CD12C760168C08A30D1F7B701EC
:10592000CE0109960E94417C29833A834B835C8394
:105930006D837E838F8398873F7009F4B9CFCE0142
:1059400001960E94297615C011E0B701CE01099693
:105950000E94417C29833A834B835C836D837E83E1
:105960008F8398873F7009F4A3CFCE0101960E94E0
:10597000E5756B017C0139C0B701CE0109960E9423
:10598000417C29833A834B835C836D837E838F8341
:1059900098873F7009F48CCF31503B3008F0B9CF75
:1059A000E32FF0E08827E852F34D8F4F0D946458B1
:1059B000EC2CEC2C892CE32CE32C472D3A2D3A2DA2
:1059C0003A2DE32CE32C2D813E814F815885AAE0AE
:1059D000B0E00F942E58CDCFCD80FAE0CF9E60017D
:1059E00011240D2C000CEE08FF088091450289302F
:1059F00020F4809144028930E8F061E070E189E3AD
:105A000090E10F94E423B40189E390E10F94CE2355
:105A10006AEF7FE089E390E10F94E4232AE030E02D
:105A2000B701A60189E390E10F943D2389E390E15A
:105A30000F947822D5011296ED91FC9162E0848159
:105A400095810E94ECED009779F581E090E06096F9
:105A50000FB6F894DEBF0FBECDBFDF91CF911F917F
:105A60000F91FF90EF90DF90CF90BF90AF909F90FD
:105A70008F90089520E030E040E251E46D817E8116
:105A80008F8198850F9409570F94755972CF6D8146
:105A90007E818F8198852AE030E040E050E00F94CD
:105AA0000F5869017A01A1CFFC0120852F702630A3
:105AB00061F6B4010E943AED5C01009731F2DC011D
:105AC00018968C9118978F709BEF980F923008F072
:105AD000BCCF4501853029F416968C901697179601
:105AE0009C90F5018085806880876BEE75E0C4012D
:105AF0000E943AEDFC01892B61F0C186D286E386D3
:105B0000F486812F8295807F10851F70182B108757
:105B10009CCF61EF7FE089E390E10F94E423D5010E
:105B20006D917C9189E390E10F94CE2389E390E11C
:105B30000F947822A70196016BEE75E0C4010E94D4
:105B400004FB6BEE75E0C4010E943AEDFC01892B69
:105B500009F47BCF1295107F90859F70192BD7CFBA
:105B60002F923F924F925F927F928F929F92AF922D
:105B7000BF92CF92DF92EF92FF920F931F93CF933A
:105B8000DF9300D000D01F921F92CDB7DEB70983FC
:105B90001A832B833C834D835E836F837887DC017C
:105BA0001496ED91FC910FEF1FEF3097F9F057012C
:105BB0004C01C288D388E114F10489F1F701808196
:105BC000882369F1C114D10489F1B701C6010E948B
:105BD0003AEDE980FA800B811C812D813E814F8155
:105BE0005885BC01C4010E94372C8C01C80128963D
:105BF0000FB6F894DEBF0FBECDBFDF91CF911F91DE
:105C00000F91FF90EF90DF90CF90BF90AF909F905B
:105C10008F907F905F904F903F902F900895C11488
:105C2000D10421F0D6011696CD90DC907B80F12C2A
:105C30000FEF1FEF272C312C512C412CC114D10414
:105C400049F166E775E0C6010E943AED0097E9F078
:105C5000FC0120852F702230C1F481859285A385B7
:105C6000B48582159305A405B50579F4E980FA8019
:105C70000B811C812D813E814F815885B601C40165
:105C80000E94372C8C01FF24F394D6011296CD90FC
:105C9000DC90D4CFF110AACF6CE170E182E99FE0F3
:105CA0000F94E423B50182E99FE00F94CE2360E1D5
:105CB00070E182E99FE00F94E423672D70E04AE0F1
:105CC00050E082E99FE00F94852382E99FE00F94E2
:105CD00078228CCF1F93CF93DF9300D000D0CDB725
:105CE000DEB76130710509F468C05CF4672B09F414
:105CF0005AC06FE97DE089E390E10F94E42380E0EE
:105D000048C06230710571F06330710591F790936E
:105D1000DD0D8093DC0D55275093DF0D4093DE0D94
:105D200084E009C09093DD0D8093DC0D5093DF0D6E
:105D30004093DE0D83E00F940A04182F80E00F9447
:105D4000C5426093960A7093970A8093980A90933D
:105D5000990A1123D9F06AE87DE082E99FE00F9467
:105D6000E423812F90E0B0E0A0E089839A83AB83A5
:105D7000BC8380E190E09E838D83BE016F5F7F4F87
:105D800082E99FE00E94B9D20F94782281E011113C
:105D9000B6CF26960FB6F894DEBF0FBECDBFDF910B
:105DA000CF911F9108959093DD0D8093DC0D50935A
:105DB000DF0D4093DE0D81E0BECF9093DD0D80932B
:105DC000DC0D5093DF0D4093DE0D82E0B4CFCF9316
:105DD000DF93EC01EC81FD8140815181052E000CA7
:105DE000660B770B22818AED9CE00F94312570E0E1
:105DF00060E08A819B810E948EB0E8EDFDE08283A5
:105E00008AED9CE0918380831092E80E1092EA0E56
:105E10001092E90EDF91CF910895CF93DF93611532
:105E2000710589F0EB01DC011296ED91FC9162E0C5
:105E3000848195810E94ECEDBE010E943AEDDF91D4
:105E4000CF910C9448FD90E080E0DF91CF910895D0
:105E50004F925F926F927F928F929F92AF92BF927A
:105E6000CF92DF92EF92FF920F931F93CF93DF9326
:105E7000CDB7DEB768970FB6F894DEBF0FBECDBFC3
:105E8000098B1A8B2B8B3C8B4D8B5E8B6F8B788F9A
:105E9000DC0112962D913C911397232B09F4DEC05F
:105EA000CC2009F4DBC06C01ED91FC91008CF18DEC
:105EB000E02D19955C0169EF7BE089E390E10F9497
:105EC000E423CE0141960E94B578A114B10471F487
:105ED00060E0CE0141960E948074682FF6018481B3
:105EE00095810F94E43C81E090E0BAC0CE014196E8
:105EF0000E9474764C0194E0F2E0AF16B10459F0C0
:105F000081E1A816B10409F445C091E0A1E0AA1608
:105F1000B10409F495E019861A861B861C861D8635
:105F20001E861F86188A8A85807F892B8A87EE24A1
:105F3000EA94FE2C09891A892B893C894D895E894E
:105F40006F89788DCE0109960E9415A56FEE7BE0D2
:105F500089E390E10F94E423CE0109960E94B5787D
:105F6000B2E0AB16B10489F0E1E1AE16B104B1F0D4
:105F7000AA94AB2809F0B7CF188963E070E0C60196
:105F80000E9425E6612F0F94E43C6F85F601848121
:105F9000958151C0888D8170888FBCCF0FE710E04C
:105FA0008FEF88169806A9F0092C000CAA08BB08E8
:105FB000A50194012959310941095109AFEFB0E018
:105FC0000F942E582BE531E040E050E00F940F582D
:105FD000890163E070E0C6010E9425E65C01288922
:105FE00030E0D8010F947B58412C512C32014A9457
:105FF000A30192010F940F58622FC5010F94E43C46
:1060000064E070E0C6010E9425E65C01AFEFB0E0FD
:10601000A01BB10B288930E00F947B58A30192019B
:106020000F940F58622FC5010F94E43C6F85D60181
:1060300014968D919C910F94E43C1E8561E070E074
:10604000C6010E9425E6612F0F94E43C1D8562E0A5
:1060500070E0C6010E9425E6612F43CF90E080E00A
:1060600068960FB6F894DEBF0FBECDBFDF91CF911B
:106070001F910F91FF90EF90DF90CF90BF90AF9066
:106080009F908F907F906F905F904F9008958F9228
:106090009F92AF92BF92CF92DF92EF92FF920F93B7
:1060A0001F93CF93DF9300D000D01F921F92CDB7E4
:1060B000DEB76D7F6130710509F4BAC0FC01E28082
:1060C000F380E114F10409F4B3C08C01C7010E940C
:1060D00002B04B015C0161E070E0C7010E9448B072
:1060E00081149104A104B10409F4A2C020E030E0BD
:1060F0004AE754E40F9409570F947C596B017C01D3
:10610000C114D104E104F10409F492C00F947F0298
:10611000681979098A099B096C157D058E059F050B
:1061200008F486C0F801A280B38070E060E0C50189
:106130000E9448B020E030E048EC52E40F94095748
:106140000F947C596B017C0180E00F94C542AB0138
:10615000BC01C5010E94C1AF19821A821B821C8238
:106160001D821E821F8218868A81807F8A83F801A1
:106170006281738140E050E3CE0101960E94BD73BD
:10618000CE0101960E9429764B015C016EEE75E00E
:1061900089E390E10F94CE232AE030E0B501A40119
:1061A00089E390E10F9493226DEF75E089E390E12C
:1061B0000F94CE232AE030E0B701A60189E390E1F5
:1061C0000F94932289E390E10F947822C80CD91C94
:1061D000EA1CFB1C8A81807F86608A83CD82DE82F6
:1061E000EF82F886F8016281738140E050E2CE01CF
:1061F00001960E94AA7261E076E089E390E10F9433
:10620000CE232AE030E0B701A60189E390E10F94A4
:10621000932289E390E10F94782230E020E040E07F
:1062200050E260E070E0F801828193810E9429B51C
:1062300090E080E028960FB6F894DEBF0FBECDBF89
:10624000DF91CF911F910F91FF90EF90DF90CF9052
:10625000BF90AF909F908F900895CF92DF92EF9272
:10626000FF920F931F93CF93DF93CDB7DEB7629763
:106270000FB6F894DEBF0FBECDBF6C010B871C8735
:106280002D873E874F87588B698B7A8B65EA7BE039
:10629000C7010F94AE50EEE0F0E0892BF1F06FE90A
:1062A0007BE0C7010F94AE50E0E1F0E0892BA9F04C
:1062B00069E97BE0C7010F94AE50EFE0F0E0892B75
:1062C00061F01D8565E97BE0C7010F94AE50E12FB9
:1062D000F0E0892B11F4EDE0F0E09B85992341F08B
:1062E000309731F4EF2809F45CC08FEF9FEFC6C000
:1062F000E131F10508F037C08827EE57FE4C8F4F8B
:106300000D9464587531D1319331B331B331B33118
:10631000B3317F323333B331B331B331B331B3310E
:106320003D3376334B33CE010B960E94E57520EF5B
:10633000260F2931D0F6D6011496ED91FC911597D0
:1063400023A39B01AC013327442755271296ED91D7
:10635000FC910280F381E02D6081718106E116E0FD
:10636000C6010E94ECE6D6011496ED91FC911597BA
:10637000118A1496ED91FC91159781E0818714960E
:10638000ED91FC9115978DE482871496ED91FC9127
:1063900015978FE5838714966D917C9145E250E0C7
:1063A00048C0F6010481158180E00F94C542D801F0
:1063B00098966D937D938D939C939B97D601ED91C9
:1063C000FC910484F585E02D64E0C6011995EB8508
:1063D000E150E53140F6F0E0D60114962D913C9164
:1063E00015978827E950FE4C8F4F0D9464580C3256
:1063F0001D32B331B3311D320C32B331B331B3314D
:10640000B331B331B331B3314D326532B331B3311E
:10641000B33161325D326332F90185A1858F149603
:10642000ED91FC91858D8160858F4DE050E06AE1B2
:1064300072E0C6010E94BC211FC0F90185A1858FB1
:106440001496ED91FC91858D8E7F858F4DE050E007
:106450006DE072E0C6010E94BC21D6011296ED915A
:10646000FC910280F381E02D4BE156E06CEF76E089
:10647000808191810F94370381E090E062960FB69E
:10648000F894DEBF0FBECDBFDF91CF911F910F916A
:10649000FF90EF90DF90CF900895F901178AD60111
:1064A0001496ED91FC91159785A1858F1496ED9129
:1064B000FC91858D8160858F56CF81E0F901878BB6
:1064C000EECF82E0FBCF84E0F9CF83E0F901878B48
:1064D0001496ED91FC91159785A1858F1496ED91F9
:1064E000FC911597858D8160858F1496ED91FC91B7
:1064F000818D833009F037CF82E0818F34CF1982CC
:10650000F601048115819031C1F190F4923009F4C3
:1065100040C09E30B9F0CE010B960E94E575611522
:1065200071058105910509F055C0F80117A240C019
:10653000913141F1923179F782E0F801818F66E57E
:106540007BE006C083E0D80159968C9362E37BE040
:10655000CE0101960F94B750D6011296ED91FC91A1
:106560000280F381E02D40E256E0BE016F5F7F4F75
:10657000808191810F943703F6CEF801118E64E487
:106580007BE0E6CF81E0D80159968C936DE47BE007
:10659000DFCFD80197961C920481158180E00F947B
:1065A000C542D80198966D937D938D939C939B974C
:1065B000D6011496ED91FC91159785A1858F1496BF
:1065C000ED91FC91858D8E7F858F4DE050E06DE0E3
:1065D00072E02FCFD80197961C9261507109810902
:1065E0009109660F771F881F991F2EEF30E040E05A
:1065F00050E00F940F58DA01C9010196A11DB11D99
:10660000813071F0A8F2823029F1833009F0A4CFF3
:10661000D6011496ED91FC91118E64E47BE008C0E4
:10662000D6011496ED91FC9182E0818F66E57BE0C6
:10663000CE0101960F94B750D6011496ED91FC91BE
:10664000159785A1858F1496ED91FC91858D8160BC
:10665000858F82CFD6011496ED91FC9181E0818FD8
:106660006DE47BE0E5CFCE010B960E94E575D60187
:106670001496ED91FC91678B76CED6011496ED9130
:10668000FC91913029F0923009F06DCE148E6BCED2
:1066900080E5848F68CEF60104811581913049F040
:1066A0009230B1F0CE010B960E94E575F801638F30
:1066B0005ACE83E0D8015B968C930280F381E02D63
:1066C0000280F381E02D45E256E06BEE76E050CF9C
:1066D000F801138ED6011296ED91FC910280F381A0
:1066E000E02D45E256E06CEF76E042CFD6011496FD
:1066F000ED91FC91913031F0923009F034CE858DDE
:10670000877FD9CE858D8860D6CE8F929F92AF92AB
:10671000BF92CF92DF92EF92FF920F931F93CF938E
:10672000DF937C014A015901C091900AD091910AEE
:10673000062F660F110B209709F45CC088858F70B7
:10674000863009F055C06CE276E0CE010E943AED49
:106750006C0182E08816910449F061E376E0E3E0A1
:106760008E16910429F0D0E0C0E006C065E376E023
:10677000CE010E943AEDEC01C114D104D9F1F60129
:1067800080858F708430B1F561857285A801C7015D
:106790000F94FF5CA80162E179E0C7010F94E15C0E
:1067A000209779F188858F70843059F569857A85CD
:1067B000A801C7010F94E15CA80162E179E0C7017B
:1067C0000F94E15CA114B10429F0A801B501C7013F
:1067D0000F94E15CC701DF91CF911F910F91FF9062
:1067E000EF90DF90CF90BF90AF909F908F900895E3
:1067F000D0E0C0E0A8016DEC73E1C7010F94E55053
:10680000C9CFF2E08F16910481F083E088169104DD
:1068100029F060918E0A70918F0ACACFA80167ECA7
:1068200073E1C7010F94C750C7CFA80164EC73E1AF
:10683000F8CFAF92BF92CF92DF92EF92FF921F9369
:10684000CF93DF9300D000D0CDB7DEB76C017C01D1
:1068500010E08AE0A82EB12C133061F1F70182819B
:1068600090E0B0E0A0E089839A83AB83BC83BE82D2
:10687000AD82BE016F5F7F4F88E89FE00E94B9D272
:1068800062EC73E10F94E4231F5FFFEFEF1AFF0A3E
:10689000143011F726960FB6F894DEBF0FBECDBFA9
:1068A000DF91CF911F91FF90EF90DF90CF90BF903D
:1068B000AF900895F601858190E0B0E0A0E0898373
:1068C0009A83AB83BC83BE82AD82BE016F5F7F4F74
:1068D00088E89FE00E94B9D260EC73E1D3CFFC015D
:1068E000DC018D918111FDCF30E020E050E040E0EF
:1068F0008AE09191992301F1443051055CF59E3273
:1069000071F42F3F310509F02CF5DB01A40FB51F01
:1069100012962C934F5F5F4F30E020E0EACF829FCA
:10692000D001839FB00D1124292F990F330B2053D1
:1069300031092A0F3B1FDDCF2F3F310509F054F4F9
:10694000443051053CF4640F751FFB01228381E044
:1069500090E0089590E080E00895CF92DF92EF926A
:10696000FF920F931F93CF93DF93EC016A017B019A
:10697000CB01BA010F9475598B011F936F9386E376
:1069800098E09F938F93DF93CF930F94565D0F9072
:106990000F900F900F900F900F9020E030E0A90122
:1069A000C701B6010F94AB59181624F0F7FAF0940A
:1069B000F7F8F09409900020E9F721978EE2888398
:1069C000B80117FF03C0719561957109072E000C7E
:1069D000880B990B0F94AA569B01AC01C701B60115
:1069E0000F94965820E030E040E251E40F940957AC
:1069F0000F947559605D69831A82DF91CF911F9161
:106A00000F91FF90EF90DF90CF900895CF93DF9399
:106A10001F921F92CDB7DEB78091B3129091B4123E
:106A2000009711F48FEB92E1BE016F5F7F4F681BFF
:106A3000790B072E000C880B990B0F900F90DF91AC
:106A4000CF9108954F925F926F927F929F92AF92F3
:106A5000BF92CF92DF92EF92FF920F931F93CF934B
:106A6000DF93CDB7DEB768970FB6F894DEBF0FBEE1
:106A7000CDBFFC01198A1A8A1B8A1C8A1D8A1E8AAC
:106A80001F8A188E8A89807F8A8BA081B181109796
:106A900009F47AC08C91882309F476C000811181B1
:106AA000D8019C91992309F443C09D3209F4DAC0BE
:106AB00090539A3028F00F5F1F4F11830083EECF61
:106AC000C801912CDC016D01C81AD90A2D91022E42
:106AD000000C330B205331092A303105A0F37F011C
:106AE0006EE270E0C8010F94C65CFC01009709F4E7
:106AF00048C0DC015D01AE1ABF0A11968C91119756
:106B0000082E000C990BC09711960A9798F3818173
:106B1000282F082E000C330B205331092A30310561
:106B200018F480330CF057C020E030E0A90108C011
:106B3000912CD12CC12CD3CF29E030E040E050E0A3
:106B4000AAE0B0E00F942E582B013C012281822F45
:106B5000022E000C990BC0978A30910570F42033F7
:106B60000CF441C02A330CF042C0092E000CAA0BD1
:106B7000BB0B480E591E6A1E7B1EA114B10409F0FE
:106B800088C0CD2809F073C088E0FE017196DE014F
:106B9000199601900D928A95E1F729853A854B85E2
:106BA0005C856D857E858F85988968960FB6F8948B
:106BB000DEBF0FBECDBFDF91CF911F910F91FF9030
:106BC000EF90DF90CF90BF90AF909F907F906F90AD
:106BD0005F904F9008958A330CF0AECF032E000CD7
:106BE000440B550BADCF80E090E0DC01C2CF89E0D3
:106BF00090E0A0E0B0E0BDCFB8E0CB16D1040CF03F
:106C00004DC0C8010F9460509B01AC01A4E6B0E0F8
:106C10000F942E58992041F07094609450944094B1
:106C2000411C511C611C711C2A89207F26602A8B03
:106C3000460E571E681E791E4D8A5E8A6F8A788EB0
:106C40006CE270E0F701808191810F94C65C00973F
:106C500021F4D7011D921C9297CF0196F7019183E1
:106C6000808392CFC8010196992493942BCFC801B9
:106C70000F946050AB01BC01CE0141960E94947309
:106C800029833A834B835C836D837E838F839887CC
:106C9000D7CFF3E0AF16B1040CF4AECFC8010F9418
:106CA0003E502A89207F27602A8B6D8B7E8B8F8BAD
:106CB000988FC6CFCF92DF92EF92FF920F931F93E0
:106CC000CF93DF93EC01A881B981109781F18C916A
:106CD000882369F108811981F8019081992351F085
:106CE0009D3241F090539A3028F00F5F1F4F198367
:106CF0000883F0CFC8010F9460506B017C016CE2F7
:106D000070E0C8010F94C65C009769F4198218827C
:106D1000C701B601DF91CF911F910F91FF90EF90C6
:106D2000DF90CF900895019699838883F1CFC12C8D
:106D3000D12C7601EDCF0097B1F1FC01DB01AC0164
:106D4000405F5F4F80E090812FE9290F263098F453
:106D500097559295907F9C9321813FE9320F363071
:106D6000B0F42755922B9D933296E417F50759F707
:106D700091E0892708952FEB290F263010F49753BF
:106D8000E8CF90539A3028F381E090E0E2CF3FEBD8
:106D9000320F363010F42753E5CF20532A3010F34A
:106DA00081E020E0DFCF80E008950097D1F0DC01A2
:106DB0001696ED91FC913097A1F080858F7084300C
:106DC00021F481859285009771F40680F781E02D8A
:106DD000309739F080858F70843019F481859285E1
:106DE000089590E080E0089508950F931F93CF9346
:106DF000DF93EC010A811B8170E060E0C8010E9412
:106E00008EB01816D4F48A8761E070E0C8010E9441
:106E10008EB0181619069CF49987888762E070E096
:106E2000C8010E948EB01816190664F49C878B87DF
:106E3000DF91CF911F910F91089583E0E4CF8BE212
:106E400090E0EACF88E590E0F1CF089508950895A5
:106E500008950F931F93CF93DF93EC011D860A8152
:106E60001B8170E060E0C8010E948EB087FD44C0C5
:106E70008C838C818150853410F080E28C8361E0BA
:106E800070E0C8010E948EB087FD3BC08D838D816C
:106E90008150853410F081E28D8362E070E0C8019A
:106EA0000E948EB0863490F58E8363E070E0C80156
:106EB0000E948EB09C01215031092115344040F5CB
:106EC0009A87898764E070E0C8010E948EB08130A3
:106ED00024E0920700F59C878B8765E070E0C8018D
:106EE0000E948EB018161906CCF498878F83DF9114
:106EF000CF911F910F91089581958C8381E08D87AB
:106F0000B8CF81958D8381E08D87C1CF1E82CDCF93
:106F10001A861986D7CF80E094E0DDCF80E197E232
:106F2000E4CF08950895CF93DF93EC0162ED72E111
:106F300089E390E10F94E4236DEC72E189E390E141
:106F40000F94E4236C817D814AE050E089E390E175
:106F50000F94852367EC72E189E390E10F94E423B9
:106F600089E390E10F94782261E08C810E9448FED1
:106F70006E818C810E941AFE8A819B81009729F084
:106F800040E050E0BA010E94C1AFE881F981048479
:106F9000F585E02D62E0CE0119958A819B810097ED
:106FA00081F00E94F2B9181619065CF40A80DB81A0
:106FB000C02D80E00F94C542AB01BC01CE010E9400
:106FC000C1AF81E090E0DF91CF910895CF93DF933F
:106FD000EC0164EA72E189E390E10F94E4236C81AF
:106FE0007D814AE050E089E390E10F94852362EAD5
:106FF00072E189E390E10F94E423EA81FB8102804E
:10700000F381E02D6081718189E390E10F94CE23BB
:107010006CE972E189E390E10F94E42389E390E164
:107020000F9478228A819B81892B09F451C08C812D
:107030009D81892B09F04CC0E881F981008CF18D8C
:10704000E02DCE0119958130910529F0029759F074
:1070500061E08C811AC063E070E0CE010E9425E6F9
:1070600061E00E9448FE61E08C810E9448FE61E080
:1070700070E0CE010E9425E661E00E9448FE62E0D9
:1070800070E0CE010E9425E661E00E9448FE8091FA
:10709000A100887F8093A10080919100887F8093D8
:1070A00091008091A10082608093A1008091910065
:1070B000826080939100E881F9810484F585E02D58
:1070C00062E0CE01199581E090E0DF91CF910895C3
:1070D00090E080E0FACF2F923F924F925F926F92B2
:1070E0007F928F929F92AF92BF92CF92DF92EF9258
:1070F000FF920F931F93CF93DF93CDB7DEB76697C1
:107100000FB6F894DEBF0FBECDBF9A838983DC0132
:107110001496ED91FC91309709F4D3C12680378005
:107120002114310409F493C1D101ED91FC91309700
:1071300009F489C18081882309F485C12FEF3FEFCD
:10714000A90161E276E0C1010E94692722E030E0F6
:1071500040E050E06CE176E0C1010E9469272FEF2A
:107160003FEFA90161E376E0C1010E94692765E76D
:1071700075E0C1010E943AED4C01009709F463C12A
:10718000FC0180858F70853009F05DC1C4010E94CB
:107190007DEE833008F457C167E176E0C1010E94BB
:1071A000A4FD6C016AE376E0C1010E94A4FD9C830A
:1071B0008B832EEF3FEF4FEF5FEF65EC75E0C10182
:1071C0000E9469278C0120E030E040E85FE370E036
:1071D00060E0C4010F9409422B013C0120E030E043
:1071E000A9010F94A356F12C87FF06C077FA70947B
:1071F00077F87094FF24F39420E030E0A90161E077
:1072000070E0C4010F9409426F83788789879A8759
:1072100020E030E0A90162E070E0C4010F9409426F
:107220006D877E878F87988B20E030E040EA50E4BE
:1072300063E070E0C4010F940942698B7A8B8B8BF9
:107240009C8B6EE376E089E390E10F94CE232B8153
:107250003C81275F3F4F3E8B2D8BA901330F660B7F
:10726000770B2AE030E089E390E10F943D2368ED4D
:1072700079E089E390E10F94CE23C80109969C83BD
:107280008B83AC01990F660B770B2AE030E089E322
:1072900090E10F943D2366E576E089E390E10F9459
:1072A000CE23D6011996BE83AD83AD01BB0F660B0D
:1072B000770B2AE030E089E390E10F943D2389E3E6
:1072C00090E10F9478228CE390E00F94754E9C87A8
:1072D0008B871F92FF92B889BF93EF85EF93FE854E
:1072E000FF932D852F93AF80B884C984DA848301FE
:1072F00072012D813E814B815C816D897E898B85F8
:107300009C850F94D027EB85FC85CF01FF0FAA0B3E
:10731000BB0BF40181879287A387B48767E476E08B
:1073200089E390E10F94CE23D4011996ED91FC915D
:10733000448D558D052E000C660B770B2AE030E04E
:1073400089E390E10F943D2368ED79E089E390E1D2
:107350000F94CE23D4011996ED91FC91468D578D53
:10736000052E000C660B770B2AE030E089E390E1F4
:107370000F943D2366E576E089E390E10F94CE23F8
:10738000D4011996ED91FC9140A151A1052E000C5C
:10739000660B770B2AE030E089E390E10F943D2300
:1073A00089E390E10F94782261E070E0F401818537
:1073B00092850F94312720E030E04AE754E4698950
:1073C0007A898B899C890F9409570F947559D40138
:1073D00019968D919C910F94832765E870E189E35C
:1073E00090E10F94E423B301A20189E390E10E94AC
:1073F00080F260E576E089E390E10F94CE234F813F
:10740000588569857A8589E390E10E9480F264E578
:1074100076E089E390E10F94CE233D852E859F850C
:107420008889432F522F692F782F89E390E10E949A
:1074300080F289E390E10F9478220F900F900F90E3
:107440000F900F900F90F1012280338069CE6AE790
:1074500070E189E390E10F94E42389E390E10F94D4
:10746000782240E050E0BA01A981BA8112968D914C
:107470009C910E94C1AFA981BA81ED91FC911197B5
:107480000484F585E02D62E0CD01199581E090E05E
:1074900066960FB6F894DEBF0FBECDBFDF91CF91D9
:1074A0001F910F91FF90EF90DF90CF90BF90AF9022
:1074B0009F908F907F906F905F904F903F902F9014
:1074C000089566E670E189E390E10F94E42389E38F
:1074D00090E10F94782290E080E0DACFCF93DF93B1
:1074E000EC010E94293768E576E089E390E10F948A
:1074F0007C2261E08C810E9448FE61E08D810E94C7
:1075000048FE6D858C810E941AFE6D858D810E94DA
:107510001AFE60E08E810E9448FE40E050E0BA0111
:107520008A819B810E94C1AF40E050E061E070E041
:107530008A819B810E946DB140E050E062E070E082
:107540008A819B810E946DB1E881F9810484F5856F
:10755000E02D62E0CE01199582E08093270281E060
:1075600090E0DF91CF9108956F927F928F929F92DA
:10757000AF92BF92CF92DF92EF92FF920F931F9341
:10758000CF93DF933C01DC0114968D919C9115976C
:10759000892B71F41296CD91DC9184E190E00F94E7
:1075A000754EBC01CE010E947EAFE3019D838C83AA
:1075B000F301C481D581209769F466E77DE082E913
:1075C0009FE00F94E42382E99FE00F94782290E0FB
:1075D00080E0B1C280E00F94C5426E837F838887CC
:1075E0009987D3011496ED90FC901597E114F1045E
:1075F000D1F01296ED91FC913097A9F0C481D5811C
:10760000209789F088858F70853069F4CE010E94BB
:107610007DEE823040F00091890A10918A0A0115AE
:10762000110509F096C069E37DE082E99FE00F94BF
:10763000E42361E070E0E3018C819D81892B11F4EA
:1076400070E060E04AE050E082E99FE00F9485231B
:1076500067E37DE082E99FE00F94E42361E070E05E
:10766000F30182819381892B11F470E060E04AE09C
:1076700050E082E99FE00F94852365E37DE082E995
:107680009FE00F94E423D3011296ED91FC9161E009
:1076900070E084819581892B11F470E060E04AE00C
:1076A00050E082E99FE00F94852363E37DE082E967
:1076B0009FE00F94E423E301EA81FB810480F581DC
:1076C000E02D80858F7061E070E0853011F470E00E
:1076D00060E04AE050E082E99FE00F94852361E397
:1076E0007DE082E99FE00F94E423D3011296ED91AF
:1076F000FC91848195810E947DEE61E070E0823092
:1077000010F070E060E04AE050E082E99FE00F9402
:10771000852382E99FE00F9478226EE47DE082E980
:107720009FE00F94E42382E99FE00F947822D30135
:10773000ED91FC910484F585E02D61E0C30119957C
:10774000E301E881F9810084F185E02DC3011995F9
:107750003ECF61E0CE010E94ECEDEC0188858F7098
:10776000843029F469857A856115710539F469E1F8
:107770007DE082E99FE00F94E423CBCFC8010E9413
:107780003AED8C01009769F467EF7CE082E99FE0B5
:107790000F94E42369857A8582E99FE00F94CE23D4
:1077A000B8CF64E676E00E943AED009709F4D2C0C3
:1077B000EC0128852F70243009F0CCC0C984DA840C
:1077C000D0E0C0E0C114D10409F4B7C0BE016D5AC5
:1077D000734FC6010F94AE50892B09F0A9C0FE016A
:1077E000E95AF34F25913491922F832FF701928319
:1077F00083836BE676E0C8010E943AEDE301EC81F9
:10780000FD81009709F4AEC0DC0118962C91189701
:107810002F70223009F0A6C019968D919D910D9080
:10782000BC91A02D0097A105B10509F49BC09183DF
:10783000808340815181052E000C660B770B2281DD
:107840008AED9CE00F94312560E776E0C8010E9444
:107850003AED7C01F301C481D581009709F488C019
:10786000DC0118968C918F70863009F081C065E735
:1078700076E0C7010E943AED9B878A876AE776E047
:10788000C7010E943AED9D878C876EE776E0C701BD
:107890000E943AED9F878E8764E876E0C7010E94D8
:1078A0003AED998B888B69E876E0C7010E943AED42
:1078B000009709F45AC0FC01818592859D838C83D1
:1078C0006FE876E0C8010E943AED9B8B8A8B892B8A
:1078D00009F40FC161EE7CE089E390E10F94E423A9
:1078E00089E390E10F947822D3011496ED91FC91F5
:1078F0000288F389E02DC681D781209709F441C021
:1079000063E976E0CE010E943AED009769F0FC0150
:1079100020852F70213041F48185882329F06881EA
:107920007981C3010E940D2F0A80DB81C02DE5CF34
:107930002696C834D10509F045CF66E37CE089E39B
:1079400090E10F94E42389E390E10F94782296E08C
:1079500080E04CCF86E090E0D70113969C938E9305
:10796000129747CF80E895E262CF88EE93E0A6CFEA
:107970001B861A8688EE93E09D838C831D861C8669
:107980009FCF6BEC7CE089E390E10F94E42389E3E3
:1079900090E10F947822D3011496ED91FC91028826
:1079A000F389E02DE680F780E114F10409F47BC04F
:1079B00067EE75E0C7010E943AED009709F468C0D0
:1079C0006CE976E00E943AED8C01009709F460C002
:1079D000EC0188858F70823009F04EC0C984DA844A
:1079E000D3011496ED91FC910288F389E02D309734
:1079F00009F456C0C681D78146010D2C000CAA0897
:107A0000BB08209709F44CC060EA76E0CE010E94E2
:107A10003AED009709F440C0FC0120852F70223018
:107A2000D9F581859285A385B48588159905AA0520
:107A3000BB0591F56AEA7CE089E390E10F94E423C9
:107A40006881798189E390E10F94CE236BE97CE032
:107A500089E390E10F94E4234AE050E0B60189E322
:107A600090E10F94852389E390E10F947822688157
:107A70007981C3010E940D2FF80180858F708430B9
:107A800039F4D80119966D917C91C3010E940D2F94
:107A9000E701EA80FB8088CF0A80DB81C02DB1CF6F
:107AA00070E060E0E6CF61EB7CE089E390E10F9469
:107AB000E42389E390E10F947822D3011296ED91AB
:107AC000FC9162E0848195810E94ECED009789F041
:107AD000FC01C681D781209761F0CE010E94451B31
:107AE000882319F0CE010E9448FD0A80DB81C02D59
:107AF000F2CF61E67DE088E89FE00F94E423D301B4
:107B00001296ED91FC910280F381E02D60817181EC
:107B100088E89FE00F94CE2388E89FE00F947822B6
:107B2000E301E881F9810484F585E02D62E0C30179
:107B3000199581E090E0DF91CF911F910F91FF9017
:107B4000EF90DF90CF90BF90AF909F908F907F90FD
:107B50006F900895CF93DF93EC0161ED7BE089E3B3
:107B600090E10F94E423EA81FB810280F381E02D10
:107B70006081718189E390E10F94CE2389E390E1E4
:107B80000F947822E881F9810484F585E02D62E084
:107B9000CE01199581E090E0DF91CF910895DC014D
:107BA000ED91FC910484F585E02D62E0199581E06A
:107BB00090E008950F931F93CF93DF93DC0112960B
:107BC0002D913C91232B81F1EC0163E67AE089E36E
:107BD00090E10F94E4234AE050E06E8189E390E164
:107BE0000F949B2289E390E10F9478228C819D81F0
:107BF000892B61F40A811B818CE290E00F94754E11
:107C0000BC01C8010E947EAF9D838C83EC81FD8105
:107C1000309769F461E57AE082E99FE00F94E4230C
:107C200082E99FE00F94782290E080E044C085E2F2
:107C3000DF011D928A95E9F7EC81FD8116A2EC81A6
:107C4000FD8115A2EC81FD8117A20C811D8180E0D0
:107C50000F94C542F80160A771A782A793A78E81F0
:107C6000811116C062E00E9448FE68E17AE088E86F
:107C70009FE00F94E42388E89FE00F9478228CE93A
:107C80009FE00F94381B1092450281E0809386118B
:107C900026E040E855E260E070E08F8198850F941F
:107CA0003125E881F9810484F585E02D62E0CE017B
:107CB000199581E090E0DF91CF911F910F91089588
:107CC0002F923F924F925F926F927F928F929F92EC
:107CD000AF92BF92CF92DF92EF92FF920F931F93DA
:107CE000CF93DF93CDB7DEB7CB57D1090FB6F8945A
:107CF000DEBF0FBECDBF3C01362EE296EFAEE2975F
:107D0000E396FFAEE397E4960FAFE497E5961FAFD7
:107D1000E597E6962FAFE697E7963FAFE797E896A9
:107D20004FAFE897E9965FAFE997EA96CFAEEA974B
:107D3000EB96DFAEEB97EC96AFAEEC972B2C2401D5
:107D400080914502893020F4809144028930C0F04E
:107D5000C3010E94F0F58C01892B91F064EA76E072
:107D600089E390E10F94CE23B80189E390E10F9469
:107D7000CE2389E390E10F947822C8010F94114F2C
:107D80006114710409F47CC1F30180858F70843023
:107D900009F461C128F4882309F466C180E02FC08A
:107DA000853009F446C08630C9F76AEA76E0C30137
:107DB0000E943AED2C01009709F476C0912C812C99
:107DC000B12CA12CD12CC12CE296EFACE297E3961A
:107DD000FFACE397E4960FADE497E5961FADE5970A
:107DE000E6962FADE697E7963FADE797E8964FAD5D
:107DF000E897E9965FADE997632D0E94603EC5580C
:107E0000DF4F0FB6F894DEBF0FBECDBFDF91CF912D
:107E10001F910F91FF90EF90DF90CF90BF90AF90A8
:107E20009F908F907F906F905F904F903F902F909A
:107E3000089580919E118F5F80939E116680778058
:107E40006114710459F14201EC96AFACEC97B22C7D
:107E5000EA96CFACEA97EB96DFACEB97E296EFAC05
:107E6000E297E396FFACE397E4960FADE497E596CF
:107E70001FADE597E6962FADE697E7963FADE797FE
:107E8000E8964FADE897E9965FADE997632DC3019A
:107E90000E94603EF30162807380D2CF80919E1178
:107EA000815080939E117ACF6EEA76E0C3010E94E2
:107EB0003AED7C0163EB76E0C3010E943AED6C0180
:107EC00068EB76E0C3010E943AED332039F0F1E02F
:107ED0003F1609F4A1C010E000E00CC06CEB76E0A6
:107EE000C3010E943AED2C0161EC76E0C3010E94CF
:107EF0003AED8C014114510409F4230101151105D7
:107F000009F48301E114F10431F4EA96EFACEA9745
:107F1000EB96FFACEB97C114D10421F4EC96CFACF7
:107F2000EC97D22C4114510409F4A7C0F2018085CA
:107F30008F70843009F0A1C061847284011511052D
:107F400009F4AAC0F80180858F70843009F0A4C0BC
:107F50004184528410E000E0E114F10409F401C10D
:107F60006114710409F4BFC06AE174E189E390E12E
:107F70000F94E423F7016185728589E390E10F9402
:107F8000CE2365E174E189E390E10F94E423B3012A
:107F900089E390E10F94CE2389E390E10F94782256
:107FA000CE018F589F4F0E94B578C114D10409F0BB
:107FB000E1C0F70180858F70843009F090C1409155
:107FC000A2115091A31161857285CE0101960E9484
:107FD0002CB8CE0101960E9471AF8823C1F00E9497
:107FE00006356B01683C71050CF091C064ED73E1DE
:107FF00082E99FE00F94E4234AE050E0B60182E971
:108000009FE00F94852382E99FE00F947822CE01B0
:1080100001960E94B6B863C166EC76E0C3010E9487
:108020003AED2C016BEC76E0C3010E943AED8C0135
:108030004114510409F055C16CEB76E0C3010E9474
:108040003AED2C010115110509F44ECF892B09F0E9
:1080500059CF230157CF10E000E0512C412CD12CF7
:10806000C12CF12CE12C46CF10E000E0512C412C2A
:10807000D12CC12CF12CE12C45CF712C612C5ECF81
:10808000EC96CFACEC97D22CEA96EFACEA97EB9655
:10809000FFACEB97712C612C00E020E030E340E175
:1080A00050E0BE016F597F4FCE018F589F4F0E9405
:1080B00095762C01E4960FADE49710E001151105BB
:1080C00009F04ACFE2968FADE297811109C0E3969D
:1080D0008FADE3978F7009F43FCF02E010E03CCF03
:1080E00001E010E039CF6BE074E189E390E10F9497
:1080F000E423F7016185728589E390E10F94CE2333
:1081000066E074E189E390E10F94E42349CF6114C0
:10811000710431F0B301CE0101960E942FF677CFA2
:10812000A12CC12CF12CE12CE2960FADE297E39645
:108130001FADE397E4962FADE497E5963FADE59745
:10814000E6964FADE697E7965FADE797E8966FAD99
:10815000E897E9967FADE997CE0101960E9401BBB1
:1081600056CFC114D10409F4BAC04114510409F422
:10817000B6C004C04114510409F41BCFF601808538
:108180008F70843009F0A7C08185928525961FAE37
:108190001EAE259748EE53E060E070E029964CAFA4
:1081A0005DAF6EAF7FAF299724E532E023963FAFF6
:1081B0002EAF23972F969FAF8EAF2F9761961FAE4E
:1081C0001EAE619763961FAE1EAE639765961FAE97
:1081D0001EAE659767961FAE1EAE679769961FAF76
:1081E0000EAF69976A961FAE6A9740E450E0BE01F1
:1081F0006F5F7F4FCE018F5B9F4F0E94E2EE21E0C9
:1082000030E02C0F3D1F820F931FFC0110826EEF98
:1082100073E189E390E10F94E423F60161857285AF
:1082200089E390E10F94CE2360ED76E089E390E15D
:108230000F94CE23BE016F5F7F4F89E390E10F94CF
:10824000CE2369EF73E189E390E10F94E423B20157
:1082500089E390E10F94CE2389E390E10F94782293
:108260000E9458ED8823B9F18091390C811133C0F7
:108270006FE270E0CE0101960F94C65C892B51F439
:10828000F6012185328543E050E060E4CE0101969D
:108290000E94853362EF73E189E390E10F94E42358
:1082A000BE016F5F7F4F89E390E10F94CE236DEEA7
:1082B00073E189E390E10F94E423B20189E390E153
:1082C0000F94CE2389E390E10F947822B201CE017E
:1082D00001960F941C03E114F10409F06ACE81E0C9
:1082E0008ECD892B09F00ECEFFCD8F929F92AF924B
:1082F000BF92CF92DF92EF92FF920F931F93CF9393
:10830000DF9300D000D01F921F92CDB7DEB7198245
:108310001A821B821C821D821E821F821886FA808E
:108320002F2D207FF22E912C812CB12CA12CD12C21
:10833000C12CE9800B811C8120E03E814F81588552
:108340000E94603E28960FB6F894DEBF0FBECDBFE8
:10835000DF91CF911F910F91FF90EF90DF90CF9021
:10836000BF90AF909F908F9008958F929F92AF9201
:10837000BF92CF92DF92EF92FF920F931F93CF9312
:10838000DF9300D000D01F921F92CDB7DEB7DC0183
:108390001296ED91FC91309709F468C024813581E3
:1083A000232B09F463C08C01662309F472C00E9478
:1083B0000F26E62EB72E6C01D8011296ED91FC9196
:1083C0000280F381E02D6081718182E99FE00F944A
:1083D000CE2360E372E182E99FE00F94E42382E917
:1083E0009FE00F94782220E030E0A9016E2D7B2DD4
:1083F000C6010F94AB5987FD39C064E272E182E98E
:108400009FE00F94E4234E2D5B2DB60182E99FE09F
:108410000E9480F282E99FE00F947822D8011296A0
:10842000ED91FC9161E0848195810E94ECED1982CF
:108430001A821B821C822A81207F2760F22E2E2D19
:108440004E2D5B2DB6014D835E836F837887912C13
:10845000812CB12CA12CD12CC12CE9800B811C8149
:108460003E814F8158856FEF0E94603E28960FB67F
:10847000F894DEBF0FBECDBFDF91CF911F910F915A
:10848000FF90EF90DF90CF90BF90AF909F908F9034
:1084900008950280F381E02D6081718188E89FE07A
:1084A0000F94CE236DE372E188E89FE00F94E423FC
:1084B00088E89FE028960FB6F894DEBF0FBECDBFC8
:1084C000DF91CF911F910F91FF90EF90DF90CF90B0
:1084D000BF90AF909F908F900D9478224F925F92B3
:1084E0006F927F928F929F92AF92BF92CF92DF92C4
:1084F000EF92FF920F931F93CF93DF93CDB7DEB729
:10850000E8970FB6F894DEBF0FBECDBF09AB1AAB2C
:108510002BAB3CAB4DAB5EAB6FAB78AFDC011496D5
:10852000ED91FC91309719F490E080E0CAC0208171
:108530003181232BC9F33C01DC01ED91FC910284D4
:10854000F385E02D1995029779F78BA9E82EF12C88
:1085500019A9112321F0E114F10409F432C1823088
:1085600009F4D8C0B8F4882309F4D4C08130B9F034
:1085700060E572E189E390E10F94E4234AE050E082
:10858000B70189E390E10F94852389E390E10F948B
:108590007822CACF833009F446C0893049F7D30125
:1085A0001296ED91FC9161E0848195810E94ECED41
:1085B0002C0119A61AA61BA61CA61DA61EA61FA640
:1085C00018AA8AA5807F8AA719A761E0CE0189969B
:1085D0000E94507329A33AA34BA35CA36DA37EA36F
:1085E0008FA398A71150153108F0FCC1E12FF0E0DE
:1085F0008827E250FD4B8F4F0D9464582744E54384
:10860000F244F244F244F244F244F244F244564456
:10861000B644F244F24427442744F244F244F2447C
:108620002744274427448AA98F7009F47DCFCE01BF
:10863000C1960E949F75D3011496ED91FC916683BB
:1086400077838087918766E972E189E390E10F94EF
:10865000E423D3011296ED91FC910280F381E02D89
:108660006081718189E390E10F94CE2368E872E123
:1086700089E390E10F94E423D3011496ED91FC91EA
:10868000468157816085718589E390E10E9480F27F
:1086900089E390E10F947822F301E480F5800F9450
:1086A0007F02D70152966D937D938D939C9355973E
:1086B000D3011496ED91FC918689811119C081E056
:1086C00090E0E8960FB6F894DEBF0FBECDBFDF9105
:1086D000CF911F910F91FF90EF90DF90CF90BF90BF
:1086E000AF909F908F907F906F905F904F90089584
:1086F000168A60E0C3010E94B541D3011496ED9142
:10870000FC9180E090E0A0E0B0EC86879787A08B9A
:10871000B18BD5CF8AA98F7009F406CFCE01C1964F
:108720000E949F75D3011496ED91FC916287738727
:108730008487958762E872E189E390E10F94E423EE
:10874000D3011296ED91FC910280F381E02D6081BE
:10875000718189E390E10F94CE2367E772E189E3A9
:1087600090E10F94E423D3011496ED91FC9142859E
:1087700053856485758589E390E10E9480F289E3E1
:1087800090E10F947822D3011296ED91FC9162E072
:10879000848195810E94ECED009709F490CF912C93
:1087A000812CB12CA12CD12CC12CE9A8FAA80BA9A1
:1087B0001CA92DA93EA94FA958AD6FEF0E94603E9C
:1087C0007ECFEE24E394F12CEACE80913A0C909186
:1087D0003B0C0597F1F019821A821B821C821D82C4
:1087E0001E821F8218868A81807F8A836BE0CE0179
:1087F00001960E947273912C812CB12CA12CD12C4A
:10880000C12C79018A019B01AC016FEFC2010E946A
:10881000603E912C812CB12CA12CD12CC12CE9A42F
:10882000FAA40BA51CA52DA53EA54FA558A96FEF31
:10883000C2010E94603E30E020E040E050E460E091
:1088400070E0F301828193810E9429B538CF1982AB
:108850001A821B821C821D821E821F8218868A81B8
:10886000807F8A8340E051E060E070E0D30112969F
:108870008D919C910E94BFB1672B682B692BA1F051
:108880006BE0CE0101960E947273912C812CB12C69
:10889000A12CD12CC12C79018A019B01AC016FEF75
:1088A000C2010E94603EBBCF6AE0EBCF80913A0CE0
:1088B00090913B0C059791F061E0D30112968D9158
:1088C0009C910E94C1B730E020E040E050E160E0C0
:1088D00070E0F301828193810E9429B540E050E06D
:1088E00061E070E0D30112968D919C910E9496B147
:1088F000912C812CB12CA12CD12CC12CE9A4FAA44F
:108900000BA51CA52DA53EA54FA558A96FEFC2012B
:108910000E94603ED301ED91FC910288F389E02D25
:10892000C3011995892B09F4E8CE19821A821B829A
:108930001C821D821E821F8218868A81807F8A8304
:1089400061E0CE0101960E94727329873A874B87B6
:108950005C876D877E878F87988B79018A019B0161
:10896000AC016FEFC2010E94603EC7CE912C812CFA
:10897000B12CA12CD12CC12CE9A4FAA40BA51CA5C7
:108980002DA53EA54FA558A96FEFC2010E94603EDC
:10899000D301ED91FC910288F389E02DC301199573
:1089A000892B09F08CCE19861A861B861C861D869B
:1089B0001E861F86188A8A85807F8A8762E0CE019C
:1089C00009960E94727329833A834B835C836D837B
:1089D0007E838F83988779018A019B01AC016FEFB9
:1089E000C201ECCE65E672E189E390E10F94E423E5
:1089F0004AE050E069A989E390E10F949B2289E362
:108A000090E10F947822B4CD2F923F924F925F92D3
:108A10006F927F928F929F92AF92BF92CF92DF928E
:108A2000EF92FF920F931F93CF93DF93CDB7DEB7F3
:108A300064970FB6F894DEBF0FBECDBF1C01DC01FA
:108A400014968D919C911597892B99F41296ED911E
:108A5000FC91FA83E98389E190E00F94754EBC01A3
:108A600089819A810E947EAFD10115969C938E9345
:108A70001497F101048115810115110569F465EC64
:108A800071E182E99FE00F94E42382E99FE00F9473
:108A9000782290E080E09CC3D8011D921C92028055
:108AA000F381E02DFC8BEB8B309791F084819581E5
:108AB0009A838983009761F0DC0118968C9118974E
:108AC0008F70853029F4CD010E947DEE811190C018
:108AD0006BE871E182E99FE00F94E42361E070E0CC
:108AE000F10184819581892B11F470E060E04AE006
:108AF00050E082E99FE00F94852369E871E182E903
:108B00009FE00F94E42361E070E0D10112968D9113
:108B10009C91892B11F470E060E04AE050E082E91A
:108B20009FE00F94852367E871E182E99FE00F944D
:108B3000E423D1011296ED91FC9161E070E0848113
:108B40009581892B11F470E060E04AE050E082E901
:108B50009FE00F94852365E871E182E99FE00F941F
:108B6000E423D1011296ED91FC910480F581E02D72
:108B700080858F7061E070E0853011F470E060E016
:108B80004AE050E082E99FE00F94852363E871E1B9
:108B900082E99FE00F94E423D1011296ED91FC91BC
:108BA000848195810E947DEE61E070E0823010F05A
:108BB00070E060E04AE050E082E99FE00F94852396
:108BC00082E99FE00F9478226FE971E182E99FE0EA
:108BD0000F94E42382E99FE00F947822D101ED9174
:108BE000FC910484F585E02D61E0C101199551CF18
:108BF00060E089819A810E94ECED9F838E830097CB
:108C000029F0FC0180858F70853039F069E671E1CB
:108C100082E99FE00F94E423D3CF8E819F810E944D
:108C20007DEE8150883008F0A3C1E82FF0E088275E
:108C3000E35EF94B8F4F0D94645889475F47324785
:108C4000AD46954695467E46254667E08E819F81D6
:108C50000E94ECEDFC0190859F70933009F041C0BB
:108C60004184528463847484F1E0FD8366E08E81E4
:108C70009F810E94ECEDFC0190859F70933009F07C
:108C800045C081859285A385B48589839A83AB830A
:108C9000BC8391E09D8364E08E819F810E94ECED16
:108CA000FC0190859F70933009F050C061857285FA
:108CB000838594850F947C594B0163E08E819F815D
:108CC0000E94ECEDFC0180858F70833009F060C05C
:108CD00081859285A385B4858A879B87AC87BD876C
:108CE00064C0923059F461857285838594850F94B0
:108CF000AA562B013C0181E08D83B8CF412C512C29
:108D00008FE7682E83E4782E1D82B0CF9230C9F4AD
:108D100061857285838594850F94AA5669837A83C9
:108D20008B839C83A1E0AD83B6CF412C512CBFE750
:108D30006B2EB3E47B2E19821A821B821C821D8249
:108D4000AACF19821A821B821C82A5CF9230C1F44D
:108D500081849284A384B484B0CFF0EC8F2EF7E2A8
:108D60009F2EF9E0AF2EB12C412C512CAFE76A2E8B
:108D7000A3E47A2E19821A821B821C821D829DCF47
:108D8000E0EC8E2EE7E29E2EE9E0AE2EB12C95CFE0
:108D9000823009F082C061857285838594850F9445
:108DA000AA566A877B878C879D8762E08E819F8128
:108DB0000E94ECEDFC0180858F70833009F072C059
:108DC00091859E87A285AF87B385B88B8485898B73
:108DD00061E08E819F810E94ECEDFC0180858F70A7
:108DE000833009F08BC0C184D284E384F48460E0D2
:108DF0008E819F810E94ECEDFC0180858F70833015
:108E000009F0A9C081859285A385B4858E839F834F
:108E1000A887B98720E030E0A9016E817F8188852D
:108E200099850F94A35687FFD0C08E819F81A88516
:108E3000B985B0588E839F83A887B98791E09A8BB4
:108E4000AB89BC891696ED91FC9180858F7082303C
:108E500009F4BDC0833009F4D4C180E090E0A0EAF9
:108E6000B1E4D3C160EC862E67E2962E69E0A62EAF
:108E7000B12C80E090E0A0EAB0E48A879B87AC87C1
:108E8000BD87412C512C7FE7672E73E4772E198222
:108E90001A821B821C821D8288CF80E090E0A0EAAB
:108EA000B0E41ACF823029F5618572858385948577
:108EB0000F94AA566E877F87888B998B89CF40EC59
:108EC000842E47E2942E49E0A42EB12C80E090E05D
:108ED000A0EAB0E48A879B87AC87BD87412C512CE0
:108EE0005FE7652E53E4752E19821A821B821C825D
:108EF0001D821E861F86188A198A6ACF823039F52C
:108F000061857285838594850F94AA566B017C01D7
:108F10006ECF20EC822E27E2922E29E0A22EB12CD9
:108F200080E090E0A0EAB0E48A879B87AC87BD87A9
:108F3000412C512C3FE7632E33E4732E19821A82A1
:108F40001B821C821D821E861F86188A198AC12CCC
:108F5000D12C76014CCF823091F561857285838565
:108F600094850F94AA566E837F838887998752CF02
:108F700080EC882E87E2982E89E0A82EB12C80E024
:108F800090E0A0EAB0E48A879B87AC87BD87412C3C
:108F9000512C9FE7692E93E4792E19821A821B8245
:108FA0001C821D821A8A1E861F86188A198AC12C65
:108FB000D12C7601CE82DF82E886F98641CF1A8AEB
:108FC0001E821F82188619863BCF1A8A39CF618587
:108FD0007285838594850F94AA56F80162877387FA
:108FE00084879587D80116961D921D921D921C921A
:108FF0001997F80112821382148215820F947F024E
:10900000D80152966D937D938D939C935597D10182
:109010001496ED91FC9181E0868B908E878A61E0B9
:10902000C1010E94B541F10104811581D8018D91E2
:109030009C9160E571E1892B09F0EACD8CE390E029
:109040000F94754E9C8B8B8B9801265F3F4FA80128
:109050004E5F5F4FB8016A5F7F4F1F92BA89BF931F
:10906000E989EF93F889FF938F858F939E859F936E
:1090700056016701EE80FF80088519858B899C89E0
:109080000F94D027D1011496ED91FC918B899C8986
:10909000918380830F900F900F900F900F900F90FF
:1090A000009709F491CD61E070E00F943127D10170
:1090B0001496ED90FC90BD81BB2309F44AC0A30136
:1090C000920169817A818B819C810F94AB5987FFD2
:1090D00040C0F7010190F081E02DFF83EE8389818C
:1090E0009A81AB81BC8182AB93ABA4ABB5AB46AAF2
:1090F00057AA60AE71AE82AD882359F1068D178DE7
:10910000F80180809180A280B380A5019401C30101
:10911000B2010F94A35687FF7EC0D8014D925D9295
:109120006D927C921397AE81BF8196968D909D90A3
:10913000AD90BC909997A5019401C301B2010F9421
:10914000A35687FF7DC0EE81FF8146A257A260A68D
:1091500071A620E030E04AE754E46A857B858C857F
:109160009D850F9409570F947559D7018D919C9146
:109170000F94832761EB71E188E89FE00F94E4236B
:10918000D1011296ED91FC910280F381E02D608176
:10919000718188E89FE00F94CE2388E89FE00F94C8
:1091A0007822D1011496ED91FC9180E090E0A0E04E
:1091B000B0EC86879787A08BB18BD101ED91FC91A4
:1091C0000484F585E02D62E0C101199581E090E00D
:1091D00064960FB6F894DEBF0FBECDBFDF91CF917E
:1091E0001F910F91FF90EF90DF90CF90BF90AF90C5
:1091F0009F908F907F906F905F904F903F902F90B7
:10920000089581859285A385B485F8018287938727
:10921000A487B587E7CEA501940169817A818B8106
:109220009C810F94AB5918160CF07DCF89819A81DF
:10923000AB81BC81F80180839183A283B38373CF18
:10924000A501940169817A818B819C810F94AB592E
:1092500018160CF07ECF89819A81AB81BC81EE819A
:10926000FF8186A397A3A0A7B1A773CF4F925F9268
:109270006F927F928F929F92AF92BF92CF92DF9226
:10928000EF92FF920F931F93CF93DF93CDB7DEB78B
:1092900060970FB6F894DEBF0FBECDBF6130710589
:1092A00009F4DBC1DC011496ED91FC913097C9F40F
:1092B00081E090E060960FB6F894DEBF0FBECDBFA0
:1092C000DF91CF911F910F91FF90EF90DF90CF90A2
:1092D000BF90AF909F908F907F906F905F904F90D6
:1092E000089520813181232B19F33C01DC01ED919C
:1092F000FC910284F385E02D19950297C9F6F301DC
:10930000E280F380E114F10499F2C7010E94E0B712
:10931000823071F240E051E060E070E0C7010E94ED
:10932000BFB1672B682B692B19F6D3011496ED9109
:10933000FC9180819181FC0122AD222309F455C169
:109340000F949325882309F450C1D3011496ED910D
:10935000FC9186898823A1F0C3010E940F266B012E
:109360007C0120E030E0A9010F94AB5987FD08C0D3
:10937000D3011496ED91FC91C282D382E482F582EE
:1093800064E072E189E390E10F94E423D301129643
:10939000ED91FC910280F381E02D6081718189E380
:1093A00090E10F94CE236EEF71E189E390E10F9489
:1093B000E423D3011496ED91FC9142855385648595
:1093C000758589E390E10E9480F269EF71E189E39C
:1093D00090E10F94E423D3011496ED91FC91468122
:1093E00057816085718589E390E10E9480F263ED89
:1093F00076E089E390E10F94CE23D3011496ED91AA
:10940000FC91428153816481758189E390E10E94DE
:1094100080F265EF71E189E390E10F94E423D301D9
:109420001496ED91FC910190F081E02D40815181E5
:109430006281738189E390E10E9480F261EF71E1C2
:1094400089E390E10F94E423D3011496ED91FC910C
:109450000190F081E02D448155816681778189E317
:1094600090E10E9480F26DEE71E189E390E10F944A
:10947000E423D3011496ED91FC910190F081E02D4D
:10948000408551856285738589E390E10E9480F271
:10949000D3011496ED91FC918689882331F066EE14
:1094A00071E189E390E10F94E42389E390E10F9463
:1094B0007822F301E480F580D70156968C918111D2
:1094C000F7CE0281138161E0F801848195810E94C9
:1094D000ECED2C0120E030E0A901D7011E966D9142
:1094E0007D918D919C9151970F94A35681110CC041
:1094F00020E030E0A901F7016281738184819581C8
:109500000F94AB5918165CF040E050E061E070E059
:10951000C8010E94BFB1672B682B692B31F11986F6
:109520001A861B861C861D861E861F86188A8A85BB
:10953000807F8A8761E0CE0109960E947273298339
:109540003A834B835C836D837E838F839887912CD2
:10955000812CB12CA12CD12CC12C79018A019B0129
:10956000AC016FEFC2010E94603E40E050E061E05C
:1095700070E0D30112968D919C910E946DB1D30140
:109580001496ED91FC913281638154814581198655
:109590001A861B861C868A85807F8760F82E8A87BC
:1095A000232F832F962FA52FB42F8D879E87AF87CC
:1095B000B88B912C812CB12CA12CD12CC12CE984FD
:1095C0000B851C853E854F8558896FEFC2010E942F
:1095D000603ED3011496ED91FC9182819381A48128
:1095E000B58186879787A08BB18BD3011496ED91B7
:1095F000FC91868981115CCE8789908D009709F452
:1096000057CE28EE33E0829F2001839F500C929F1B
:10961000500C11240F947F02D3011496ED91FC910C
:109620004114510499F06201F12CE12C0289138953
:1096300024893589AB01BC01401B510B620B730BB4
:109640004C155D056E057F0508F432CE81E0868BF2
:1096500061E0C3010E94B5412BCE90E080E02ACEAC
:109660002F923F924F925F926F927F928F929F9232
:10967000AF92BF92CF92DF92EF92FF920F931F9320
:10968000CF93DF93CDB7DEB7C258D1090FB6F894A8
:10969000DEBF0FBECDBFFC01A2960FAFA297A3966F
:1096A0001FAFA397A4962FAFA497A5963FAFA597FA
:1096B000A6964FAFA697A7965FAFA797A8966FAF4E
:1096C000A897A9967FAFA99786EF800F823008F4FC
:1096D000F3C4EB96FFAEEEAEEB97AD96FFAFEEAFF9
:1096E000AD97922F222E312C002309F4E8C42114C7
:1096F000310409F4D4C0F3E02F16310409F4EAC4AC
:10970000973009F0F9C4013109F4A1C0023109F41C
:10971000BEC0003109F0F0C46FEF70E0CE018F5988
:109720009F4F0E944C746A962FAF6A976B963FAF1B
:109730006B976C964FAF6C976D965FAF6D976E960B
:109740006FAF6E976F967FAF6F97A0968FAFA09712
:10975000A1969FAFA197D0C46AE471E189E390E13B
:109760000F94E4236CE371E189E390E10F94E42327
:10977000CE018F599F4F0E949F75AB01BC0189E3B9
:1097800090E10E9480F289E390E10F947822AD96F7
:10979000AEADBFADAD9712960D911C9180E00F94C8
:1097A000C542AB01BC01C8010E94C1AFCE018F59B7
:1097B0009F4F0E94E57503E110E06F3171053CF4A5
:1097C0000FE010E06131710514F404E110E0AD9692
:1097D000EEADFFADAD97E280F380C7010E94E0B728
:1097E00080171106E1F481E090E0CE57DF4F0FB60D
:1097F000F894DEBF0FBECDBFDF91CF911F910F91C7
:10980000FF90EF90DF90CF90BF90AF909F908F90A0
:109810007F906F905F904F903F902F900895602FB2
:10982000C7010E94C1B7AD96AEADBFADAD97129660
:109830008D919C910E94F2B961E0892B09F460E05E
:10984000AD968EAD9FADAD970E943AE6CCCF60E865
:1098500070E0CE018F599F4F0E944C7462962FAFDB
:10986000629763963FAF639764964FAF6497659630
:109870005FAF659766966FAF669767967FAF67979E
:1098800068968FAF689769969FAF699735C46AE00D
:1098900070E0CE018F599F4F0E944C752DC4222439
:1098A0002394312C29C423E02216310409F41AC26E
:1098B00037E02316310409F0A4C4A3968FADA39713
:1098C0008F7009F48AC0CE018F599F4F0E94E575B1
:1098D000AB96AEADBFADAB9719960D911D912D9185
:1098E0003C911C97672B682B692B09F4A3C00230AD
:1098F000110521053105B1F56DED76E089E390E1C3
:109900000F94CE2389E390E10F94782221E030E098
:1099100040E050E0AB96AEADBFADAB9719962D933E
:109920003D934D935C931C9761E0CE018F599F4FFF
:109930000E9472732A962FAF2A972B963FAF2B97D0
:109940002C964FAF2C972D965FAF2D972E966FAF1D
:109950002E972F967FAF2F9760968FAF6097619667
:109960009FAF6197CE018F599F4F0E94E575E19699
:10997000EEADFFADE1976187728783879487809111
:109980003A0C90913B0C059741F1D301AD90BC90FE
:10999000C12C40E3D42EE12CF12CA2960FADA2975E
:1099A000A3961FADA397A4962FADA497A5963FAD00
:1099B000A597A6964FADA697A7965FADA797A89631
:1099C0006FADA897A9967FADA997AD96EEADFFAD07
:1099D000AD97828193810E94E3B1A2968FADA29749
:1099E000882309F40EC4A2969FADA297992309F487
:1099F00008C4EFEFE90FE53108F04EC1F0E0882729
:109A0000EB5FF24B8F4F0D9464585E4DF64D4C4E0C
:109A10004C4E4C4E4C4E4C4E4C4E4C4E144E2A4ED0
:109A20004C4E4C4E3A4E3A4E4C4E4C4E4C4E3A4E9C
:109A30003A4E3A4E0130110521053105B1F56EEE71
:109A400076E089E390E10F94CE2389E390E10F94CF
:109A5000782222E030E040E050E0AB96AEADBFAD02
:109A6000AB9719962D933D934D935C931C9762E0B1
:109A7000CE018F599F4F0E94727322962FAF22976B
:109A800023963FAF239724964FAF249725965FAF39
:109A9000259726966FAF269727967FAF279728960C
:109AA0008FAF289729969FAF2997E196EEADFFAD2E
:109AB000E197118612861386148661CFE196AEADCA
:109AC000BFADE19719966D917C91CE018F599F4F53
:109AD0000E944C7429AF3AAF4BAF5CAF6DAF7EAF15
:109AE0008FAF21969FAF219767E0CE018F599F4F8F
:109AF0000E94507329AB3AAB4BAB5CAB6DAB7EAB0A
:109B00008FAB98AFA2968FADA29790E0B0E0A0E0A7
:109B1000AB96EEADFFADAB9781879287A387B487F5
:109B2000C12C30E3D32EE12CF12C80913A0C909192
:109B30003B0C059779F1AB96EEADFFADAB97818508
:109B40009285A385B4850197A105B10519F5E19624
:109B5000EEADFFADE19781859285A385B4854497ED
:109B6000A105B105BCF42EE130E040E050E02187D2
:109B70003287438754876EE170E0CE018F599F4F43
:109B80000E944C74298F3A8F4B8F5C8F6D8F7E8F24
:109B90008F8F98A380913A0C90913B0C059709F414
:109BA00030C3F301A080B180A2960FADA297A39617
:109BB0001FADA397A4962FADA497A5963FADA597EB
:109BC000A6964FADA697A7965FADA797A8966FAD3F
:109BD000A897A9967FADA997AD96AEADBFADAD974D
:109BE00012968D919C910E94E3B10BC370E060E0EE
:109BF000CE018F599F4F0E944C7429A73AA74BA7BB
:109C00005CA76DA77EA78FA798AB67E0CE018F59A1
:109C10009F4F0E94507329A33AA34BA35CA36DA34B
:109C20007EA38FA398A76ECF8114910469F0F401ED
:109C300081859285A385B4850097A105B10521F0A2
:109C400061E070E00F943127C12C90E4D92EE12C13
:109C5000F12C6BCF81149104B9F3F40181859285C5
:109C6000A385B4850097A105B10571F3DC01DA96EF
:109C70001C92EACF892F90E0B0E0A0E0AB96EEAD69
:109C8000FFADAB9781879287A387B487C12C20E172
:109C9000D22EE12CF12C49CFC12CD12C760145CF0D
:109CA000A3968FADA3978F7009F4ABC2CE018F59E5
:109CB0009F4F0E949F759B01AC0167E176E0C30155
:109CC0000E941D2780913A0C90913B0C059709F456
:109CD00098C2F301A080B180C12C80E2D82EE12C83
:109CE000F12C62CFA3968FADA3978F7009F47BCD33
:109CF000CE018F599F4F0E949F759B01AC016AE373
:109D000076E0C3010E941D276ECDE9961FAE1EAE00
:109D1000E997E3961FAE1EAEE397512C412CE796D0
:109D20001FAE1EAEE7974114510409F4C5C1E79672
:109D30008EAD9FADE797B2010F9450583B016DE295
:109D400071E189E390E10F94E4234AE050E0B2012D
:109D500089E390E10F94852362E271E189E390E168
:109D60000F94E4230FEF10E0E7968EAD9FADE797D9
:109D7000B8010F9450584AE050E089E390E10F9405
:109D800085236BE171E189E390E10F94E4234AE0DC
:109D900050E0B30189E390E10F94852361E171E123
:109DA00089E390E10F94E423E9968EAD9FADE997A6
:109DB000B8010F9450584AE050E089E390E10F94C5
:109DC00085236AE071E189E390E10F94E4234AE09E
:109DD00050E0E3966EAD7FADE39789E390E10F9499
:109DE000852366E071E189E390E10F94E42389E340
:109DF00090E10F94782219821A821B821C821D82A4
:109E00001E821F8218868A81807F8A83B301CE01D9
:109E100001960E944C7429873A874B875C876D872F
:109E20007E878F87988B67E0CE0109960E945073DA
:109E300079018A011B012C01298BFA8A4B8B1C8B1F
:109E40006D8B3E8A8F8B588E65E37AE0AD96EEADD2
:109E5000FFADAD97848195810E943AED912C812CC4
:109E6000B12CA12CD12CC12C9101A2016FEF0E9429
:109E7000603E672809F4B7CCAD96AEADBFADAD97E7
:109E80001496ED91FC91309709F4ADCC6680778003
:109E9000E3962EAD3FADE397032E000C440B550B1C
:109EA000E5962CAF3DAF4EAF5FAFE597E9968EAD2F
:109EB0009FADE997092E000CAA0BBB0BAF968CAF98
:109EC0009DAFAEAFBFAFAF976114710409F48BCCF7
:109ED000C3010E94CCFD6B0161E376E0C3010E94E7
:109EE0003AEDAB969FAF8EAFAB9761E276E0C301E0
:109EF0000E943AED8C016CE176E0C3010E943AEDDC
:109F0000AB96AEADBFADAB97109709F4CDC00115C0
:109F1000110509F4C9C0009709F4C6C018962C9120
:109F20002F70223009F0C0C0F80120852F70223038
:109F300009F0BAC0DC0118962C9118972F702230C6
:109F400009F0B2C0C114D10409F4AEC019968D91C4
:109F50009D910D90BC91A02D82309105A105B10578
:109F600009F4A6C08F3F9F4FAF4FBF4F09F4A0C069
:109F7000E9962EAD3FADE997232B09F499C0D8019E
:109F800019968D919C918C9D80018D9D100D9C9DAD
:109F9000100D11242FEF30E0D8010F947B5896015B
:109FA000DD0C440B550B0F940F58E5966CAD7DAD51
:109FB0008EAD9FADE5970F94DD57AF962CAD3DADBF
:109FC0004EAD5FADAF970F940F5819012A016FEF97
:109FD00070E189E390E10F94E423F30160817181E2
:109FE00089E390E10F94CE2369EF70E189E390E17A
:109FF0000F94E423C8016FEF70E00F9450584AE0CB
:10A0000050E089E390E10F94852363EF70E189E3E9
:10A0100090E10F94E4232AE030E0B201A10189E34A
:10A0200090E10F943D2389E390E10F947822AB9661
:10A03000EEADFFADAB9781859285A385B485821582
:10A040009305A405B50581F119861A861B861C8621
:10A050001D861E861F86188A8A85807F8A87B101A1
:10A06000CE0109960E944C7429833A834B835C830A
:10A070006D837E838F839887912C812CB12CA12CAA
:10A08000D12CC12C79018A019B01AC016FEFC30176
:10A090000E94603EAB96AEADBFADAB9719962D92C8
:10A0A0003D924D925C921C97F301628073800CCFBD
:10A0B000212C312C2101BBCF90E080E096CB23E016
:10A0C00022163104C9F4EB96AEADBFADEB97AB2BC6
:10A0D00099F407C0EB964EAD5FADEB97452B09F0B9
:10A0E0000FCBA3968FADA3978F7009F035CB63E0AC
:10A0F000262E312C011104CBAD96AEADBFADAD9780
:10A100001496ED91FC91309709F4FFCD668077802D
:10A11000C158DF4F19821882CF57D040E9961FAE41
:10A120001EAEE997E3961FAE1EAEE397512C412C6D
:10A13000E7961FAE1EAEE7976114710409F4F3CDE4
:10A1400061E276E0C3010E943AEDE1969FAF8EAFE7
:10A15000E1976CE176E0C3010E943AEDAB969FAFC8
:10A160008EAFAB9769ED76E0C3010E943AEDCF5711
:10A17000DF4F99838883C158D04065E775E0C301FC
:10A180000E943AED4C01E196EEADFFADE1973097BC
:10A1900009F4B8C0AB962EAD3FADAB972115310594
:10A1A00009F4B0C080858F70823009F0ABC0D9014E
:10A1B00018968C918F70823009F0A4C0C3010E9460
:10A1C000CCFDEF966CAF7DAF8EAF9FAFEF97EB9668
:10A1D000EEADFFADEB973097F1F1BF01D3018D915B
:10A1E0009C910F94D15C892BB1F5B2E02B16310410
:10A1F00009F456CD0CF057CBF1E02F16310409F4D9
:10A20000F2CBCF57DF4FE881F981C158D04030976A
:10A2100011F1912C812CB12CA12CD12CC12CA29606
:10A22000EFACA297A396FFACA397A4960FADA4970B
:10A23000A5961FADA597A6962FADA697A7963FAD5D
:10A24000A797A8964FADA897A9965FADA9976FEF6E
:10A25000CF010E94603EAB96EEADFFADAB9781851E
:10A260009285A385B48582309105A105B10509F4D5
:10A2700043C08F3F9F4FAF4FBF4FF1F1E196EEAD1F
:10A28000FFADE19781859285A385B485ED964EADAE
:10A290005FADED97849F9001859F300D949F300DA9
:10A2A0001124E796EEADFFADE797E20FF31FE796B7
:10A2B000FFAFEEAFE797C158DF4FE881F981CF5785
:10A2C000D040AF01FF0F660B770B481759076A079D
:10A2D0007B0794F4C158DF4F99838883CF57D040D0
:10A2E000E9963FAF2EAFE997ED962EAD3FADED97D6
:10A2F000E3963FAF2EAFE397ED964EAD5FADED9792
:10A30000440E551ED30112966D907C9015CF2F925E
:10A310003F924F925F926F927F928F929F92AF92F5
:10A32000BF92CF92DF92EF92FF920F931F93CF9342
:10A33000DF93CDB7DEB7CF58D1090FB6F894DEBFA3
:10A340000FBECDBF3C011A01CD57DF4F2883C35844
:10A35000D040C457DF4F19830883CC58D040C25730
:10A36000DF4FF982E882CE58D040C957DF4FC8820C
:10A37000C758D040CB57DF4FB982A882C558D040CC
:10A38000DC011496ED91FC910288F389E02D868022
:10A390009780AB2849F4FE01EE57FF4FCB57DF4FB4
:10A3A000F983E883C558D04081E0CB57DF4FA881BF
:10A3B000B981C558D0408C936B01F12CE12C8114EC
:10A3C000910409F4F6C5CD57DF4FB881C358D0408A
:10A3D000B13009F488C008F47FC0B23041F0B33026
:10A3E00009F477C0D40112968D909C90E8CF60EA72
:10A3F00076E0C4010E943AED11E0009799F3FC0168
:10A4000081859285A385B4858C159D05AE05BF0514
:10A4100049F766E775E0C4010E943AEDC857DF4F7F
:10A4200099838883C858D040D3011296ED91FC914E
:10A4300062E0848195810E94ECEDC657DF4F9983DD
:10A440008883CA58D040822D0E949CFA7C01CF5745
:10A45000DF4F1882C158D04019AA1AAA1BAA1CAAF9
:10A460001DAA1EAA1FAA18AE8AA9807F8AAB62EE17
:10A4700075E0C4010E943AED6C0167EE75E0C4011D
:10A480000E943AED5C01C114D10451F0F6018085BF
:10A490008F70843029F4818592850E949921182F2C
:10A4A000EFEFE10FEB3008F09DC10E2E000CFF0B1B
:10A4B0008827E25AFD4A8F4F0D9464587652045310
:10A4C000E2522953F253F25371534E539553A6530C
:10A4D000BE5360E077E08DCF63E077E0C4010E9477
:10A4E0003AED1BE08ACF68E077E0F8CF1701512CF6
:10A4F000412CA701FF0C660B770BCE01C1960E9481
:10A500009473EA962FAFEA97EB963FAFEB97EC96F2
:10A510004FAFEC97ED965FAFED97EE966FAFEE977E
:10A52000EF967FAFEF97C158DF4F8883CF57D0406A
:10A53000C058DF4F9883C058D04080914502893081
:10A5400020F4809144028930B8F167E77EE089E326
:10A5500090E10F94E42300E020E030E340E150E09C
:10A56000BE016F5F7F4FCE01C1960E949576BC0100
:10A5700089E390E10F94CE236BE67EE089E390E1DE
:10A580000F94E423612F110F770B4AE050E089E329
:10A5900090E10F94852369E67EE089E390E10F94D2
:10A5A000E423D4016D917C9189E390E10F94CE2353
:10A5B00089E390E10F947822A114B10409F016C147
:10A5C000D12C71C31701512C412CB201A701CE012E
:10A5D000C1960E949473E2962FAFE297E3963FAF45
:10A5E000E397E4964FAFE497E5965FAFE597E6967D
:10A5F0006FAFE697E7967FAFE797E8968FAFE8975C
:10A60000E9969FAFE99799CFFE24EF24FE24170126
:10A61000512C412CB201A101CE01C1960E9494732C
:10A62000AA962FAFAA97AB963FAFAB97AC964FAF1A
:10A63000AC97AD965FAFAD97AE966FAFAE97AF9656
:10A640007FAFAF97E0968FAFE097E1969FAFE1972E
:10A6500074CFFE24EF24FE241701512C412CB201AB
:10A66000A101CE01C1960E949473A2962FAFA2972A
:10A67000A3963FAFA397A4964FAFA497A5965FAFBD
:10A68000A597A6966FAFA697A7967FAFA797A89610
:10A690008FAFA897A9969FAFA9974FCFFF24170117
:10A6A000512C412CB201A701CE01C1960E94947396
:10A6B0006A962FAF6A976B963FAF6B976C964FAFCA
:10A6C0006C976D965FAF6D976E966FAF6E976F9646
:10A6D0007FAF6F97A0968FAFA097A1969FAFA197DE
:10A6E0002CCFEF2CFF241701512C412CB201A701D4
:10A6F000CE01C1960E94947362962FAF62976396C3
:10A700003FAF639764964FAF649765965FAF659769
:10A7100066966FAF669767967FAF679768968FAFBD
:10A72000689769969FAF699708CF1701512C412C04
:10A730008AA9807F86608AAB2AE030E0D7010F9437
:10A740007B586DAB7EAB8FAB98AFF7CE1701512C1A
:10A75000412C8AA9807F87608AABB701FF0C880BE8
:10A76000990B0F94AA5620E030E048EC52E40F9485
:10A7700003596DAB7EAB8FAB98AFDFCEC10124E048
:10A78000969587952A95E1F70E949CFAFFE02F2283
:10A79000332402C0969587952A94E2F78170992711
:10A7A0001C01512C412CB201AC01CE01C1960E947A
:10A7B00094732A962FAF2A972B963FAF2B972C9600
:10A7C0004FAF2C972D965FAF2D972E966FAF2E978C
:10A7D0002F967FAF2F9760968FAF609761969FAF50
:10A7E0006197ABCE212C312C2101A7CEF5018085BC
:10A7F0008F708550823008F0E3CEB501CE01C1964E
:10A800000E94D27929A33AA34BA35CA36DA37EA394
:10A810008FA398A788E0FE01B196DE01999601907A
:10A820000D928A95E1F788E0FE01B996DE01D19696
:10A8300001900D928A95E1F789A9811103C08AA937
:10A840008F7009F180914502893008F4B9C264EE35
:10A850007DE089E390E10F94E42300E020E030E321
:10A8600040E150E0BE016F5F7F4FCE01C1960E9474
:10A870009576BC0189E390E10F94CE2389E390E1C2
:10A880000F9478229DCE6CE976E0C5010E943AEDE6
:10A890007C01009709F494CEDC0118968C918F709E
:10A8A000823009F41DC1843009F08ACE80914502BE
:10A8B000893020F480914402893090F06AE17EE092
:10A8C00089E390E10F94E423D70119966D917C916F
:10A8D00089E390E10F94CE2389E390E10F947822ED
:10A8E000C657DF4FE881F981CA58D040309709F444
:10A8F00071C380858F70863009F06AC3D7011996BD
:10A90000CD90DC90C114D10409F462C3D301129636
:10A91000ED91FC9162E0848195810E94ECEDB6019D
:10A920000E943AED0E948DFD6C01892B09F450C301
:10A9300080914502893020F4809144028930A8F04A
:10A9400068E07EE089E390E10F94E423F60141851D
:10A950005285638574852AE030E089E390E10F94A5
:10A960003D2389E390E10F947822D70119966D91E8
:10A970007C91D3011496ED91FC91828993890E9478
:10A980003AED7C01009709F423C362EE75E00E9462
:10A990003AED009749F0FC0120852F70243021F416
:10A9A000818592850E949921D60119964D915D91DC
:10A9B0006D917C911C97CE01C1960E949473229652
:10A9C0002FAF229723963FAF239724964FAF24971C
:10A9D00025965FAF259726966FAF269727967FAF70
:10A9E000279728968FAF289729969FAF299767EECC
:10A9F00075E0C7010E943AEDBC01009721F1FC010E
:10AA000090859F7095509230F0F4CE01C1960E94CF
:10AA1000D279298B3A8B4B8B5C8B6D8B7E8B8F8B9A
:10AA2000988F88E0FE017196DE01599601900D9293
:10AA30008A95E1F788E0FE017996DE01D1960190D2
:10AA40000D928A95E1F780914502893020F480913A
:10AA500044028930D8F063EF7DE089E390E10F9400
:10AA6000E42300E020E030E340E150E0BE016F5F0E
:10AA70007F4FCE01C1960E949576BC0189E390E19B
:10AA80000F94CE2389E390E10F947822D601189693
:10AA90008C911897982F92959F7090FD99C221E004
:10AAA000CF57DF4F2883C158D04091609295907F57
:10AAB0008F70892B18968C93DD24D394C957DF4F60
:10AAC000B881C758D040BB2309F406C1C857DF4F2F
:10AAD00048815981C858D040452B09F4FDC08CC22B
:10AAE00080914502893020F4809144028930A8F099
:10AAF00063E57EE089E390E10F94E423F70141856B
:10AB00005285638574852AE030E089E390E10F94F3
:10AB10003D2389E390E10F947822D70119966D9136
:10AB20007D918D919C911C97C457DF4FE881F981ED
:10AB3000CC58D0408F0130E020E0601771078207C9
:10AB400093070CF455C0C257DF4F48815981CE5846
:10AB5000D0408A0130E020E00617170728073907A0
:10AB60000CF446C0AB014E1B5F0BDE01AF57BF4F6D
:10AB70005D01C12CC257DF4FE880F980CE58D0402C
:10AB80008F01CD57DF4F2881C358D040C3010E94A9
:10AB9000875129AB3AAB4BAB5CAB6DAB7EAB8FABAC
:10ABA00098AF80914502893020F480914402893029
:10ABB000E0F06CE077E089E390E10F94CE2369E266
:10ABC00077E089E390E10F94CE23CF57DF4F688180
:10ABD000C158D04070E04AE050E089E390E10F9422
:10ABE000852389E390E10F947822DD24D3945BC020
:10ABF00069E47EE089E390E10F94E423F701418565
:10AC00005285638574852AE030E089E390E10F94F2
:10AC10003D236AE27EE089E390E10F94E42389E337
:10AC200090E10F94782281E08093DB0DCE01419674
:10AC30009093610E8093600ECD57DF4FF881C3581B
:10AC4000D0406F2F70E041E050E0D70119968D9110
:10AC50009C910E946A2ED82E8823E1F0F70161852D
:10AC600072859E012F573F4F5901C12C7B018B01EB
:10AC7000CD57DF4F2881C358D04050E040E0C3019A
:10AC80000E94875129AB3AAB4BAB5CAB6DAB7EAB53
:10AC90008FAB98AF80E48093DB0D80EE9DE09093C6
:10ACA000610E8093600EC957DF4FB881C758D040FE
:10ACB000BB2349F0C857DF4FE881F981C858D0401D
:10ACC000EF2B09F099C1C657DF4FE881F981CA58C7
:10ACD000D040EF2B09F447C0C657DF4FA881B98198
:10ACE000CA58D04018968C9118978F708630D9F535
:10ACF000F40160817181CD010E943AED3C01009721
:10AD000091F10E948DFD7C01009709F4D6C0FC01F1
:10AD100081859285A385B48582159305A405B50523
:10AD200009F09CC0C957DF4FF881C758D040F111D6
:10AD300057C0D70118968C91189782958F7080FD17
:10AD40004FC091E0CB57DF4FE881F981C558D04023
:10AD5000908381608295807F18969C9118979F7050
:10AD6000892B18968C9388E0FE01F196DE01D99626
:10AD700001900D928A95E1F729AD3AAD4BAD5CADEE
:10AD80006DAD7EAD8FAD21969FAD2197C157DF4F41
:10AD90000FB6F894DEBF0FBECDBFDF91CF911F91EC
:10ADA0000F91FF90EF90DF90CF90BF90AF909F906A
:10ADB0008F907F906F905F904F903F902F9008956D
:10ADC00080914402893008F4FBCB41CDF3016281CC
:10ADD000738140E050E1CE01C1960E94AA7273CF08
:10ADE000CB57DF4FA881B981C558D0401C92DD20D8
:10ADF00009F4B9CFC957DF4FB881C758D040BB233A
:10AE000009F4B1CFCF57DF4F8881C158D0408111AD
:10AE10000AC0CB57DF4FA881B981C558D0408C916B
:10AE2000882309F4A0CF912C812CB12CA12CD12CFA
:10AE3000C12CE9A8FAA80BA91CA92DA93EA94FA9C4
:10AE400058AD6FEFC3010E94603E81E0CB57DF4FEA
:10AE5000E881F981C558D040808385CF218632862C
:10AE60004386548680914502893020F480914402C3
:10AE70008930F8F06EE277E089E390E10F94CE2319
:10AE80002AE030E0B201A10189E390E10F9493221E
:10AE90006CE377E089E390E10F94CE23D4016D91C8
:10AEA0007C9189E390E10F94CE2389E390E10F94A4
:10AEB0007822F70180858F7E8087D1109BCFCB577A
:10AEC000DF4FA881B981C558D0408C91882309F4FF
:10AED0004ACFC957DF4FB881C758D040BB2309F4C8
:10AEE00042CFF30180858F708530D1F586819781BF
:10AEF0006BEE75E00E943AEDCD57DF4F9983888362
:10AF0000C358D040009771F1DC0118968C911897C6
:10AF10008F70823039F519968D919D910D90BC916D
:10AF2000A02D82159305A405B505E1F48091450295
:10AF3000893020F480914402893050F06DEB7DE03F
:10AF400089E390E10F94E42389E390E10F94782260
:10AF5000CB57DF4FE881F981C558D040108203CF2D
:10AF6000C301C6CF912C812CB12CA12CD12CC12C8A
:10AF7000E9A8FAA80BA91CA92DA93EA94FA958AD6B
:10AF80006FEFC3010E94603ECD57DF4F28813981AA
:10AF9000C358D0402115310509F4E5CED3011896E8
:10AFA0008C9187FDE0CEF901218632864386548656
:10AFB000DACE19821A821B821C828A81807F8A8360
:10AFC0001D821E821F82188688E0FE013196CECE39
:10AFD000D12C74CDC957DF4FE881C758D040EE233C
:10AFE00009F4C1CEC857DF4F28813981C858D040F5
:10AFF000D12C232B09F4B7CEC857DF4FA881B981D4
:10B00000C858D04018968C9118978F70823009F0EC
:10B010005ACE19968D919D910D90BC91A02D8130A5
:10B020009105A105B10509F4D1CE0297A105B1059D
:10B0300009F049CED30112966D917C9140E050E227
:10B04000CACE2F923F924F925F926F927F928F92D1
:10B050009F92AF92BF92CF92DF92EF92FF920F93A7
:10B060001F93CF93DF93CDB7DEB768970FB6F894F1
:10B07000DEBF0FBECDBF6115710509F491C05E8BB7
:10B08000498B9D8B8C8BFB0186809780811491046A
:10B0900009F486C0F40180858F70823031F08530EC
:10B0A00031F1F40182809380F1CF6184728441E0B8
:10B0B00050E069897E89C3010E946A2E882389F342
:10B0C000B12CA12CCC24C39473018301298950E0B5
:10B0D00040E0B3018C899D890E94875129873A8776
:10B0E0004B875C876D877E878F87988BDACFC4010B
:10B0F0000E947DEE8230A9F660E0C4010E94ECED72
:10B10000FC01C184D284E384F48461E0C4010E9420
:10B11000ECEDFC012184328443845484388E2F8AE0
:10B12000DB8ACA8AA1014C195D094F5F5F4F6989AB
:10B130007E89C6010E946A2E882309F4B2CF8091CD
:10B140004502893020F480914402893020F089E35F
:10B1500090E10F947822712C612C6A897B89660DAD
:10B16000771D8F89988D861797070CF49ACFB12C8D
:10B17000A12CCC24C39471010A891B892989A301BC
:10B180008C899D890E94875129833A834B835C83F4
:10B190006D837E838F8398879FEF691A790ADDCF4D
:10B1A00068960FB6F894DEBF0FBECDBFDF91CF918A
:10B1B0001F910F91FF90EF90DF90CF90BF90AF90D5
:10B1C0009F908F907F906F905F904F903F902F90C7
:10B1D00008952F923F924F925F926F927F928F923B
:10B1E0009F92AF92BF92CF92DF92EF92FF920F9316
:10B1F0001F93CF93DF9300D01F921F92CDB7DEB77E
:10B2000061307105D1F490E080E00F900F900F90C5
:10B210000F900F90DF91CF911F910F91FF90EF90C2
:10B22000DF90CF90BF90AF909F908F907F906F9066
:10B230005F904F903F902F90089520918B0A30910E
:10B240008C0A232B01F78C01DC01ED91FC91028427
:10B25000F385E02D19950297B1F68091960A9091A9
:10B26000970AA091980AB091990A892B8A2B8B2B67
:10B2700079F4D8011296ED91FC9162E08481958178
:10B280000E94ECED9C838B83892BB1F4B12C05C417
:10B290000F947F02C090960AD090970AE090980A87
:10B2A000F090990A6C197D098E099F09683C710517
:10B2B00081059105F0F6A7CFEB81FC8180858F7029
:10B2C000863021F7C680D7801D82B12CC114D104ED
:10B2D00009F4DFC3D60118968C91982F9F702BEF3D
:10B2E000290F223008F0D5C3BD81B111D2C3282F58
:10B2F00022952F7087FF71C522FD6FC5953009F02B
:10B30000A7C0F601868197816BEE75E00E943AED49
:10B310001C01892B09F461C581E090E090938C0AAF
:10B3200080938B0AB11003C0C8010E94E72ED1019F
:10B3300019964D905C9067E477E089E390E10F9473
:10B34000CE23D8011296ED91FC910280F381E02D7D
:10B350006081718189E390E10F94CE2362E179E00D
:10B3600089E390E10F94CE23F6016081718189E336
:10B3700090E10F94CE2366E576E089E390E10F94A7
:10B38000CE23D10119964D915D916D917C911C97C1
:10B390002AE030E089E390E10F943D2389E390E1D6
:10B3A0000F947822F60180809180D8011496ED9157
:10B3B000FC916CE57FE0309759F0B4018289938964
:10B3C0000E943AED7C01009709F044C069E37FE0F8
:10B3D00082E99FE00F94E42382E99FE00F947822B2
:10B3E000EE24EA94FE2C4201550CAA08BB08D101B8
:10B3F00019964D905D906D907C901C9784149504E7
:10B40000A604B70409F49EC48091960A9091970A05
:10B41000A091980AB091990A892B8A2B8B2B09F459
:10B4200086CF0F947F022091960A3091970A40911F
:10B43000980A5091990A621B730B840B950B683C18
:10B4400071058105910508F072CF0E94E9A3D6CF5E
:10B45000C6015ACF60EA76E00E943AED3C01892BA2
:10B4600079F463E077E0C7010E943AED3C0166E1C0
:10B470007FE0892B69F0F10180858F70806B808778
:10B48000D30118968C918F70823079F060E07FE064
:10B4900082E99FE00F94E42382E99FE00F947822F1
:10B4A000EEEFEE2EFF24FA949ECF63E976E0C7011B
:10B4B0000E943AED7C01009709F43FC1FC018085B0
:10B4C0008F70813009F05EC18185882309F45AC1EB
:10B4D000D10118968C91807FF12CE12C803B19F0E2
:10B4E00072E0E72EF12C65EF7EE089E390E10F94A6
:10B4F000E423B40189E390E10F94CE2362EF7EE070
:10B5000089E390E10F94E423F3014185528563853B
:10B5100074852AE030E089E390E10F943D2363E5F0
:10B5200077E089E390E10F94CE234AE050E0B70141
:10B5300089E390E10F9485236FEF75E089E390E153
:10B540000F94CE23F1E0F093DB0D81E090E08C0FBF
:10B550009D1F9093610E8093600E41E050E0B70113
:10B56000D30119968D919C910E946A2EF82E80E04D
:10B570000F94C5426093960A7093970A8093980A35
:10B580009093990AFF2009F4FAC0D8011296ED9120
:10B59000FC9162E0848195810E94ECED7C01009732
:10B5A00009F4C2C0FC0180858F70863009F0E7C0C5
:10B5B000B401C7010E943AED7C01009709F4B4C0C0
:10B5C0000E948DFD7C01892B09F4AEC0809145025B
:10B5D000893020F480914402893028F16BEE7EE0BE
:10B5E00089E390E10F94E423D70119964D915D9181
:10B5F0006D917C911C972AE030E089E390E10F94F3
:10B600003D2365EE7EE089E390E10F94E4236981B8
:10B610007A814AE050E089E390E10F94952289E332
:10B6200090E10F947822F7014185528563857485F6
:10B6300089819A81B0E0A0E0481759076A077B0723
:10B6400019F16FED7EE089E390E10F94E423B401FA
:10B6500089E390E10F94CE2361ED7EE089E390E1F0
:10B660000F94E42389E390E10F947822F0E4F093BF
:10B67000DB0D80EE9DE09093610E8093600E6DEF88
:10B68000E62EFF24FA94AFCEF10181859285A38541
:10B69000B485481759076A077B0789F56BEC7EE08C
:10B6A00089E390E10F94E423B40189E390E10F94DE
:10B6B000CE2369EC7EE089E390E10F94E423698175
:10B6C0007A814AE050E089E390E10F94952268EB9B
:10B6D0007EE089E390E10F94E42389E390E10F9405
:10B6E0007822F0E4F093DB0D80EE9DE09093610E04
:10B6F0008093600E5CEFE52EFF24FA9474CE62EB2B
:10B700007EE089E390E10F94E423B40189E390E1C2
:10B710000F94CE2367E97EE089E390E10F94E42360
:10B7200089E390E10F94782290E49093DB0DA0EEF2
:10B73000BDE0B093610EA093600ED1011896EC911C
:10B74000E295EF70E150AA24AA94BA2CEB3008F0ED
:10B7500066C0F0E0D30119962D913C918827EC54F6
:10B76000F44A8F4F0D946458C55BDA5BC55BDA5BB6
:10B77000815C7C5C815C7C5CC55BC55B8D5CF12C19
:10B78000E12CD2CFF12CE12CD8CFF101818592852B
:10B790003093630E2093620E1092650E1092640E29
:10B7A0009093670E8093660E86E00F940A04A82E8D
:10B7B000B12C35C0D10119968D919C91982789277C
:10B7C00098273093630E2093620E1092650E1092AC
:10B7D000640E9093670E8093660E86E00F940A04C1
:10B7E000A82EB12CF10181859285A385B4853A2FCD
:10B7F0002B2FD30119968D919C9101969093630EF6
:10B800008093620E1092650E1092640E3093670E54
:10B810002093660E86E00F940A04A80EB11C80E007
:10B820000F94C5426093960A7093970A8093980A82
:10B830009093990A6CE87EE089E390E10F94E42309
:10B840004AE050E0B50189E390E10F9485236AE86E
:10B850007EE089E390E10F94E423B40189E390E171
:10B860000F94CE236AE577E089E390E10F94CE232D
:10B87000F30141855285638574852AE030E089E3D0
:10B8800090E10F943D2364E87EE089E390E10F941A
:10B89000E423D10119964D915D916D917C911C9796
:10B8A0002AE030E089E390E10F943D2389E390E1C1
:10B8B0000F947822A114B104B9F4F10180858F703E
:10B8C000823091F4E114F10479F0D70118968C914B
:10B8D0008F70823049F481859285A385B485F70104
:10B8E00081879287A387B48791E080E0AB2809F035
:10B8F00090E0E92EF82E77CDF10181859285992788
:10B9000047CFF10181859285A385B485892F9A2F30
:10B91000AB2FBB27A7FDBA95F2CFD10119968C9119
:10B920003093630E2093620E882341F080E09FEFF6
:10B930009093650E8093640E85E037CF90E080E0B1
:10B94000F7CFD60118968C911897806418968C932F
:10B9500069EE7FE082E99FE00F94E423D80112961C
:10B96000ED91FC910280F381E02D6081718182E98B
:10B970009FE00F94CE2362E179E082E99FE00F948B
:10B98000CE23F6016081718182E99FE00F94CE237E
:10B990006BED7FE082E99FE00F94E423D6011896D7
:10B9A0008C911897982F92959F70292F2370233090
:10B9B00039F09F5F9295907F8F70892B18968C93AA
:10B9C00063ED7FE082E99FE00F94E423D8011296B3
:10B9D000ED91FC910280F381E02D6081718182E91B
:10B9E0009FE00F94CE2362E179E082E99FE00F941B
:10B9F000CE23F6016081718182E99FE00F94CE230E
:10BA000060E677E082E99FE00F94CE23D601189696
:10BA10006C916295637070E04AE050E082E99FE0CB
:10BA20000F94852382E99FE00F947822D4C165ECBE
:10BA30007FE082E99FE00F94E423D8011296ED9114
:10BA4000FC910280F381E02D6081718182E99FE0A9
:10BA50000F94CE2362E179E082E99FE00F94CE2338
:10BA6000F6016081718182E99FE00F94CE2362EB41
:10BA70007FE082E99FE00F94E42382E99FE00F9446
:10BA80007822D60118968C9118978F7018968C93FF
:10BA9000A2C110928C0A10928B0AD8011496ED91D3
:10BAA000FC91C480D580F12CE12C0F947F02C1144D
:10BAB000D104E104F10491F0D8011496ED91FC91C8
:10BAC00046805780608471846419750986099709D6
:10BAD0006C157D058E059F0508F4C3C08091960AFC
:10BAE0009091970AA091980AB091990A892B8A2B74
:10BAF0008B2B09F0A2C0EB81FC81EF2B09F0B8C0C1
:10BB0000D8011496ED91FC9182859385892B69F477
:10BB100084859585892B49F486859785892B29F419
:10BB200080899189892B09F4FFC080914502893071
:10BB300020F4809144028930B8F06CE87FE089E31A
:10BB400090E10F94E423D8011296ED91FC910280CC
:10BB5000F381E02D6081718189E390E10F94CE2320
:10BB600089E390E10F94782281E090E090938C0A31
:10BB700080938B0AB11003C0C8010E94E72ED80140
:10BB80001496ED91FC916285738542E050E0C80106
:10BB90000E942158D8011496ED91FC916485758519
:10BBA00043E050E0C8010E942158D8011496ED915D
:10BBB000FC916685778550E040E0C8010E942158DD
:10BBC000D8011496ED91FC916089718941E050E0B3
:10BBD000C8010E94215880914502893020F480914B
:10BBE00044028930B8F06CE77FE089E390E10F947C
:10BBF000E423D8011296ED91FC910280F381E02DAF
:10BC00006081718189E390E10F94CE2389E390E113
:10BC10000F9478220F947F026B017C010F947F02B6
:10BC20006C197D098E099F096233710581059105A3
:10BC300008F076C00E94E9A3F1CF0F947F02C09074
:10BC4000960AD090970AE090980AF090990A6C1999
:10BC50007D098E099F09683C71058105910508F0F1
:10BC60004ACFD8011496ED91FC9184819581CDCA7B
:10BC7000AB81BC8118968C9118978F70863009F033
:10BC80003FCF1696ED90FC90E114F10409F438CF03
:10BC9000F7018085982F9F702BEF290F223008F035
:10BCA0002FCF82958F7082FF05C08B708295807F29
:10BCB000892B8087D70118968C9182958370833069
:10BCC00059F56BE677E082E99FE00F94CE23D80127
:10BCD0001296ED91FC910280F381E02D60817181DB
:10BCE00082E99FE00F94CE2362E179E082E99FE050
:10BCF0000F94CE23F7016081718182E99FE00F9458
:10BD0000CE2382E99FE00F947822D70118968C9178
:10BD100018978F7018968C93F701E280F380B4CF58
:10BD200010928C0A10928B0AF801E480F58080E072
:10BD30000F94C542D70116966D937D938D939C9376
:10BD400019978FCFBDEFEB16BFEFFB0609F46FCE4F
:10BD5000ACF5FCEFEF16FFEFFF06B9F164EA7FE008
:10BD600082E99FE00F94E423D8011296ED91FC91B3
:10BD70000280F381E02D6081718182E99FE00F9460
:10BD8000CE2362E179E082E99FE00F94CE23F601B1
:10BD90006081718182E99FE00F94CE2369E97FE0A1
:10BDA00082E99FE00F94E42382E99FE00F947822D8
:10BDB000D60118968C9118978F7768CEE114F1040C
:10BDC00009F4BFCDEA94EF2849F6F60180858F701B
:10BDD0008087F1E0FD83BB24B394F601C280D38059
:10BDE00075CA8F929F92AF92BF92CF92DF92EF92DD
:10BDF000FF920F931F93CF93DF9300D000D01F9239
:10BE00001F92CDB7DEB7E982FA820B831C832D83A4
:10BE10003E834F835887DC011296ED91FC91309759
:10BE200091F1048115810115110569F1F8018085F1
:10BE30008F70853041F57B01C8010E947DEE823014
:10BE400010F161E0C8010E94ECED0097E1F0DC0127
:10BE500018962C912F702630B1F4B7010E943AED5C
:10BE6000009789F0912C812CB12CA12CD12CC12CC4
:10BE7000E980FA800B811C812D813E814F8158859C
:10BE80006FEF0E94603E28960FB6F894DEBF0FBE9B
:10BE9000CDBFDF91CF911F910F91FF90EF90DF9079
:10BEA000CF90BF90AF909F908F9008953F924F9208
:10BEB0005F926F927F928F929F92AF92BF92CF923A
:10BEC000DF92EF92FF920F931F93CF93DF93CDB743
:10BED000DEB7C258D1090FB6F894DEBF0FBECDBF92
:10BEE000DC0114962D913C911597232B09F403C581
:10BEF0008B016C01ED91FC910284F385E02D199585
:10BF00008230910509F404C1C4F597FFF4C4F60129
:10BF100087819085DC01ED91FC910084F185E02D15
:10BF2000199585970CF4E0C0F6016481758145E2AE
:10BF300050E0878190850F94FA21D60117968D9154
:10BF40009C91DC01ED91FC910084F185E02D199527
:10BF50008C01892B09F423C162E070E080E090E05D
:10BF60000F948D00F60187819085DC01ED91FC91A5
:10BF70000284F385E02D1995E0CF8430910509F412
:10BF800063C054F1059719F60130110509F0ECC0B2
:10BF90006DE97AE089E390E10F9408244DE050E0E8
:10BFA00060E072E0C6010E94BC21F60104811581A7
:10BFB00080E00F94C542D80198966D937D938D9340
:10BFC0009C939B97D601ED91FC910484F585E02D1F
:10BFD00062E0C60119959BCFD6011496ED91FC91B4
:10BFE00080A591A5A2A5B3A5892B8A2B8B2B09F43B
:10BFF0008ECF0F947F02D6011496ED91FC91159788
:10C0000000A511A522A533A5601B710B820B930B14
:10C01000663971058105910508F479CFED91FC91A0
:10C020000484F585E02D62E0C6011995F6010481CE
:10C03000158180E00F94C542D80198966D937D9349
:10C040008D939C939B9763CFD6011496ED91FC91B1
:10C0500080A591A5A2A5B3A5892B8A2B8B2BC1F115
:10C060000F947F02D6011496ED91FC9100A511A5C5
:10C0700022A533A5601B710B820B930B68387341AB
:10C080008105910528F1D601ED91FC910484F58597
:10C09000E02D65E0C6011995F6010481158180E067
:10C0A0000F94C542D80198966D937D938D939C9380
:10C0B0009B97D6011496ED91FC9117A269EA7AE05C
:10C0C00089E390E10F94E42389E390E10F947822CF
:10C0D000F60187819085DC01ED91FC910084F1856A
:10C0E000E02D1995892B19F481E090E03FC062E0C2
:10C0F00070E080E090E00F948D00F60187819085DC
:10C10000DC01ED91FC910284F385E02D1995E0CFDF
:10C11000D6011496ED91FC9180A591A5A2A5B3A599
:10C12000892B8A2B8B2BE1F00F947F02D60114967A
:10C13000ED91FC9140A451A462A473A46419750903
:10C1400086099709683873418105910548F0D60141
:10C15000ED91FC910484F585E02D65E0C60119950B
:10C160000130110509F4D3CE90E080E0CE57DF4FC7
:10C170000FB6F894DEBF0FBECDBFDF91CF911F91F8
:10C180000F91FF90EF90DF90CF90BF90AF909F9076
:10C190008F907F906F905F904F903F90089568E9E7
:10C1A0007AE089E390E10F94E4234AE050E0F6015D
:10C1B000668189E390E10F949B2263E97AE089E349
:10C1C00090E10F94E423D6011496ED91FC91E00FD9
:10C1D000F11F608140E150E06A3078F462EA75E076
:10C1E00089E390E10F94CE23D6011496ED91FC9152
:10C1F000E00FF11F40E150E0608189E390E10F948E
:10C200009B220F5F1F4F04321105E9F6D6011496E9
:10C21000ED91FC9184A1DF011296AF014C5D5F4F5F
:10C2200090E04A175B0719F02D91920FFACF89130E
:10C230007AC297A160E87AE0981709F470C287A3E0
:10C24000D6011496ED91FC91EF961CAE1DAE1EAE7C
:10C250001FAEEF97C158DF4F188219821A821B82D6
:10C26000CF57D040ED968FADED97807FED968FAF95
:10C27000ED9783A190E04C01B0E18B0E911C4997A2
:10C2800008F04BC23584878986A3118D738CD60143
:10C2900014962D913C91858DD90195968C93E48CC3
:10C2A000F12C878DD6011296ED91FC910280F381DD
:10C2B000E02D4EE757E06BEE76E080FD02C06CEFBC
:10C2C00076E0808191810F943703B0E8EB16F1049A
:10C2D00009F084C0D6011296ED91FC910280F381A1
:10C2E000E02D45E857E06BEE76E0808191810F9478
:10C2F00037036BE877E089E390E10F94CE23D60112
:10C300001496ED91FC914AE050E065A189E390E13B
:10C310000F949B2289E390E10F947822D601149622
:10C32000ED91FC91159785A11296ED91FC910280FB
:10C33000F381E02D46E957E06BEE76E083FD02C025
:10C340006CEF76E0808191810F943703D6011296CD
:10C35000ED91FC9113970280F381E02D8081918112
:10C360001496ED91FC9125A14DE957E06BEE76E036
:10C3700021FD02C06CEF76E00F9437031982113073
:10C3800009F4D6C1D0F1123009F4F7C1133009F421
:10C3900019C26CE77AE0CE0101960F94B75060E0C5
:10C3A000CE0185589F4F0E94727364962FAF649799
:10C3B00065963FAF659766964FAF669767965FAF96
:10C3C000679768966FAF689769967FAF69976A9627
:10C3D0008FAF6A976B969FAF6B9733C0EF2809F0CA
:10C3E00088CFD6011296ED91FC910280F381E02D69
:10C3F00045E857E06CEF76E078CF64E47BE0CE016F
:10C4000001960F94B75060E1CE0185589F4F0E946E
:10C410007273E4962FAFE497E5963FAFE597E69603
:10C420004FAFE697E7965FAFE797E8966FAFE8976D
:10C43000E9967FAFE997EA968FAFEA97EB969FAFC1
:10C44000EB97D6011296ED91FC910280F381E02DDD
:10C4500040E256E0BE016F5F7F4F808191810F9473
:10C460003703EC96EFACEC97ED96FFACED97EE96BC
:10C470000FADEE97EF961FADEF97C158DF4F2881B4
:10C48000CF57D040C058DF4F3881C058D040CF5729
:10C49000DF4F4881C158D040CE57DF4F5881C25836
:10C4A000D04061E276E0C6010E94F15ED6011296AC
:10C4B000ED91FC910280F381E02D45E256E06CEFB6
:10C4C00076E0772011F06BEE76E0808191810F9419
:10C4D0003703092C000CAA08BB08D6011296ED916F
:10C4E000FC910280F381E02D6081718106E116E00C
:10C4F000A5019401C6010E94ECE6432C512C712C3D
:10C50000612CBFEF3B1681F0D6011296ED91FC91A4
:10C510000280F381E02D6081718109EA17E0A301B7
:10C520009201C6010E94ECE61B861C861D861E86B3
:10C530001F86188A198A1A8A8C85807F8C87B50194
:10C54000A401CE010B960E9494732C962FAF2C97CA
:10C550002D963FAF2D972E964FAF2E972F965FAF0C
:10C560002F9760966FAF609761967FAF61976296E5
:10C570008FAF629763969FAF639779018A019B01A2
:10C58000AC0167E176E0C6010E94F15E1B861C8665
:10C590001D861E861F86188A198A1A8A8C85807FB6
:10C5A0008C87B301A201CE010B960E9494732B8B52
:10C5B0003C8B4D8B5E8B6F8B788F898F9A8F63E06E
:10C5C000CE0143960E94507324962FAF2497259650
:10C5D0003FAF259726964FAF269727965FAF2797B1
:10C5E00028966FAF289729967FAF29972A968FAF05
:10C5F0002A972B969FAF2B9779018A019B01AC015B
:10C600006AEA77E0C6010E94F15E1982D6011496AB
:10C61000ED91FC9186A18111FAC062E37BE0CE012D
:10C6200001960F94B7506EE0CE0185589F4F0E943F
:10C6300072732BAF3CAF4DAF5EAF6FAF21967FAF44
:10C64000219722968FAF229723969FAF2397D601EB
:10C650001496ED91FC91159726A130E050E040E052
:10C660001296ED91FC910280F381E02D6081718141
:10C670000FEA17E0C6010E94ECE6D6011496ED9190
:10C68000FC9185A180FD14C066EC7AE0CE01019694
:10C690000F94B75062E0CE0185589F4F0E9472738D
:10C6A0002B873C874D875E876F87788B898B9A8B2A
:10C6B000D6011296ED91FC910280F381E02D4BE1C1
:10C6C00056E0BE016F5F7F4F808191810F943703E9
:10C6D000EC96EFACEC97ED96FFACED97EE960FADC8
:10C6E000EE97EF961FADEF97C158DF4F2881CF57D8
:10C6F000D040C058DF4F3881C058D040CF57DF4FAF
:10C700004881C158D040CE57DF4F5881C258D040E1
:10C710006CE176E0C6010E94F15E6CE87AE089E3A4
:10C7200090E10F94E42389E390E10F947822DCCC2C
:10C730006DE47BE0CE0101960F94B75061E1CE012C
:10C7400085589F4F0E947273AC962FAFAC97AD96F1
:10C750003FAFAD97AE964FAFAE97AF965FAFAF9787
:10C76000E0966FAFE097E1967FAFE197E2968FAFEB
:10C77000E297E3969FAFE39764CE66E57BE0CE0158
:10C7800001960F94B75062E1CE0185589F4F0E94E9
:10C790007273A4962FAFA497A5963FAFA597A696C0
:10C7A0004FAFA697A7965FAFA797A8966FAFA8972A
:10C7B000A9967FAFA997AA968FAFAA97AB969FAF7E
:10C7C000AB973FCE62E37BE0CE0101960F94B7506A
:10C7D0006EE0CE0185589F4F0E9472736C962FAF0A
:10C7E0006C976D963FAF6D976E964FAF6E976F9645
:10C7F0005FAF6F97A0966FAFA097A1967FAFA197FD
:10C80000A2968FAFA297A3969FAFA3971ACE81301F
:10C81000A9F468E67BE0CE0101960F94B75064E17D
:10C82000CE0185589F4F0E9472732BAB3CAB4DAB32
:10C830005EAB6FAB78AF89AF9AAF09CF8230A9F406
:10C840006FE57BE0CE0101960F94B75063E1CE0116
:10C8500085589F4F0E9472732BA73CA74DA75EA7D8
:10C860006FA778AB89AB9AABF2CE8330A9F46BE3B8
:10C870007BE0CE0101960F94B7506FE0CE01855852
:10C880009F4F0E9472732BA33CA34DA35EA36FA383
:10C8900078A789A79AA7DBCE8430A9F461E77BE06B
:10C8A000CE0101960F94B75065E1CE0185589F4F98
:10C8B0000E9472732B8F3C8F4D8F5E8F6F8F78A38A
:10C8C00089A39AA3C4CE8D3609F0C1CE6CE77AE075
:10C8D000CE0101960F94B75060E0CE0185589F4F6E
:10C8E0000E9472732B8B3C8B4D8B5E8B6F8B788F82
:10C8F000898F9A8FACCE8FEF9FEF38CC2F923F92DB
:10C900004F925F926F927F928F929F92AF92BF925F
:10C91000CF92DF92EF92FF920F931F93CF93DF930B
:10C92000CDB7DEB768970FB6F894DEBF0FBECDBFA8
:10C930003C018091870A68EF79E0882309F46AC195
:10C9400061E070E080E090E00F948D00BE016F5FC9
:10C950007F4F80E00E944DF9892B09F059C18981F0
:10C9600083FF56C144E0BE016F5F7F4F82E00E94AB
:10C9700047FA009791F429813A81322723273227F9
:10C980003093A50D2093A40D2B813C8132272327C2
:10C9900032273093A30D2093A20D0E941AF967ED60
:10C9A00079E089E390E10F94E4236091A40D709104
:10C9B000A50D90E080E00F94A856562E798B8A8BB7
:10C9C000492E462F572F682F792F89E390E10E9437
:10C9D00080F26FEC79E089E390E10F94E4236091B9
:10C9E000A20D7091A30D90E080E00F94A8566B8B80
:10C9F0007C8B8D8B9E8BAB01BC0189E390E10E9407
:10CA000080F263EC79E089E390E10F94E42342E063
:10CA1000BE016F5F7F4F81E10E9447FA49815A81D1
:10CA2000542745275427892B11F050E040E070E04F
:10CA300060E04093920A5093930A6093940A709333
:10CA4000950A2AE030E089E390E10F943D2320E04D
:10CA500030E44CE156E4652D79898A89942D0F9450
:10CA6000A35687FF7AC0D3011296ED91FC912080E6
:10CA7000318065EB77E0C1010E943AED988F8F8B92
:10CA800069EB77E0C1010E943AED1C0119821A821C
:10CA90001B821C828A81807F8760F82E8A83252DE5
:10CAA000852D9989AA89B42D8D839E83AF83B887FC
:10CAB000912C812CB12CA12CD12CC12CE9800B8183
:10CAC0001C813E814F8158856FEF8F89988D0E9420
:10CAD000603E19821A821B821C828A81807F876055
:10CAE000F82E8A832B89822F9C89AD89BE898D83FC
:10CAF0009E83AF83B887E9800B811C813E814F8183
:10CB000058856FEFC1010E94603E2EEB37E0452D46
:10CB100059896A89742DC3010E94C4E623EC37E069
:10CB20004B895C896D897E89C3010E94C4E660914E
:10CB3000920A7091930A8091940A9091950A2AE042
:10CB4000AE014F5F5F4F0F94525149EC57E0BE0169
:10CB50006F5F7F4FC3010E949AE66FEC77E089E335
:10CB600090E10F947C22BE016F5F7F4F80EE0E94A8
:10CB70004DF9892B19F419811F3F49F46AE979E0CD
:10CB800082E99FE00F94082481E090E04DC01123DA
:10CB900031F06BE879E082E99FE00F94E42315FF20
:10CBA00006C06EE779E082E99FE00F94E42314FF6A
:10CBB00006C062E779E082E99FE00F94E42313FF67
:10CBC00006C064E679E082E99FE00F94E42312FF57
:10CBD00006C064E579E082E99FE00F94E42311FF49
:10CBE00006C065E479E082E99FE00F94E42310FF3A
:10CBF0000BC06AE379E082E99FE00F94E42382E9C5
:10CC00009FE00F947822C0CF112309F4BDCFF7CF56
:10CC10006DED79E089E390E10F94E42389E390E1FD
:10CC20000F94782290E080E068960FB6F894DEBF0B
:10CC30000FBECDBFDF91CF911F910F91FF90EF906D
:10CC4000DF90CF90BF90AF909F908F907F906F902C
:10CC50005F904F903F902F9008952F923F924F9268
:10CC60005F926F927F928F929F92AF92BF92CF927C
:10CC7000DF92EF92FF920F931F93CF93DF93CDB785
:10CC8000DEB760970FB6F894DEBF0FBECDBF613040
:10CC9000710579F42C018091860A811125C061E229
:10CCA00079E082E99FE00F94E42382E99FE00F940A
:10CCB000782290E080E060960FB6F894DEBF0FBE59
:10CCC000CDBFDF91CF911F910F91FF90EF90DF903B
:10CCD000CF90BF90AF909F908F907F906F905F901C
:10CCE0004F903F902F90089560E179E089E390E1C3
:10CCF0000F94E42382E00F94C000692E712C40E170
:10CD000050E0B30189E390E10F9485238FEF68161B
:10CD1000710409F42DC161ED77E089E390E10F948E
:10CD2000CE2380E00F94C000BC0190E080E00F941F
:10CD3000A85620E030E040E857E30F94095720E080
:10CD400030E045E253E40F94095720E030E040E240
:10CD500052E40F949658762E272E382E692E462FA1
:10CD6000572F682F792F89E390E10E9480F269E0C4
:10CD700079E089E390E10F94E42381E00F94C0000F
:10CD8000BC0190E080E00F94A85620E030E040E83D
:10CD900057E30F94095720E030E048EC52E40F9439
:10CDA000095769877A878B879C87AB01BC0189E328
:10CDB00090E10E9480F265ED77E089E390E10F94C5
:10CDC0007C22D2011296ED91FC91E080F1806AEA1A
:10CDD00077E0C7010E943AED9E878D8767ED77E087
:10CDE000C7010E943AED988B8F87272D322D432D56
:10CDF000562D672D722D832D962D0F940B5A811170
:10CE000040C019821A821B821C828A81807F8760BF
:10CE1000F82E8A83272D872D922DA32DB62D8D8355
:10CE20009E83AF83B887912C812CB12CA12CD12C5F
:10CE3000C12CE9800B811C813E814F8158856FEFA9
:10CE40008D859E850E94603E19821A821B821C82FB
:10CE50008A81807F8760F82E8A832985822F9A8530
:10CE6000AB85BC858D839E83AF83B887E9800B81BA
:10CE70001C813E814F8158856FEF8F8598890E9474
:10CE8000603E2BED37E0472D522D632D762DC201EC
:10CE90000E94C4E62EED37E049855A856B857C8576
:10CEA000C2010E94C4E68091870A882309F45DC00C
:10CEB00020E030E048EC51EC672D722D832D962D4B
:10CEC0000F94A35687FD51C020E030E048E452E4BF
:10CED000672D722D832D962D0F94AB5918160CF4D7
:10CEE00044C020E030E048EC52E469857A858B85C7
:10CEF0009C850F94AB591816C4F120E030E04AE746
:10CF000054E469857A858B859C850F9409570F9425
:10CF10007C5966507F4F8F4F9F4F24EFC22EDD24E8
:10CF2000D394E12CF12CA70196010F94ED5729839E
:10CF30001A8220E030E04AE754E4672D722D832DF9
:10CF4000962D0F9409570F947C596E557D498F4F3C
:10CF50009F4FA70196010F94ED572B831C82BE01B2
:10CF60006F5F7F4F85E00E949DF988EE93E0A3CE2E
:10CF700089E390E10F9478220F944B42F6CF0F9300
:10CF80001F93CF93DF93EC010E94F53661EE77E0BB
:10CF900089E390E10F947C2280919A0A90919B0AF8
:10CFA000892B19F586E190E00F94754E8C012B8545
:10CFB0003C854A85042E000C550B688579850F94B5
:10CFC000332910939B0A00939A0AF801868197816E
:10CFD00097FD08C061E00E9448FE60E0F80186818C
:10CFE0000E941AFE81E0F8018183E881F9810484BE
:10CFF000F585E02D62E0CE01199581E090E0DF91AA
:10D00000CF911F910F9108958FE090E090933B0C8A
:10D0100080933A0C88EC90E00895FC01848195811E
:10D02000089568EF73E2811102C06AEF73E288E845
:10D030009FE00D94E4236AE87FE188E89FE00F9485
:10D04000E423F0E0E0E0199584EF91E00895809109
:10D05000690B8823B1F0E0916A0BF0916B0B30976C
:10D0600031F0868197819093680B8093670B6FED09
:10D070007CE188E89FE00F94E42388E89FE00D942A
:10D0800078220895EF92FF920F931F93CF93DF932F
:10D09000CDB7DEB760970FB6F894DEBF0FBECDBF39
:10D0A0008091860A8823C9F06AEC77E289E390E1EF
:10D0B0000F94E42389E390E10F94782290E080E0DC
:10D0C00060960FB6F894DEBF0FBECDBFDF91CF9153
:10D0D0001F910F91FF90EF9008956EE178E289E340
:10D0E00090E10F94E4230E94D7F980E48093AE0D81
:10D0F0000E94D7F910E01B7F8091AE0D0E9443F98A
:10D1000062E08BE89DE00F94851D612F8BE89DE028
:10D110000F94851D60E08BE89DE00F94851D8BE8E2
:10D120009DE00F94B73E6AE070E080E090E00F94DD
:10D130008D006BE078E289E390E10F94E4238EEFB9
:10D140000F94C00040E150E0BC0189E390E10F94EE
:10D1500095226DEF77E289E390E10F94E4238FEF5E
:10D160000F94C00040E150E0BC0189E390E10F94CE
:10D17000952289E390E10F94782267EE77E288E8C0
:10D180009FE00F94E4238BEF0F94C000182F092F1A
:10D190008CEF0F94C000F82EE92E8DEF0F94C00095
:10D1A0009F938F93EF92FF920F931F938EEE97E0D2
:10D1B0009F938F938E010F5F1F4F1F930F930F94B9
:10D1C000565DB80188E89FE00F947C2281E080934F
:10D1D000860A0FB6F894DEBF0FBECDBF81E090E0A7
:10D1E0006FCF0F931F93CF93DF9300D000D01F9288
:10D1F000CDB7DEB78091870A882369F06DE877E2C2
:10D2000082E99FE00F94E42382E99FE00F94782263
:10D2100090E080E0B0C06DEB77E288E89FE00F948B
:10D2200008240E94D7F98091640290916502A09130
:10D230006602B091670289839A83AB83BC838BE8D3
:10D240009DE09093980D8093970D1E8280E197E268
:10D250002E812F5F2E830197D9F71D82BE016B5F50
:10D260007F4F80E20E944DF98C01892BF1F48D8172
:10D2700001E010E08138C9F4BE016F5F7F4F8FEF8E
:10D280000E949DF91F8280E89EE32F812F5F2F83EC
:10D290000197D9F7BE016B5F7F4F80E00E944DF987
:10D2A0008D8180FF0CC003E010E069EA77E282E93B
:10D2B0009FE00F94E423C8010E941AF9A9CFBE0190
:10D2C0006B5F7F4F80E00E944DF9892B61F78D8164
:10D2D00084FFE9CF8091990D0E9443F98091970DC9
:10D2E0009091980DDC01ED91FC910190F081E02D81
:10D2F00064EF19958091970D9091980D0F94B73E1A
:10D30000882319F002E010E0D0CFBE016B5F7F4FA1
:10D3100081E00E944DF98C01892B39F61D811F781F
:10D3200010611D838091990D0E9443F98091970DA2
:10D330009091980DDC01ED91FC910190F081E02D30
:10D3400061E019958091970D9091980DDC01ED9118
:10D35000FC910190F081E02D612F19958091970D3E
:10D360009091980D0F94B73E8111CCCF81E08093BE
:10D37000870A81E090E027960FB6F894DEBF0FBED3
:10D38000CDBFDF91CF911F910F910895CF93DF9380
:10D3900000D000D01F921F92CDB7DEB7E2E7FFE0CA
:10D3A000128A118A80E090E19587848784E890E072
:10D3B000948B838B81E0868787E7858B1C821B8219
:10D3C00086E193E09A838983FE83ED838FEF9FEF5D
:10D3D00098878F8363E777E288E89FE00F94E423E0
:10D3E0006091F40A7091F50ACE0101960E94A9F4A9
:10D3F00082E79FE00E94C4AB63E677E288E89FE0A3
:10D400000F94E42388E89FE00F9478220F94A20BF6
:10D4100028960FB6F894DEBF0FBECDBFDF91CF9137
:10D42000089560E08DE00C941AFE61E08DE00C94AC
:10D430001AFE892B71F0FB01828193810E940CEF0F
:10D4400061EE73E288E89FE00F94E42388EC90E0BB
:10D45000089590E080E0F2CF0F931F93CF93DF9376
:10D46000EB0102970CF49FC00A811B816EED72E202
:10D47000C8010F949050892B61F40E9472F17E7F55
:10D480000E94CCF188EC90E0DF91CF911F910F9139
:10D49000089567EE72E2C8010F949050892B21F431
:10D4A0000E9472F17160ECCF65EB72E288E89FE058
:10D4B0000F94E4230E9472F1672F609561704AE037
:10D4C00050E070E088E89FE00F94852388E89FE0B3
:10D4D0000F9478228091640F9091650F892B09F445
:10D4E00052C00A811B810E948DEE882309F44BC033
:10D4F000F80101900020E9F73197E01BF10BB0979C
:10D5000008F041C0A091640FB091650F52961C9233
:10D510001E92519754961C921E92539784E890E065
:10D520001D969C938E931C971E961C921E9782E7C5
:10D5300055968C935597ED91FC9111970088F18940
:10D54000E02D60E270E0CD011995B8018091640F83
:10D550009091650F0F94CE238091640F9091650F89
:10D56000DC01ED91FC910190F081E02D60E01995D6
:10D570008091640F9091650FDC01ED91FC9104881E
:10D58000F589E02D19956A817B8188E89FE00F94E9
:10D59000CE236EEA72E288E89FE00F94E42388E8E5
:10D5A0009FE00F94782280913A0C90913B0C029767
:10D5B0003CF080EF9FEF90933B0C80933A0C62CF4E
:10D5C00061EA72E282E99FE00F94E42382E99FE03E
:10D5D0000F94782284EF91E057CFCF93DF93EB0144
:10D5E0000297BCF16EED72E28A819B810F9490509C
:10D5F000892B29F40E9472F17D7F0E94CCF167EEA5
:10D6000072E28A819B810F949050892B29F40E94A9
:10D6100072F172600E94CCF16AE372E288E89FE0E6
:10D620000F94E4230E9472F171FB662760F971E0A8
:10D63000672770E04AE050E088E89FE00F94852378
:10D6400088E89FE00F94782288EC90E0DF91CF91FA
:10D6500008950E94C669F8CF892B71F0FB01828181
:10D6600093810E946DEF6BE872E288E89FE00F946F
:10D67000E42388EC90E0089590E080E0F2CFEF9210
:10D68000FF920F931F93CF93DF93CDB7DEB72C9705
:10D690000FB6F894DEBF0FBECDBF8C017B0180E5D5
:10D6A00095E09A8389831B821C821D821E82988743
:10D6B0008F8319861A861B861C8605301105ECF0AF
:10D6C000BE01695F7F4FF701808591850E946F34AD
:10D6D000892B99F0CE0107960E9437F0BE01695F51
:10D6E0007F4FF701868197810E946F34892B61F00B
:10D6F000CE0107960E9409F10EC0CE0101960E944C
:10D7000037F00430110554F7CE0101960E9409F15B
:10D7100003301105A4F1BE01695F7F4FF7018481D9
:10D7200095810E946F34892B51F1CE0107960E949A
:10D73000A0F0BE01695F7F4FF701828193810E9453
:10D740006F34892B19F1CE0107960E94CEEF64E762
:10D7500072E288E89FE00F94E42380E00E9430F2B8
:10D7600088EC90E02C960FB6F894DEBF0FBECDBFCC
:10D77000DF91CF911F910F91FF90EF900895CE010F
:10D7800001960E94A0F0023011059CF6CE01019690
:10D790000E94CEEF01301105D1F6CE0101960E9414
:10D7A000CEEF6BE772E288E89FE00F94E423CFCFDF
:10D7B000CF93C1E068EE73E080E090E00F948D00BD
:10D7C0004AE050E06C2F88E89FE00F949B22CF5FE7
:10D7D000C43181F784EF91E0CF9108950F931F93A7
:10D7E000CF93DF938C01EB010297C4F08A819B8178
:10D7F0000F9442508093450299270E9439F20230DB
:10D80000110549F08C819D810F9442508093440210
:10D8100099270E9443F2C8ECD0E002C0C0E9D1E0F1
:10D8200060E672E288E89FE00F94E4234AE050E06B
:10D830006091450288E89FE00F949B226BE472E2BE
:10D8400088E89FE00F94E4234AE050E060914402AE
:10D8500088E89FE00F949B2288E89FE00F9478224D
:10D86000CE01DF91CF911F910F9108950F931F93D8
:10D87000CF93DF93CDB7DEB769970FB6F894DEBFCD
:10D880000FBECDBFE0919A11F0919B11309709F432
:10D8900060C08091A4119091A511892B09F459C001
:10D8A0008FEF838714861382148215821682178263
:10D8B0001086118612866BEA7FE188E89FE00F945C
:10D8C000E42388E89FE00F947822BE016E5E7F4FCC
:10D8D00080919A1190919B110F943E411816CCF5AE
:10D8E000A895AE014F5F5F4F68E0CE0142960F945E
:10D8F000E041198ABE016F5F7F4F8091A411909122
:10D90000A5110E943AED8C0166EA7FE188E89FE06C
:10D910000F94E423BE016F5F7F4F88E89FE00F9470
:10D92000CE230115110591F0C8010E94D5368C0156
:10D93000892B59F261EA7FE188E89FE00F94E423A4
:10D94000B80188E89FE00F94CE23BBCF6CE97FE15C
:10D95000B4CF88EC90E069960FB6F894DEBF0FBEA6
:10D96000CDBFDF91CF911F910F910895CF92DF929C
:10D97000EF92FF920F931F93CF93DF9300D000D0CD
:10D98000CDB7DEB780918D0A81119CC080913A0C91
:10D9900090913B0C02970CF495C08091F40A909101
:10D9A000F50A009709F48EC06DEF77E00E943AED1A
:10D9B0008C01009709F486C00E947DEEE82EF12CC0
:10D9C000E114F10409F47EC070E060E0C8010F9436
:10D9D00035426C01EA94EF2809F483C061E0C80184
:10D9E0000E94ECEDFC0101851285CE0101960E949A
:10D9F0004FFBCE0101960E946DFB6EE578E188E851
:10DA00009FE00F94E423B60188E89FE00F94CE23B3
:10DA100062ED75E088E89FE00F94CE234AE050E085
:10DA2000B80188E89FE00F94852362ED75E088E8EF
:10DA30009FE00F94CE2363ED7BE088E89FE00F9496
:10DA4000CE2388E89FE00F94782262E072E087E5B9
:10DA500090E10F94AC33D0924D10C0924C101093C3
:10DA60004F1000934E1083ED9BE0892BE9F588ED74
:10DA700099E090935110809350108091670B909192
:10DA8000680B009741F070E060E00F94354290938E
:10DA90008F0A80938E0A80918E0A90918F0A009748
:10DAA00031F19093531080935210109255101092B0
:10DAB000541081E080938D0A65E478E188E89FE066
:10DAC0000F94E42326960FB6F894DEBF0FBECDBFA9
:10DAD000DF91CF911F910F91FF90EF90DF90CF904A
:10DAE000089502E012E081CF83ED9BE0C2CF8FEC7E
:10DAF00092E0D7CFEF92FF920F931F93CF93DF93D4
:10DB000000D000D0CDB7DEB77C018B016AE274E1B2
:10DB100089E390E10F94E423D7011296ED91FC91F3
:10DB20006081718189E390E10F94CE2361E274E119
:10DB300089E390E10F94E423012E000C220B330BB8
:10DB400009831A832B833C8380E190E09E838D833D
:10DB5000BE016F5F7F4F89E390E10E94B9D20F94BD
:10DB6000782240E050E860E070E0C7010E9496B182
:10DB700026960FB6F894DEBF0FBECDBFDF91CF91D2
:10DB80001F910F91FF90EF900895CF92DF92EF9247
:10DB9000FF920F931F93CF93DF93CDB7DEB7C1549E
:10DBA000D1090FB6F894DEBF0FBECDBF6C01AB013B
:10DBB00030E020E060E4CE0101967C010E948533D4
:10DBC000F70101900020E9F731978F010E191F0925
:10DBD000A801B701C6010F94F15C892B11F010E088
:10DBE00000E0C801CF5BDF4F0FB6F894DEBF0FBE79
:10DBF000CDBFDF91CF911F910F91FF90EF90DF90FC
:10DC0000CF9008953F924F925F926F927F928F9242
:10DC10009F92AF92BF92CF92DF92EF92FF920F93BB
:10DC20001F93CF93DF93CDB7DEB72C970FB6F89441
:10DC3000DEBF0FBECDBF5C01362E972E3A016901C3
:10DC40006BE874E189E390E10F94E4234AE050E04B
:10DC5000632D792D89E390E10F94852363E874E1C6
:10DC600089E390E10F94E423C301B0E0A0E08F8347
:10DC70009887A987BA8730E1432E512C5C864B8662
:10DC8000BE01695F7F4F89E390E10E94B9D24C01E8
:10DC90006FE774E10F94E4234AE050E0B601C40159
:10DCA0000F94852367E774E1C4010F94E423C7014F
:10DCB000B0E0A0E089839A83AB83BC835E824D820F
:10DCC000BE016F5F7F4FC4010E94B9D20F947822CA
:10DCD00080918B0A90918C0A70E060E0892B09F0AA
:10DCE00047C081E090E090938C0A80938B0A26E0F5
:10DCF00040E855E260E070E08AED9CE00F94312549
:10DD00003092DA0D8AED9CE09093D90D8093D80D76
:10DD10001092E80E1092EA0E1092E90E01301105F1
:10DD200009F44EC00CF041C0012B09F44EC0C114DF
:10DD3000D10409F457C082E0C816D10409F062C0CA
:10DD40007092630E6092620E1092650E1092640ED5
:10DD5000F092670EE092660E86E00F940A0410922D
:10DD60008C0A10928B0A882309F456C0682F70E041
:10DD7000C5010E947A6D90E080E02C960FB6F89471
:10DD8000DEBF0FBECDBFDF91CF911F910F91FF90EE
:10DD9000EF90DF90CF90BF90AF909F908F907F904B
:10DDA0006F905F904F903F9008950330110581F080
:10DDB0000430110509F0BBCFFE24EF24FE24B7CFB9
:10DDC000FE2CEE24EE24EA94B2CFFF24FA94AFCFD7
:10DDD000EF2821F492E0E92EF12CEECFEE24E3942B
:10DDE000F12CEACF7092630E6092620E90E080E0B8
:10DDF000EE2011F080E09FEF9093650E8093640E0B
:10DE000085E0ABCF6BE574E189E390E10F94E42307
:10DE100010928C0A10928B0A81E090E0AECFEF92C4
:10DE2000FF921F93CF93DF93192F7B01C82FD92F18
:10DE3000D7FF03C0D195C195D10961E08C2F0E9415
:10DE400048FE82E0E816F10499F460E08C2F0E940D
:10DE50001AFE6BE577E289E390E10F94E42389E30E
:10DE600090E1DF91CF911F91FF90EF900D94782278
:10DE7000612FEF2851F46095661F6627661F8C2F6F
:10DE80000E941AFE67E577E2E6CF661F6627661FE7
:10DE90008C2F0E941AFE62E577E2DDCFAF92BF922F
:10DEA000DF92EF92FF920F931F93CF93DF93CDB743
:10DEB000DEB72E970FB6F894DEBF0FBECDBF209110
:10DEC000A0113091A111232B09F4B8C020919F110A
:10DED0002111B4C07C0180919F118F5F80939F11AD
:10DEE00080919E118F5F80939E110F947F0200910D
:10DEF000710B1091720B2091730B3091740B601B9E
:10DF0000710B820B930B6B3071058105910508F441
:10DF10008BC083E0E816F104A9F00F947F02009112
:10DF20006D0B10916E0B20916F0B3091700B601B7D
:10DF3000710B820B930BDD24D3946436710581053C
:10DF4000910508F4D12CE091A011F091A111068166
:10DF500017810115110509F449C0F80180858F70FA
:10DF6000863009F03FC01987088770E060E0CE0175
:10DF700008960E948CD9B701CE0108960E94B3DFA3
:10DF8000DD2031F064E070E0CE0108960E94B3DF3E
:10DF90006AEA76E0C8010E943AEDFC01892B11F192
:10DFA00090859F7095509230E8F4A680B780A114B8
:10DFB000B104C1F0BA82A982B801CE0101960E94D3
:10DFC0008CD9B701CE0101960E94B3DFDD2031F07C
:10DFD00064E070E0CE0101960E94B3DFF501A280FB
:10DFE000B380E5CFF80102811381B3CFF3E0EF16E0
:10DFF000F10451F00F947F026093710B7093720BD8
:10E000008093730B9093740BDD2051F00F947F027B
:10E0100060936D0B70936E0B80936F0B9093700BEE
:10E020001092A6101092A71080919E11815080939B
:10E030009E1180919F11815080939F112E960FB653
:10E04000F894DEBF0FBECDBFDF91CF911F910F912E
:10E05000FF90EF90DF90BF90AF900895A89582E079
:10E0600090E00C944E6F8091390C8F5F8093390C47
:10E07000A89583E090E00E944E6F0F94752B8091DD
:10E08000390C81508093390C089560E377E288E879
:10E090009FE00F94E4236DE177E288E89FE00F941E
:10E0A000E4236FE077E288E89FE00F94E42367E0E1
:10E0B00077E288E89FE00F94E42388E89FE00F94DC
:10E0C000782267EF76E288E89FE00F94E4236BEE16
:10E0D00076E288E89FE00F94E4236EED76E288E82C
:10E0E0009FE00F94E42369EC76E288E89FE00F94C8
:10E0F000E4236AEB76E288E89FE00F94E42362EB86
:10E1000076E288E89FE00F94E42361EA76E288E80B
:10E110009FE00F94E4236BE776E288E89FE00F949A
:10E12000E4236EE676E288E89FE00F94E42364E659
:10E1300076E288E89FE00F94E42365E576E288E8DC
:10E140009FE00F94E4236DE476E288E89FE00F946B
:10E15000E42361E476E288E89FE00F94E42367E239
:10E1600076E288E89FE00F94E42368E076E288E8AE
:10E170009FE00F94E42363EF75E288E89FE00F943B
:10E18000E4236BED75E288E89FE00F94E4236DECE7
:10E1900075E288E89FE00F94E42361EC75E288E87B
:10E1A0009FE00F94E42369EB75E288E89FE00F9409
:10E1B000E4236EEA75E288E89FE00F94E42361EAC5
:10E1C00075E288E89FE00F94E42369E975E288E846
:10E1D0009FE00F94E4236EE875E288E89FE00F94D7
:10E1E000E4236FE775E288E89FE00F94E42366E795
:10E1F00075E288E89FE00F94E42368E675E288E81A
:10E200009FE00F94E4236AE575E288E89FE00F94AD
:10E21000E4236EE475E288E89FE00F94E42366E46B
:10E2200075E288E89FE00F94E42363E375E288E8F1
:10E230009FE00F94E42369E275E288E89FE00F9481
:10E24000E42388E89FE00D9478220F931F93CF93E7
:10E25000DF9300D000D0CDB7DEB70E94457066EFE7
:10E260007CE188E89FE00F94E423CE0101960E94B0
:10E270004FFBCE0101960E94193400E515E01A8388
:10E2800009838091850D9091860DA091870DB091A5
:10E29000880D8B839C83AD83BE83CE0101960E9443
:10E2A00019341A8309831B821C821D821E8280E519
:10E2B00090E00E944CFB44E050E0BE016D5F7F4F58
:10E2C00081E090E00F94622E0F94592FCE010196B9
:10E2D0000E9419341A8309831B821C821D821E82AC
:10E2E00080E590E00E944CFB44E050E0BE016D5F91
:10E2F0007F4F85E090E00F94622E0F94592FCE014E
:10E3000001960E9419346CE17DE188E89FE00F944A
:10E31000E42388EC90E026960FB6F894DEBF0FBE9B
:10E32000CDBFDF91CF911F910F910895CF92DF92D2
:10E33000EF92FF921F93CF93DF9300D000D0CDB721
:10E34000DEB760E478E188E89FE00F94E4238CE690
:10E35000E82E8FE0F82E10E090E1C92ED12CF701C5
:10E3600081917F01803130F462EA75E088E89FE0B6
:10E370000F94CE23153041F1F7013197808190E061
:10E38000B0E0A0E089839A83AB83BC83DE82CD8238
:10E39000BE016F5F7F4F88E89FE00E94B9D26EE3B5
:10E3A00078E10F94E4231F5F1630C9F626960FB666
:10E3B000F894DEBF0FBECDBFDF91CF911F91FF90CC
:10E3C000EF90DF90CF9008958091710F90E0B0E0D2
:10E3D000A0E089839A83AB83BC83DE82CD82BE01B9
:10E3E0006F5F7F4F88E89FE00E94B9D20F94782238
:10E3F000DACFEF92FF920F931F93CF93DF9300D06A
:10E4000000D01F92CDB7DEB77B01CE0107969F9358
:10E410008F9301979F938F9301979F938F9301976A
:10E420009F938F9301979F938F9301979F938F93C0
:10E430008E010F5F1F4F1F930F9384E098E09F930F
:10E440008F93DB0113968C9113978F9312968C9177
:10E450008F930F94865D0FB6F894DEBF0FBECDBFCD
:10E460000697ECF466EB73E282E99FE00F94E423F5
:10E47000D70112966D917C9182E99FE00F94CE2393
:10E4800080E991E027960FB6F894DEBF0FBECDBFAE
:10E49000DF91CF911F910F91FF90EF9008958091A0
:10E4A000640F9091650F892B09F449C00E948DEE8D
:10E4B000882309F444C0A091640FB091650F52966F
:10E4C0001C921E92519754961C921E92539784E868
:10E4D00090E01D969C938E931C971E961C921E97FF
:10E4E00082E755968C935597ED91FC911197008892
:10E4F000F189E02D64E070E0CD0119958091640F01
:10E500009091650FDC01ED91FC910280F381E02D8B
:10E5100046E050E0B801199586E0F801ACE6BFE0AE
:10E5200001900D928A95E1F78091640F9091650FAB
:10E53000DC01ED91FC910488F589E02D19950E948C
:10E54000967168EC73E288E89FE00F94E42388EC0E
:10E5500090E098CFCF92DF92FF920F931F93CF93CB
:10E56000DF93F12C6115710509F48DC06A01EB018F
:10E570008C01CB010E9471AFF82E882309F483C06F
:10E58000D6FE0EC0D8018C918B3009F450C008F033
:10E5900041C040E051E060E070E08A3009F450C0D2
:10E5A000D4FE09C0F801608186EF860F843018F030
:10E5B000CE010E94C1B7D5FE66C0D80114964D9118
:10E5C0005D916D917C91179711968C918F7087302A
:10E5D00030F08930C8F18A50823008F45DC0CE0135
:10E5E0000E941EB0EE81FF81309709F44CC08085F7
:10E5F0008F709EEF980F923010F0811144C0D801B7
:10E6000011968C91982F9295907F80858F70892B91
:10E61000808739C08C3081F040E056E060E070E0E7
:10E620008D3009F0BDCFCE010E9496B1B9CF40E048
:10E6300051E060E070E0F7CF40E056E060E070E06D
:10E64000CE010E946DB1ACCFEE81FF813097D9F041
:10E6500080858F709EEF980F923010F0811113C05B
:10E660004187528763877487EE81FF818085807F31
:10E6700083608087EE81FF818085982F907F8F70E7
:10E680008067903629F28F2DDF91CF911F910F91E6
:10E69000FF90DF90CF900895CE010E941EB0F3CF7F
:10E6A000CF93DF9300D000D01F921F92CDB7DEB77B
:10E6B000FC01628398E0DE01119601900D929A951B
:10E6C000E1F729813A814B815C816D817E818F8167
:10E6D000988528960FB6F894DEBF0FBECDBFDF91A8
:10E6E000CF910895CF93DF9300D000D01F921F9257
:10E6F000CDB7DEB7FC01608398E0DE011196019092
:10E700000D929A95E1F729813A814B815C816D8167
:10E710007E818F81988528960FB6F894DEBF0FBE54
:10E72000CDBFDF91CF910895CF93DF9300D000D07C
:10E730001F921F92CDB7DEB7FC019181907F9A6046
:10E740009183448355836683778388E0DE01119645
:10E7500001900D928A95E1F729813A814B815C8184
:10E760006D817E818F81988528960FB6F894DEBFE3
:10E770000FBECDBFDF91CF910895AF92BF92CF92E0
:10E78000DF92EF92FF920F931F93CF93DF9300D00E
:10E7900000D01F921F92CDB7DEB76115710509F445
:10E7A0005FC05A016B017C01CB010E9471AF082F41
:10E7B000882369F1D60116968D919C91009709F4F2
:10E7C00043C0FC011085212F2F703EEF320F3230F5
:10E7D00010F021112EC012951F70B4FE59C0C60151
:10E7E0000E94E0B7F7018083112381F18181807F4E
:10E7F000182B1183D6011696ED91FC918185928597
:10E80000A385B485F70184839583A683B783802F7E
:10E8100028960FB6F894DEBF0FBECDBFDF91CF9123
:10E820001F910F91FF90EF90DF90CF90BF90AF902E
:10E830000895253049F460E00E94ECED009721F046
:10E84000DC0118961C91C7CF10E0C7CFD6011696F1
:10E85000ED91FC9180858F70823021F0833051F0F2
:10E8600000E0D5CF4185528563857485C7010E943C
:10E870009473CDCF4185528563857485F70181817D
:10E88000807F876081834483558366837783BFCF8E
:10E890001123E1F2F701AACFCF93DF9300D000D08C
:10E8A0001F921F92CDB7DEB7FC016F3F710519F0C3
:10E8B00014F06FEF70E077FD60E09181892F8F7029
:10E8C00081508230C8F4648388E0DE0111960190A3
:10E8D0000D928A95E1F729813A814B815C816D81A6
:10E8E0007E818F81988528960FB6F894DEBF0FBE83
:10E8F000CDBFDF91CF910895907F91609183E3CF59
:10E90000CF92DF92EF92FF92DC01362F1196EC91BD
:10E910001197EF70EC3008F0B6C0F0E08827EC56A5
:10E92000FB488F4F0D9464584675CC74CC74437576
:10E93000437543751175D37443754375A074A07402
:10E9400014968D919D910D90BC91A02D662399F008
:10E95000B7FD9FC08F3F9105A105B10529F024F0B7
:10E960008FEF90E0A0E0B0E02FEF30E0A901481B6E
:10E97000590BCA010CC0B7FD89C08F3F9105A10595
:10E98000B10529F024F08FEF90E0A0E0B0E0FF9017
:10E99000EF90DF90CF90089514962C91822F90E005
:10E9A0006623A9F3E1CF1496CD90DD90ED90FC9015
:10E9B0001797662301F120E030E0A901C701B601F5
:10E9C0000F94A35687FD65C020E030E04FE753E485
:10E9D000C701B6010F94AB5918160CF457C0A70124
:10E9E000960160E070E08FE793E40F9496580F94DF
:10E9F0007559CB01CCCF20E030E0A901C701B601A9
:10EA00000F94A35687FD42C020E030E04FE753E467
:10EA1000C701B6010F94AB591816DCF1C701B60156
:10EA2000E6CF14966D917D918D919C91179733232C
:10EA3000B1F06D395FEF75078507950754F16115E2
:10EA400024E67207810591050CF52CE93FEF4FEFA5
:10EA50005FEF0F940F58C90181509F4F98CF6D39C8
:10EA60004FEF7407840794078CF0611554E675071F
:10EA70008105910574F424E630E040E050E00F9405
:10EA80000F58C90184CF8FEF9FEF81CF90E080E0D6
:10EA90007ECF8FEF90E07BCFCF93DF93EC01DB0154
:10EAA00089818F708630E1F128F481508230C8F07E
:10EAB00080E014C0873009F18A508230C8F72FEF08
:10EAC00030E00F947B5824E630E040E050E00F94B3
:10EAD0000F582C833D834E835F8381E0DF91CF917C
:10EAE00008952FEF30E00F947B5824E630E040E0AB
:10EAF00050E00F940F582C83F0CF2FEF30E00F949D
:10EB00007B5824E630E040E050E00F940F58CA01F3
:10EB1000B9010F94AA566C837D838E839F83DDCFCA
:10EB20002CE933E60F947B5824E630E040E050E0D7
:10EB30000F940F582C833D834E835F83B9CFDC0144
:10EB40001196EC911197EF70E150EB3008F039C05D
:10EB5000F0E08827E155FA488F4F0D946458D2753C
:10EB6000D275E175BA75BA75C375DA75DA75DA7585
:10EB7000BA75BA7514966D917D918D919C91179788
:10EB80000F94AA56089514966D917D918D919C9144
:10EB9000179724E630E040E050E00F940F58CA0188
:10EBA000B901EECF14966C9170E090E080E00F9484
:10EBB000A856089514966D917D918D919C9117970B
:10EBC000089560E070E0CB010895DC011196EC91AE
:10EBD0001197EF70E150EB3008F037C0F0E0882774
:10EBE000EB50FA488F4F0D946458077607762576D8
:10EBF0000076007616760D760D760D760076007628
:10EC000014966D917D918D919C911797089514960E
:10EC10006C9170E090E080E0089514966D917D9184
:10EC20008D919C9117970F947559089514966D9135
:10EC30007D918D919C91179724E630E040E050E063
:10EC40000F940F58CA01B901089560E070E0CB013C
:10EC50000895DC011196EC911197EF70E150EB30C3
:10EC600008F03EC0F0E08827E75CF9488F4F0D942C
:10EC700064584F764F7670764476447669765A7645
:10EC80005A765A764476447614962D913D914D915C
:10EC90005C911797A4E6B0E00F942E58089514964F
:10ECA0006C9184E6689FB0011124072E000C880B3C
:10ECB000990B089520E030E048EC52E414966D91F1
:10ECC0007D918D919C9117970F9409570F947559C9
:10ECD000089514966D917D918D919C91179708954B
:10ECE00060E070E0CB010895FC01A7812A2F2E7F00
:10ECF000C9F081818F7081508330A0F4A695A15016
:10ED0000BB0B2BE531E00F947B5824E630E040E06C
:10ED100050E00F940F58DA01C90187569F4FAF4F4B
:10ED2000BF4F08958FEF9FEF08952F923F924F921C
:10ED30005F926F927F928F929F92AF92BF92CF928B
:10ED4000DF92EF92FF920F93CF93DF9300D01F9249
:10ED5000CDB7DEB77C017A8369835C834B83DB01AB
:10ED60001C92FC0160818FEF860F883108F04BC048
:10ED700034FF49C0F9E06F9FB00111246C59794EFE
:10ED8000CD010F94E550D70111968C918F7041F011
:10ED90004B815C816FEF75E089819A810F94E15C12
:10EDA000E981FA8101900020E9F7319729813A81C0
:10EDB000E21BF30B19012E0E3F1E4B815C814E1B93
:10EDC0005F0B415051095C834B83D7011196EC9145
:10EDD0001197EF7009F4F5C0E150EC3008F0F1C084
:10EDE000F0E08827E950F9488F4F0D946458067772
:10EDF000A9771678757890785477267826782678CB
:10EE000042772A77AC7829803A80DFCFF701848176
:10EE1000282F30E050E040E0002359F030E0A4E635
:10EE2000B0E00F9441582FEF30E040E050E00F94F5
:10EE30000F585F934F933F932F9388E198E09F93F0
:10EE40008F93FC81FF932B812F933F922F920F94EE
:10EE5000195DB2C017968C9117978F9316968C9167
:10EE600016978F9315968C9115978F9314968C9176
:10EE70008F938BE198E09F938F93BC81BF93EB813D
:10EE8000EF93E3CF17968C9117978F9316968C91EB
:10EE900016978F9315968C9115978F9314968C9146
:10EEA0008F938FE198E0E7CF1496CD90DD90ED90B1
:10EEB000FC901797F7FE34C084E6882E912CA12C85
:10EEC000B12CC701B601A50194010F940F589B0105
:10EED000AC0188279927DC01821B930BA40BB50B8F
:10EEE000BF93AF939F938F9366277727CB016C19BE
:10EEF0007D098E099F09A50194010F940F585F9316
:10EF00004F933F932F9383E298E09F938F933C819D
:10EF10003F934B814F933F922F920F94195D4CC0BA
:10EF2000C701B60124E630E040E050E00F940F58EE
:10EF30009F938F937F936F935F934F933F932F9301
:10EF400084E298E09F938F939C819F93AB81AF93D2
:10EF5000E2CFC7010E947476BC01D7011696CC900F
:10EF600016971796DC901797D0FADD24D0F81496F0
:10EF70009C9114971596FC90EB80BC80292F30E073
:10EF800050E040E077FD35C0011135C07F936F93AD
:10EF90001F921F921F929F931F92FF92DF92CF9218
:10EFA0008DE298E09F938F93FC81FF932B812F93A9
:10EFB0003F922F920F94195D0FB6F894DEBF0FBEEB
:10EFC000CDBF89819A810F900F900F900F90DF91A4
:10EFD000CF910F91FF90EF90DF90CF90BF90AF90C7
:10EFE0009F908F907F906F905F904F903F902F9069
:10EFF0000895002361F0292F30E0A4E6B0E00F94DB
:10F0000041582FEF30E040E050E00F940F585F93ED
:10F010004F933F932F931F92FF92DF92CF9280E303
:10F0200098E09F938F93BF92EF9275CF15968C9136
:10F0300015971F928F9316969C91169717968C9101
:10F0400081708F939F9383E398E015CF14968D90F2
:10F050009D90AD90BC90179720E030E0A901C501CC
:10F06000B4010F94A3562401350187FF04C077FA39
:10F07000709477F87094C301B2010F9475596B01C5
:10F08000072E000C880B990B0F94AA569B01AC011C
:10F09000C301B2010F94965820E030E04AE754E4EF
:10F0A0000F9409570F94005A0F947559062F772E15
:10F0B00020E030E0A901C501B4010F94A35687FFF9
:10F0C00007C07F920F93DF92CF9289E398E0D3CE6F
:10F0D0007F920F93DF92CF928AE398E09F938F9372
:10F0E0003C813F934B814F93B0CE14968C911497F3
:10F0F0001F928F9315968C9115971F928F9316964A
:10F100008C911F928F9380E398E09F938F93BC81A3
:10F11000BF93EB81EF933F922F920F94195D4CCFE9
:10F1200017968C9117971F928F9314968C91149722
:10F130001F928F9315968C9115971F928F93169609
:10F140008C911F928F938DE298E09F938F93BC8157
:10F15000BF93EB81EF93DFCE14966D917C914B8141
:10F160005C81C1010F94FF5C2CCFEF92FF920F9353
:10F17000CF93DF93CDB7DEB7A0970FB6F894DEBF7D
:10F180000FBECDBF7C0100E020E030E340E250E064
:10F19000BE016F5F7F4F0E949576BE016F5F7F4F0C
:10F1A00089E390E10F94CE236CE477E189E390E169
:10F1B0000F94E423F70161816F704AE050E089E326
:10F1C00090E10F949B2265E477E189E390E10F944D
:10F1D000E4234AE050E0F701628189E390E10F9473
:10F1E0009B2289E390E10F947822A0960FB6F894C1
:10F1F000DEBF0FBECDBFDF91CF910F91FF90EF909B
:10F200000895CF93DF93EC016115710539F48F8177
:10F2100081708F8381E0DF91CF9108958981982F4C
:10F220009F7029F180E09430B0F79B01770F440B79
:10F23000550B2959310941095109A4E6B0E00F9451
:10F240002E582BE531E040E050E00F940F5837FF87
:10F2500002C030E020E02536310514F024E630E02D
:10F260002F5F220F8F818170282B2F83D3CF807F38
:10F2700082608983DACFFC019181892F8F7021F020
:10F28000823029F080E00895907F926091839B0105
:10F2900077FF02C030E020E02E3681E0380714F01E
:10F2A0002DE631E02683878130FB80F9878381E07A
:10F2B0000895EF92FF920F931F93CF93DF93FC017A
:10F2C000892B69F19081992351F19D3291F180ED63
:10F2D000890F8A3070F1C8E0D0E0953211F1CEEF9D
:10F2E000DFEF9B37F1F0C7E1D0E09332D1F08F012F
:10F2F0008DE6E82E86E1F82EC1E0D0E0C7010F943C
:10F30000BE50AC01B701C8010F94D750892B49F00A
:10F31000219689E0E80EF11CC931D10579F7CFEFCC
:10F32000DFEFCE01DF91CF911F910F91FF90EF9012
:10F330000895D0E0C0E0F5CFEF92FF920F931F93B6
:10F34000CF93DF93EC01892B51F188858F70843046
:10F3500009F5E984FA84C7010E9459798C011816CD
:10F360001906ECF4C7010F94C92BC801012E000C3B
:10F37000AA0BBB0B89879A87AB87BC878885807F60
:10F3800082608887C801DF91CF911F910F91FF9014
:10F39000EF900895823019F409851A85F3CF10E0B3
:10F3A00000E0F0CF2F923F924F925F926F927F9248
:10F3B0008F929F92AF92BF92CF92DF92EF92FF9285
:10F3C0000F931F93CF93DF93CDB7DEB7A4970FB6FC
:10F3D000F894DEBF0FBECDBF7C016B016CE176E01F
:10F3E000C6010E943AEDFC01892B09F422C18085F7
:10F3F0008F70843009F455C0853009F01AC1068138
:10F4000017810115110509F414C1D80118968C91C2
:10F4100018978F70823019F412960D911C91011576
:10F42000110509F406C1F80180858F70853011F04F
:10F43000D801F2CFC8010E947DEE8230C9F760E0AA
:10F44000C8010E94ECED5C010E949C7961E0C8015A
:10F450000E94ECED4C01FC0180858F70823041F7F9
:10F46000C7010E94E575D40119964D905D906D908D
:10F470007C901C976415750586059705C9F6A1143F
:10F48000B10409F4D6C019861A861B861C861D860F
:10F490001E861F86188A8A85807F8A87F501618586
:10F4A0004DC061E276E0818592850F94D15C892B15
:10F4B00009F0BFC0C7010E94E5756115710581059E
:10F4C000910509F49CC0660F771F881F991F2FEFC5
:10F4D00030E040E050E00F940F5857FD16C0233045
:10F4E0003105410551050CF070C0DA01C9010196E2
:10F4F000A11DB11D82309105A105B10509F44BC0D4
:10F500000397A105B10509F460C0198A1A8A1B8AFC
:10F510001C8A1D8A1E8A1F8A188E8A89807F8A8B80
:10F5200067E0CE0141960E94507329873A874B8746
:10F530005C876D877E878F87988B62E1CE01099605
:10F540000E94727329833A834B835C836D837E832D
:10F550008F83988729813A814B815C816D817E817F
:10F560008F819885A4960FB6F894DEBF0FBECDBFED
:10F57000DF91CF911F910F91FF90EF90DF90CF908F
:10F58000BF90AF909F908F907F906F905F904F90C3
:10F590003F902F900895198A1A8A1B8A1C8A1D8A07
:10F5A0001E8A1F8A188E8A89807F8A8B67E0CE0127
:10F5B00041960E94507329873A874B875C876D87F5
:10F5C0007E878F87988B61E1B9CF198A1A8A1B8A47
:10F5D0001C8A1D8A1E8A1F8A188E8A89807F8A8BC0
:10F5E00067E0CE0141960E94507329873A874B8786
:10F5F0005C876D877E878F87988B60E19FCF198AA4
:10F600001A8A1B8A1C8A1D8A1E8A1F8A188E8A895A
:10F61000807F8A8B67E0CE0141960E9450732987D4
:10F620003A874B875C876D877E878F87988B62E0F0
:10F6300085CF6AE376E0C6010E943AED8C0100971F
:10F6400009F41CC1DC0118968C918F70853009F08B
:10F65000FEC0C8010E947DEE843008F40FC160E056
:10F66000C8010E94ECED5C0161E0C8010E94ECED74
:10F670003C0162E0C8010E94ECEDDC0119962D917D
:10F680003D914D915C911C97298F3A8F4B8F5C8FE8
:10F6900063E0C8010E94ECED4C0165E0C8010E94E6
:10F6A000ECED6C0167E0C8010E94ECED8C01C70134
:10F6B0000E94E575298D3A8D4B8D5C8D621773071D
:10F6C0008407950714F5C114D10409F4C2C0D6010A
:10F6D00018968C9118978F70823009F0BAC01986ED
:10F6E0001A861B861C861D861E861F86188A8A859A
:10F6F000807F8A8719964D915D916D917C911C97C1
:10F70000CE0109960E9494731DCFD40119962D91B4
:10F710003D914D915C911C972D8F3E8F4F8F58A33B
:10F720002617370748075907D4F40115110509F4BE
:10F7300090C0F80180858F70823009F08AC01986E8
:10F740001A861B861C861D861E861F86188A8A8539
:10F75000807F8A874185528563857485D1CFD501A5
:10F760001996CD90DC90F3012184328419861A8693
:10F770001B861C861D861E861F86188A8A85807FAA
:10F780008A872101032C000C6608770846010D2C9E
:10F79000000CAA08BB08098D1A8D012E000C220B43
:10F7A000330B09A31AA32BA33CA3C7010E94E57541
:10F7B0009B01AC01E9A0FAA00BA11CA12E193F09E5
:10F7C000400B510BC301B201681979098A099B09E1
:10F7D0000F94DD570D8D1E8D9801110F440B550BA5
:10F7E000E9A0FAA00BA11CA12E193F09400B510B57
:10F7F0000F940F58820E931EA41EB51EC1018C19C2
:10F800009D096D8D7E8D098D1A8D601B710B0F9476
:10F81000505877FF02C06F5F7F4F75956795CB019A
:10F82000770FAA0BBB0B880D991DAA1DBB1D40E0CD
:10F8300050E0BA01B7FD64CFB301A2018417950768
:10F84000A607B7070CF05CCFAC01BD0159CF811101
:10F8500015C019861A861B861C868A85807F8A8732
:10F860001D861E861F86188A88E0FE013996DE01F5
:10F87000119601900D928A95E1F76CCE88E0F70120
:10F88000F6CF2F923F924F925F926F927F928F921C
:10F890009F92AF92BF92CF92DF92EF92FF920F931F
:10F8A0001F93CF93DF93CDB7DEB765970FB6F8946C
:10F8B000DEBF0FBECDBF6115710549F528E0FC0123
:10F8C000DE01119601900D922A95E1F729813A8186
:10F8D0004B815C816D817E818F81988565960FB6A5
:10F8E000F894DEBF0FBECDBFDF91CF911F910F9176
:10F8F000FF90EF90DF90CF90BF90AF909F908F9050
:10F900007F906F905F904F903F902F9008953B01B4
:10F910008C016CE176E0C3010E943AED6C01D801E4
:10F92000FC90FF2009F45AC0009709F457C0FC016D
:10F9300080858F70843009F4DEC0853009F04EC0B8
:10F9400080914502893020F480914402893050F042
:10F9500062E478E089E390E10F94CE2389E390E1BB
:10F960000F947822D6011696ED90FC90E114F104E4
:10F97000A9F1F70180858F705701823069F0B12CB1
:10F98000A12CE114F10409F436C1D70118968C9129
:10F990008F70853021F0F701E280F380F2CFC7014C
:10F9A0000E947DEE8230B9F760E0C7010E94ECED65
:10F9B0000E949C794C0161E0C7010E94ECED6C0152
:10F9C000D8018C918815190431F7F60180858F7064
:10F9D000823009F7C114D10409F017C16AE376E057
:10F9E000C3010E943AED7C01D80111968C918F7071
:10F9F00009F43BC1E114F10409F43BC1F70180852E
:10FA00008F70853009F0D0C1C7010E947DEE84302F
:10FA100008F4CAC164E0C7010E94ECED6C0166E025
:10FA2000C7010E94ECED1C01C8010E94E5754B0165
:10FA30005C0160E0C7010E94ECEDDC0119964D907D
:10FA40005D906D907C901C97B0914502B98B8414A9
:10FA50009504A604B7040CF016C1B93020F48091C7
:10FA60004402893050F164E476E189E390E10F9437
:10FA7000E423C8010E94E575AB01BC012AE030E037
:10FA800089E390E10F943D236EE276E189E390E112
:10FA90000F94E42360E0C7010E94ECEDFC01418576
:10FAA0005285638574852AE030E089E390E10F9404
:10FAB0003D2389E390E10F947822C114D10409F425
:10FAC00079C1D60118968C9118978F70823009F001
:10FAD00071C119821A821B821C821D821E821F82A2
:10FAE00018868A81807F8A8319964D915D916D91E8
:10FAF0007C911C9743C061E276E0818592850F94EA
:10FB0000D15C892B09F06ACFB0E1FB1609F463C020
:10FB1000BF1580F0E2E0FE1619F1D8014D915D911C
:10FB20006D917C91139714968D919D910D90BC9140
:10FB3000A02D38C0F1E1FF16F1F122E1F212EDCF74
:10FB400019821A821B821C821D821E821F821886C5
:10FB50008A81807F8A8344E150E060E070E00EC0DB
:10FB600019821A821B821C821D821E821F821886A5
:10FB70008A81807F8A8340E050E0BA01CE010196FD
:10FB80000E94947329873A874B875C876D877E87AD
:10FB90008F87988B49855A856B857C858D859E8559
:10FBA000AF85B88949835A836B837C838D839E8319
:10FBB000AF83B8878BCE19821A821B821C821D826A
:10FBC0001E821F8218868A81807F8A8340E850E0E7
:10FBD00060E070E0D3CF19821A821B821C821D82E2
:10FBE0001E821F8218868A81807F8A834FEF50E0B1
:10FBF00060E070E0C3CFA114B10409F4EFCEF501C9
:10FC000080858F7009F4EACE6501809145028930C4
:10FC100020F4809144028930B8F060E576E189E310
:10FC200090E10F94E423D60119964D915D916D9169
:10FC30007C911C972AE030E089E390E10F943D230A
:10FC400089E390E10F94782219821A821B821C8228
:10FC50001D821E821F8218868A81807F8A83F60118
:10FC6000418552856385748589CFE114F10409F0DB
:10FC70009BC0F801408151816281738184819581AB
:10FC8000A681B7818FCF61E0C7010E94ECEDDC0156
:10FC900019962D913D914D915C911C972A8B3B8B30
:10FCA0004C8B5D8B281539054A055B053CF5B989F8
:10FCB000B93020F480914402893050F060E176E15F
:10FCC00089E390E10F94E42389E390E10F94782293
:10FCD0002114310409F46EC0F10180858F708230E7
:10FCE00009F068C019821A821B821C821D821E8242
:10FCF0001F8218868A81807F8A83B2CF63E0C70122
:10FD00000E94ECED8C0162E0C7010E94ECEDDC0189
:10FD10001996CD90DD90ED90FC901C97F80121850F
:10FD20003285438554852C193D094E095F09C5016B
:10FD3000B40164197509860997090F94DD572A895A
:10FD40003B894C895D8924193509460957090F9467
:10FD50000F58C20ED31EE41EF51EF989F93020F4A7
:10FD600080914402893090F06BEF75E189E390E176
:10FD70000F94E4232AE030E0B701A60189E390E183
:10FD80000F943D2389E390E10F94782219821A821F
:10FD90001B821C821D821E821F8218868A81807FA0
:10FDA0008A83B701A601EACED70118968C918F708D
:10FDB00009F05FCF19821A821B821C828A81807FA0
:10FDC0008A8349815A816B817C8180E090E0DC01EB
:10FDD000E9CE8F929F92AF92BF92CF92DF92FF9225
:10FDE0000F931F93CF93DF93EC018A819B810E9435
:10FDF0007DEE082F10E00430110554F40E944DF3FD
:10FE0000BC018A819B810E945AF30F5F1F4FF3CF81
:10FE1000EA81FB81068117810115110531F0D801B6
:10FE200012968D919C919D838C83EC81FD813097FE
:10FE300021F0828193819F838E83EE81FF813097B1
:10FE400049F00280F381E02D309721F08281938187
:10FE5000998788870115110541F0F80180858F7019
:10FE6000843059F128F4823071F0FF24FA940CC0E8
:10FE7000853001F18630C9F762EE75E0C8010E9455
:10FE80003AED8C01E7CFF184FA86CE010E9471AF82
:10FE9000811138C010E000E01C870B87DF91CF9103
:10FEA0001F910F91FF90DF90CF90BF90AF909F90E8
:10FEB0008F90089506811781CDCFC184D284C1145B
:10FEC000D10499F2F6018081882379F295E9892E8F
:10FED00094E1992EB12CA12CFA2CC4010F94BE50A0
:10FEE000AC01B401C6010F94D750892BB9F1FFEFD3
:10FEF000AF1ABF0A89E0880E911CA7E1AA16B104C7
:10FF000059F7B3CFCE010E9462F28C010097B1F095
:10FF1000FC0182819381892B39F08F2D0E9478F327
:10FF20008C01892B09F4B6CFD801ED91FC910684A0
:10FF3000F785E02DBE01C8011995AECF8F2D0E9427
:10FF400078F38C01892B09F4A5CFEA85F0E0EE0F58
:10FF5000FF1FE858FF4E11830083E6CFC6010F94C0
:10FF6000C92B8A2D90E0B0E0A0E0F801818792874C
:10FF7000A387B4878085807F8260808785CF8F92BA
:10FF80009F92AF92BF92CF92DF92EF92FF920F9328
:10FF90001F93CF93DF93CDB7DEB760970FB6F8947A
:10FFA000DEBF0FBECDBF8C017B0140E050E860E0BA
:10FFB00070E00E94BFB1672B682B692B09F0B5C0B8
:10FFC00062E070E0C8010E948EB06C0119861A864A
:10FFD0001B861C861D861E861F86188A8A85807F42
:10FFE0008A87D7FCA2C040E050E2B801CE01099652
:10FFF0000E94BD7363E070E0C8010E948EB0AC0146
:020000021000EC
:100000001816190614F04FE350E081E0C816D10429
:1000100029F4EF2CFF0CFF08FF2404C082E0C8166F
:10002000D104D4F32FEF30E0D7010F947B589A011D
:10003000550F440B550B0F940F5849016901C80126
:100040000E94E0B7E82EF12C60E0CE0109960E94F4
:10005000807488169906F9F4CD2841F082E0E816FC
:10006000F10419F185E0E816F104F9F081E090E07F
:1000700060960FB6F894DEBF0FBECDBFDF91CF9173
:100080001F910F91FF90EF90DF90CF90BF90AF90B6
:100090009F908F900895CD2899F186E0E816F1049D
:1000A00041F081E0E816F10421F061E0C8010E940E
:1000B000C1B7B401CE0109960E944C7440E050E2F1
:1000C000B801CE0109960E94AA7282E0E816F104F6
:1000D00021F085E0E816F10449F430E020E040E04A
:1000E00050E160E070E0C8010E9429B530E020E0F6
:1000F00040E050E260E070E0C8010E9429B5B6CF50
:1001000085E0E816F10409F4B1CF82E0E816F104C5
:1001100009F4ACCF62E0C8010E94C1B730E020E032
:1001200040E050E160E070E0E7CF90E080E0A0CFF9
:10013000CF92DF92EF92FF920F931F93CF93DF93B3
:1001400000D000D01F921F92CDB7DEB77C0109838B
:100150001A832B833C834D835E836F837887CE0124
:1001600001960E94FBED8C018981882351F09B81CF
:10017000923008F0BAC0823011F0853011F410E0EE
:1001800000E070E060E0C7010E948EB0D82EC92E5A
:100190006EE374E189E390E10F94E4234AE050E0D8
:1001A0006D2D7C2D89E390E10F9485236CE374E140
:1001B00089E390E10F94E4234AE050E0B80189E339
:1001C00090E10F94852389E390E10F947822809148
:1001D0008B0A90918C0A892BE9F040E050E3B7013B
:1001E000CE0101960E94AA7270E060E0C7010E94F1
:1001F0007A6D90E080E028960FB6F894DEBF0FBECF
:10020000CDBFDF91CF911F910F91FF90EF90DF90C5
:10021000CF90089581E090E090938C0A80938B0AB0
:1002200026E040E855E260E070E08AED9CE00F9443
:100230003125D092DA0D8AED9CE09093D90D809310
:10024000D80D1092E80E1092EA0E1092E90E80ED91
:1002500097E09093630E8093620E1092650E109259
:10026000640E01151105E1F185E090E09093670EB1
:100270008093660E86E00F940A04D82E64E670E040
:1002800080E090E00F948D00D1100AC065E374E126
:1002900089E390E10F94E42389E390E10F947822BD
:1002A00082ED97E09093630E8093620E1092650E3C
:1002B0001092640E24E6209FC001219F900D11240E
:1002C0009093670E8093660E86E00F940A04109256
:1002D0008C0A10928B0A882359F0682F70E086CF21
:1002E0001092670E1092660EC5CF8FEF9FEF83CFEF
:1002F00081E090E080CF2F923F924F925F926F9279
:100300007F928F929F92AF92BF92CF92DF92EF92A5
:10031000FF920F931F93CF93DF93CDB7DEB72C9748
:100320000FB6F894DEBF0FBECDBF5C0109831A8300
:100330002B833C834D835E836F837887CE01019648
:100340000E94FBED1C01023011F0053011F4312C3C
:10035000212CF50104811581F80180858F7085308D
:1003600009F07FC0C8010E947DEEE82EF12CF2E07A
:10037000EF16F1040CF475C060E0C8010E94ECEDCA
:10038000FC01818592859C878B8761E0C8010E9472
:10039000ECEDFC01418452846384748488248A9443
:1003A000982CF2E0EF16F10459F062E0C8010E94C7
:1003B000ECEDFC0181849284F3E0EF16F104A1F4EA
:1003C0008FE390E09A87898792E0C92ED12C298506
:1003D0003A85D1010F94735824E630E040E050E0B4
:1003E0000F940F5879011CC063E0C8010E94ECED26
:1003F000FC01818592859A87898782E0C82ED12C5D
:10040000F4E0EF16F10439F064E0C8010E94ECED6D
:10041000FC01C184D28489859A857101892BB9F642
:1004200084019601A2016B857C85C5010E94026E44
:100430002C960FB6F894DEBF0FBECDBFDF91CF91E3
:100440001F910F91FF90EF90DF90CF90BF90AF90F2
:100450009F908F907F906F905F904F903F902F90E4
:10046000089590E080E0E4CFFF920F931F93CF9325
:10047000DF9300D000D0CDB7DEB78C01BC01CE0138
:1004800001960F940520BE016F5F7F4F89E390E1D5
:100490000F94D62389E390E10F947822CE01019640
:1004A0000F94FD1F1A8219821C821B821E821D82DC
:1004B0006CEF73E2CE0101960F94A01FF801248126
:1004C00035818D819E81F12C2817390738F0BE01C6
:1004D0006F5F7F4FC8010E94AFFCF82ECE010196DE
:1004E0000F94FD1FFF2069F0B801CE0101960F9413
:1004F0000520CE0101960F94210BCE0101960F9499
:10050000FD1F26960FB6F894DEBF0FBECDBFDF915C
:10051000CF911F910F91FF9008950F931F93CF9349
:10052000DF9300D000D0CDB7DEB7A091640FB091BB
:10053000650F109709F478C052961C921E9251973D
:1005400054961C921E92539784E890E01D969C93BB
:100550008E931C971E961C921E9787E755968C9338
:100560005597ED91FC9111970088F189E02D70E08D
:1005700060E0CD01199510E000E08091640F90914A
:10058000650FDC01ED91FC9111971C962D913C912A
:100590000217130740F40190F081E02D60E01995F7
:1005A0000F5F1F4FEACF0088F189E02D70E060E017
:1005B00019950FE914E08091640F9091650FF8018F
:1005C00061918F01DC01ED91FC910190F081E02DB2
:1005D0001995B4E0033A1B0771F78091640F90916D
:1005E000650FDC01ED91FC910488F589E02D1995EA
:1005F00065E37AE0CE0101960F940E20CE010196BC
:100600000F94210BCE0101960F94FD1F87E090E01F
:100610000E9439F287E090E00E9443F261ED73E2BC
:1006200088E89FE00F94E4231092840F1092830FC8
:1006300080E090E190937F0F80937E0F84E890E0BC
:100640009093860F8093850F81E08093800F82E7DF
:100650008093870F82E79FE00E945EAB82E79FE076
:100660000E94C4AB88EC90E026960FB6F894DEBFEB
:100670000FBECDBFDF91CF911F910F9108952F92A3
:100680003F924F925F926F927F928F929F92AF9222
:10069000BF92CF92DF92EF92FF920F931F93CF936F
:1006A000DF93CDB7DEB7E0970FB6F894DEBF0FBE8D
:1006B000CDBF8091F40A9091F50A892B09F432C7D5
:1006C00080919E1181112EC780919E118F5F809322
:1006D0009E1164EC71E288E89FE00F94E42388E8BF
:1006E0009FE00F9478220091F40A1091F50A60E5DA
:1006F00078E0C8010E943AED9093A3118093A21173
:1007000066E578E0C8010E943AED9093910A8093E3
:10071000900A62EF79E0C8010E943AED9093A1112E
:100720008093A0116DE578E0C8010E943AED9093A6
:100730006B0B80936A0B009749F1DC011696ED91E3
:10074000FC91309719F120852F702530F9F460EB7A
:1007500071E288E89FE00F94E42380916A0B909106
:100760006B0B0E947DEE8093690B4AE050E0682F8E
:1007700088E89FE00F949B2288E89FE00F947822FE
:10078000E0916A0BF0916B0B868197819093680BD7
:100790008093670B0E94B66C62E678E08091F40A61
:1007A0009091F50A0E943AED9093F30A8093F20A31
:1007B000009709F4B2C00E947DEE082F10E00115E9
:1007C000110509F4AAC0000F111F000F111F80911D
:1007D000F00A9091F10A892B09F08EC07801013856
:1007E00011051CF050E8E52EF12CC7010F94754E51
:1007F0009093F10A8093F00AE092EF0A109293111D
:10080000109292111092660B1092650B109291113A
:100810001092951110929411C70101960F94754E84
:1008200090939711809396119093901180938F11CC
:100830008E0D9F1D90938A11809389110F947F02D2
:1008400060938B1170938C1180938D1190938E1106
:1008500090E080E0E0919611F0919711E80FF91F78
:1008600010820196E816F906ACF782E090E09093CA
:100870009311809392118091650B9091660B009774
:1008800041F061E00E9448FE60E08091650B0E94AB
:100890001AFE80E98093C9001092C8001092CD0022
:1008A00083E08093CC008EE08093CA00F0924302F4
:1008B000E09242022091961130919711809142026C
:1008C00090914302820F931F90938A118093891114
:1008D000232B09F45FC060E471E289E390E10F9497
:1008E000E423B70189E390E10E944EF285E69EEA97
:1008F000909388118093871166E971E288E89FE000
:100900000F94E4234AE050E0B80188E89FE00F9498
:10091000852388E89FE00F94782268E678E080914C
:10092000F40A9091F50A0E943AED8C01009709F4BF
:1009300071C00E947DEE882309F46CC06FEF680FD0
:10094000C8010E94ECEDFC01E184F28490918511D4
:10095000992359F0809170008E7F809370001092DF
:10096000851110923E0210923D0282E180933C027A
:1009700091110F94883CC7010F94B03C01E010E046
:10098000E016F10674F060E0C8010F94E43C0F5FDC
:100990001F4FF6CF69E271E289E390E10F940824DA
:1009A000A5CF6BE171E289E390E10F94E4230E940B
:1009B0000635AB01BC012AE030E089E390E10F94F9
:1009C000932289E390E10F9478226AE771E288E844
:1009D0009FE00F94E4234AE050E0B70188E89FE0ED
:1009E0000F94852388E89FE00F94782264E771E2F2
:1009F00089E390E10F94E4230E940635AB01BC012A
:100A00002AE030E089E390E10F94932289E390E1BA
:100A10000F9478220091F40A1091F50A6CE678E0C0
:100A2000C8010E943AED90938A0A8093890A63E78D
:100A300078E0C8010E943AED9093A5118093A4112B
:100A4000892B09F448C08091A611811144C080917E
:100A50009A1190919B11892B09F0DFC165EF70E22B
:100A600089E390E10F94E42389E390E10F947822E5
:100A70008FE090E00F94754E8C0188E1D8011196BB
:100A80008C93119712961C9212971C921E961C9290
:100A90001E921D970E94D7F910939B1100939A11F3
:100AA000012B09F08CC066EE70E282E99FE00F94A2
:100AB000E42382E99FE00F94782280E081708093A4
:100AC000A6118091A611882331F064E671E288E8CE
:100AD0009FE00F94E42310929D1110929C11E091DD
:100AE000A211F091A311309709F4CCC2C680D7802F
:100AF0000091A2111091A3110115110509F4BBC2B7
:100B0000C114D10409F4B7C2F60180858F70853015
:100B100099F7C6010E947DEE823070F3A801B601FC
:100B2000CE0101960E94E9B8CE0101960E9471AFF4
:100B30008823E1F18C859D85009709F40DC2DC01C5
:100B4000ED91FC910284F385E02D1995892B49F0F4
:100B50008C859D85DC01ED91FC910084F185E02D73
:100B600019958C859D85DC01ED91FC910680F781BE
:100B7000E02D1995892BD1F0CE0101960E94E0B7A6
:100B8000882341F040E050E160E070E0CE01019642
:100B90000E9496B18F819885892B41F040E050E208
:100BA00060E070E0CE0101960E9496B1D6011296E7
:100BB000CD90DC90CE0101960E94B6B899CF0E94EC
:100BC000D7F980919A1190919B110F94123D8BE867
:100BD0009DE00F94B73E811189C067EC70E288E810
:100BE0009FE00F94082480919A1190919B110F948B
:100BF0005640E0919A11F0919B1181E080838091A1
:100C00009A1190919B110F94644063EB70E28111F3
:100C100002C06EE970E289E390E10F9408248091AC
:100C2000A4119091A511892B09F447CF80919811B7
:100C300090919911892B09F0E2C083E190E00F9423
:100C4000754E8C0180919A1190919B1123EC32E0AA
:100C5000F801328B218B968385831482108289E080
:100C6000818381E08283838310939911009398118B
:100C70000F947F026B017C01F0E1CF0EF7E2DF1EE3
:100C8000E11CF11CD8011596ED91FC9116978FEFA0
:100C90008387148613821482158216821782108627
:100CA0001186128614961C92BB24B394BE01605E1A
:100CB0007F4FF801858196810F943E4118160CF004
:100CC00099C00F947F026C157D058E059F0508F075
:100CD00091C0DE01909698E080E0915039F1ED915D
:100CE000E827F0E0EB52FE4C8491F7CF0F944B4293
:100CF00080919A1190919B110F94123D8BE89DE089
:100D00000F94B73E81110BC061E870E288E89FE064
:100D10000F94E42388E89FE00F94782280CF65E663
:100D200070E282E99FE00F940824C7CE9FA1981338
:100D3000BDCFD8018C91811138C015968D919C91B1
:100D40000F946440BE01605E7F4FF80185819681FB
:100D50000F94374040E064EBD80115968D919C913B
:100D60000F941140F80185809680C4010F94953F3F
:100D7000C4010F94123D67E88BE89DE00F94851D38
:100D800060E88BE89DE00F94851D0E9443FAC40142
:100D90000F94953FA82ED80115968D919C910F9494
:100DA0006440A5FC02C0F801B082AE014F5F5F4F06
:100DB000BE01605E7F4FC8010F94A540D801119617
:100DC000AC9088A1803109F4AFC3BE01605E7F4F53
:100DD000C8010F9414418A1510F5F8018181D801DA
:100DE00011968C93119714968C9114978F5F14968B
:100DF0008C935CCFE0919811F09199111282E0915F
:100E0000A411F091A511E680F7804FE7D42E8091D0
:100E1000A4119091A511892B71F481E04FCE88A186
:100E2000803111F48CE0DBCFBE01605E7F4FC801E2
:100E30000F941441D4CFE114F10479F3BE01605E44
:100E40007F4FF701808191810E949B36882329F38F
:100E50006EE470E289E390E10F94E423D7016D9191
:100E60007C9189E390E10F94CE2389E390E10F9484
:100E700078220091981110919911AE014F5F5F4F48
:100E8000BE01605E7F4FC8010F94FA40882309F4C9
:100E90005EC088A1803109F45AC0DD82F8018581E5
:100EA00096810F946440BE01605E7F4FD801159615
:100EB0008D919C910F94374040E06EE4F80185815C
:100EC00096810F94114040E06B81D80115968D9169
:100ED0009C910F94114040E06C81F80185819681CE
:100EE0000F94114088A1803141F040E06D81D8011C
:100EF00015968D919C910F941140F80185819681F2
:100F00000F946440BE01605E7F4FD80115968D91AD
:100F10009C910F943740F801408168E48581968167
:100F20000F94114064E170E080E090E00F948D0038
:100F3000D8018C91882331F06AE070E080E090E085
:100F40000F948D00F801858196810F946440D7013C
:100F50001296ED90FC905BCF70E060E0CE010196C0
:100F60000E948EB08C01912C812C97FF06C01195A8
:100F70000195110988248394912CCE0101960E9439
:100F8000E0B7E82EF12C8B85853091F0863009F0A2
:100F90000DCEB02E61E0802F0E9448FE61E08928CE
:100FA00009F443C0EA94EF2809F043C060E041C06F
:100FB000EF2829F462E0CE0101960E94C1B740E01B
:100FC00050E160E070E0CE0101960E9496B18F8101
:100FD0009885892B41F040E050E260E070E0CE015E
:100FE00001960E9496B161E0802F0E9448FE60E069
:100FF000802F0E941AFE6CE571E289E390E10F9464
:10100000E4234AE050E0B80189E390E10F9485239E
:1010100067E571E289E390E10F94E42365E571E20D
:1010200089E390E10F94E423C1CDEA94EF2809F01D
:10103000BDCFE62EF12C8B2D0E941AFE60E571E2E9
:1010400089E390E10F94E4234AE050E0B80189E39A
:1010500090E10F9485236EE471E289E390E10F94AF
:10106000E4234AE050E0B70189E390E10F9485233F
:101070006CE471E2D5CFF8018681978190939D1140
:1010800080939C1189E390E10F9478226AE370E2E7
:1010900088E89FE00F94E42388E89FE00F9478228B
:1010A000E091A011F091A111309709F47EC18091D7
:1010B0009E118F5F80939E11C680D7801E01F8E23B
:1010C0002F0E311CC114D10409F46AC1D60118963F
:1010D0008C918F70863009F07FC0D9A6C8A670E0C9
:1010E00060E0C1010E948CD98DA59EA5892B09F4D1
:1010F00073C08091F40A9091F50A892B09F46CC0B1
:1011000008A519A501151105B9F1F80180858F70A1
:10111000863091F519A308A370E060E0CE018096B7
:101120000E948CD9EDA1FEA110821182128213823D
:101130006AEA76E0C8010E943AEDFC01892BE1F0F1
:1011400090859F7095509230B8F4E680F780E11456
:10115000F10491F0FA82E982B801CE0101960E9471
:101160008CD9EE81FF811082118212821382D70105
:101170001296ED90FC90EBCF65E370E289E390E18D
:101180000F94E4234AE050E06BA589E390E10F94CB
:101190009B2263E370E289E390E10F94E4234AE049
:1011A00050E06AA589E390E10F949B2289E390E1E6
:1011B0000F947822EDA5FEA510821182128213826F
:1011C0008AA5853009F4E1C060F4823008F4D1C00A
:1011D00060E0843008F4CEC0D6011296CD90DC9049
:1011E00071CF8032C1F068F48630B1F73C822B8237
:1011F0008CED92E09A838983CE0101960E94426829
:10120000EBCF803409F4BFC060E0823429F78BA5AE
:101210000E9448FEE1CF88A599A5009709F4A9C0CE
:101220002091F40A3091F50A232B09F4A2C0FC01A5
:1012300020852F70263009F09CC06CE079E00E9478
:101240003AED7C01009709F494C0DC0119968D9168
:101250009C911A97892B09F08CC018968C918F70ED
:10126000853009F086C02FEF3FEFA90161E070E003
:10127000C7010F9426476FA74B012FEF3FEFA9013E
:1012800062E070E0C7010F94264768AB5B0121E084
:1012900030E040E050E063E070E0C7010F94264783
:1012A0002B0197FC66C0B7FC64C08BE190E00F9403
:1012B000754E8C01FC0191828082B382A28255829C
:1012C000448262E08FA50E9448FE62E088A90E94E5
:1012D00048FED8018C910E94F1FD8FA7F801828110
:1012E0000E94F1FD880F991FFFA58F2BD80116963C
:1012F0008C931697F80117821086118612861B961A
:101300001D921D921D921C921E971786108A118A9B
:10131000128AD7011A961C930E9319976BE170E20B
:1013200089E390E10F94E4234AE050E0B40189E3BB
:1013300090E10F94852366E778E089E390E10F94CC
:10134000CE234AE050E0B50189E390E10F94852374
:1013500064E170E289E390E10F94E4234AE050E015
:10136000B20189E390E10F94852389E390E10F9422
:10137000782262E08BA50E9448FEEDA5FEA5818142
:10138000807F818329CF62E042CF3C822B82EEEEC8
:10139000F2E0FA83E983CE0101960E94F1681CCF46
:1013A00080919E11815080939E1167E070E288E8E1
:1013B0009FE00F94E4236FEF7FE188E89FE00F94B4
:1013C000E42381E02091A2113091A311232B09F491
:1013D00080E00E94116866EF7FE188E89FE00F944B
:1013E000E42381E02091A0113091A111232B09F475
:1013F00080E00E94116867EE7FE188E89FE00F942B
:10140000E4236CED7FE188E89FE00F94E42381E022
:101410002091890A30918A0A232B09F480E00E94E6
:10142000116865ED7FE188E89FE00F94E42381E097
:101430002091670B3091680B232B09F480E00E9408
:1014400011686CEC7FE188E89FE00F94E42381E071
:101450002091A4113091A511232B09F480E00E9462
:10146000116863EC7FE188E89FE00F94E4238091AA
:101470008D0A0E94116888E89FE00F9478226EEB35
:101480007FE188E89FE00F94E4230E940635AB01DA
:10149000BC012AE030E088E89FE00F94932288E8BE
:1014A0009FE00F94782281E080936C0B87E59FE0AA
:1014B0000F94E133882351F087E59FE00F94993A28
:1014C00084E090E090933B0C80933A0C80913A0C2E
:1014D00090913B0C079731F484E090E090933B0CA3
:1014E00080933A0C80919E11815080939E1180913F
:1014F0006C0BE0960FB6F894DEBF0FBECDBFDF9148
:10150000CF911F910F91FF90EF90DF90CF90BF9000
:10151000AF909F908F907F906F905F904F903F9093
:101520002F90089580E0E5CFBCE0BA1508F455CCC3
:1015300079CC8F929F92AF92BF92CF92DF92EF922F
:10154000FF920F931F93CF93DF93CDB7DEB7CF55A5
:10155000D1090FB6F894DEBF0FBECDBF8C016B0171
:101560006115710519F04115510579F56CE378E1C4
:1015700089E390E10F94E42363E378E189E390E168
:101580000F94E423B80189E390E10F94CE2361E343
:1015900078E189E390E10F94E42389E390E10F94EB
:1015A0007822C15ADF4F0FB6F894DEBF0FBECDBF11
:1015B000DF91CF911F910F91FF90EF90DF90CF902F
:1015C000BF90AF909F908F900895460F571FDA01FC
:1015D0001C920E9406354B016BE278E189E390E1B1
:1015E0000F94E4234AE050E0B40189E390E10F94C2
:1015F000852368E278E189E390E10F94E423B80160
:1016000089E390E10F94CE2365E278E189E390E1EC
:101610000F94E423BAE38B16B1E09B064CF468E127
:1016200078E182E99FE00F94E42382E99FE0B7CF5D
:1016300066E178E189E390E10F94E423B60189E360
:1016400090E10F94CE2364E178E189E390E10F9477
:10165000E42389E390E10F9478221A821982FE0133
:1016600033968EE3DF011D928A95E9F780913A0C5B
:1016700090913B0C059791F563E070E0C8010E94E2
:10168000C56D7C01892BD1F5E091B50DF091B60DBA
:10169000808180FF86CF61E070E0C8010E94C56D47
:1016A000892B09F47ECF64E270E0C8010F940E5DCF
:1016B000892B09F076CF66EF77E189E390E10F940B
:1016C000E423B80189E390E10F94CE2389E390E10C
:1016D0000F947822C8010E94FFFC63CF61E070E0A4
:1016E000C8010E94C56D7C01892B09F465C04FE3D8
:1016F00050E0B801CE0101960F94FF5CA12CBB24F1
:10170000B394E00EF11E6DEE77E1C7010F94AE5079
:10171000892B09F45EC064E270E0C8010F940E5D8D
:10172000892B09F03ECFB11003C0AA2009F439CFAC
:101730004091A2115091A311B701CE018F5B9F4F31
:101740000E942CB8CE018F5B9F4F0E9471AF182F63
:10175000882359F0B601CE018F5B9F4F0E942FF670
:1017600011E0181619060CF010E0CE018F5B9F4FA8
:101770000E94B6B8112309F414CF8981882309F493
:1017800010CF80913A0C90913B0C059709F409CF4A
:101790006FEC77E189E390E10F94E423BE016F5F82
:1017A0007F4F89E390E10F94CE2389E390E10F947A
:1017B0007822CE0101968FCF62E070E0C8010E94CE
:1017C000C56D7C01892B09F4ECCEAA24A394B12C1D
:1017D00098CFF60101900020E9F73197EC19FD0947
:1017E000329708F498CFC8010E94FFFCB11003C0E3
:1017F000AA2009F4D6CEF6018081882309F4D1CE3F
:10180000C6010F94052BCDCEEF92FF920F931F933D
:10181000CF93DF93CDB7DEB76F970FB6F894DEBFE7
:101820000FBECDBF2091F40A3091F50A232B09F4A5
:1018300053C120919E11022E000C330B8217930787
:10184000C4F468EB77E182E99FE00F94E42382E936
:101850009FE00F94782280E06F960FB6F894DEBF79
:101860000FBECDBFDF91CF911F910F91FF90EF90F1
:10187000089562EA77E189E390E10F94E42389E334
:1018800090E10F9478228091F60A8F5F8093F60A98
:101890006DE577E188E89FE00F94E42388E89FE016
:1018A0000F947822E091A011F091A111309709F4E2
:1018B0005BC080919E118F5F80939E11068117817E
:1018C0000115110509F44BC0D80118968C918F7041
:1018D000863009F03FC01A83098370E060E0CE01D2
:1018E00001960E948CD989819A81009799F1209163
:1018F000F40A3091F50A232B69F1FC0120852F7041
:10190000263041F56CE079E00E943AED7C018B8154
:10191000803201F5E114F104E9F0D70119962D9117
:101920003C911A9721153105A9F018969C919F704A
:10193000953081F4C9010F94114FF7011286118679
:1019400061E577E189E390E10F94E42389E390E195
:101950000F947822D80112960D911C91B1CF8091ED
:101960009E11815080939E11E091A211F091A311DC
:10197000309799F10681178101151105C1F1F80120
:1019800080858F70853029F5C8010E947DEE8823FF
:1019900001F14091A2115091A311D8016D917C9158
:1019A000CE0101960E942CB8CE0101960E9471AF23
:1019B000882359F08C859D85009739F0DC01ED91E5
:1019C000FC910084F185E02D1995CE0101960E94CD
:1019D000B6B8F80102811381CFCF62E977E189E3DC
:1019E00090E10F94E42389E390E10F947822109220
:1019F0009D1110929C116AE877E189E390E10F94C0
:101A0000E42389E390E10F94782264E670E080E0BB
:101A100090E00F948D0010928D0A10926C0B62E78B
:101A200077E189E390E10F94E4230E940635AB014E
:101A3000BC012AE030E089E390E10F949322809189
:101A4000F40A9091F50A009711F00E94B0FA1092F2
:101A5000F50A1092F40A1092A1111092A01110929E
:101A6000A3111092A2111092910A1092900A109252
:101A70006B0B10926A0B1092680B1092670B10920E
:101A80008F0A10928E0A1092690B1092F30A10922C
:101A9000F20A1092A5111092A41110928A0A1092C3
:101AA000890A6DE677E189E390E10F94E4230E94CF
:101AB0000635AB01BC012AE030E089E390E10F94E8
:101AC000932289E390E10F9478221092630B809126
:101AD000F60A81508093F60A81E0BECE4F925F9263
:101AE0006F927F928F929F92AF92BF92CF92DF922E
:101AF000EF92FF920F931F93CF93DF93CDB7DEB793
:101B0000C659D1090FB6F894DEBF0FBECDBF8E0106
:101B10000F5B1F4FD8011D921C92FE01ED5BFF4F22
:101B20008EE1DF011D928A95E9F78091640F909113
:101B3000650F892B09F4FEC10E948DEE882309F4FC
:101B4000F9C1A091640FB091650F52961C921E923C
:101B5000519754961C921E92539784E890E01D96DC
:101B60009C938E931C971E961C921E9782E7559607
:101B70008C935597ED91FC9111970088F189E02D98
:101B800060E270E0CD0119954FE150E0B80180911D
:101B9000640F9091650F0E94E2EE7C018091640FCA
:101BA0009091650FDC01ED91FC910488F589E02DA1
:101BB0001995E114F10409F4BDC1F801EE0DFF1D02
:101BC00010828091710F1F928F938091700F1F92DE
:101BD0008F9380916F0F1F928F9380916E0F1F9242
:101BE0008F9380916D0F1F928F9380916C0F1F9236
:101BF0008F9388E798E09F938F931F9280E48F9351
:101C0000FE0131966F01FF93EF930F94195D6BEE18
